:100000000C94D30A0C94000B0C94000B0C94000B72
:100010000C94000B0C94000B0C94000B0C94000B34
:100020000C94000B0C94000B0C94000B0C94000B24
:100030000C94000B0C94000B0C94000B0C94000B14
:100040000C94000B0C940E790C94000B0C94000B88
:100050000C94000B0C94000B0C9467830C94FE948E
:100060000C94000B0C94951A0C94000B0C94000B40
:100070000C94000B0C94000B0C94000B0C94000BD4
:100080000C94DE490C94000B0C94000B0C94000BA8
:100090000C94000B0C94000B0C94000B0C946993C3
:1000A0000C94000B0C94000B0C94B1490C94000BB5
:1000B0000C94000B0C94000B0C94000B0C948449D2
:1000C0000C94000B0C94000B0C94000B0C94000B84
:1000D0000C94000B0C94000B0C94000B0C94000B74
:1000E0000C94000B084AD73B3BCE016E84BCBFFD8D
:1000F000C12F3D6C74319ABD56833DDA3D00C77FF8
:1001000011BED9E4BB4C3E916BAAAABE0000008090
:100110003F05A84CCDB2D44EB93836A9020C50B91F
:10012000918688083CA6AAAA2ABE000000803F65E6
:1001300063686F3A0048617264636F646564204469
:10014000656661756C742053657474696E6773209D
:100150004C6F616465640053746F726564207365ED
:100160007474696E6773207265747269657665640C
:10017000002044002049002020204D333031205001
:10018000005049442073657474696E67733A0020A7
:100190005A0020590020204D323036205800486F38
:1001A0006D65206F666673657420286D6D293A0051
:1001B000204500205A0020580020420020540020F2
:1001C000204D323035205300416476616E636564A2
:1001D000207661726961626C65733A20533D4D69A6
:1001E0006E20666565647261746520286D6D2F737D
:1001F000292C20543D4D696E2074726176656C2007
:10020000666565647261746520286D6D2F73292C95
:1002100020423D6D696E696D756D207365676D6512
:100220006E742074696D6520286D73292C20583DEB
:100230006D6178696D756D205859206A65726B2003
:10024000286D6D2F73292C20205A3D6D6178696DC2
:10025000756D205A206A65726B20286D6D2F732989
:100260002C2020453D6D6178696D756D2045206AB3
:1002700065726B20286D6D2F73290020540020209B
:100280004D323034205300416363656C6572617494
:10029000696F6E3A20533D616363656C657261748A
:1002A000696F6E2C20543D726574726163742061B5
:1002B0006363656C65726174696F6E002045002030
:1002C0005A0020590020204D3230312058004D6115
:1002D00078696D756D20416363656C6572617469E1
:1002E0006F6E20286D6D2F7332293A002045002053
:1002F0005A0020590020204D3230332058004D61E3
:1003000078696D756D2066656564726174657320CA
:10031000286D6D2F73293A00204500205A0020597E
:100320000020204D393220580053746570732070BE
:10033000657220756E69743A0053657474696E67EE
:10034000732053746F726564006563686F3A00458B
:1003500072726F723A005072696E746572207374B3
:100360006F707065642064756520746F20657272AB
:100370006F72732E204669782074686520657272EA
:100380006F7220616E6420757365204D3939392094
:10039000746F20726573746172742E202854656DB9
:1003A000706572617475726520697320726573651A
:1003B000742E205365742069742061667465722000
:1003C00072657374617274696E6729005072696E28
:1003D0007465722068616C7465642E206B696C6C46
:1003E00028292063616C6C656421006F6B00526585
:1003F00073656E643A20002200556E6B6E6F776EE7
:1004000020636F6D6D616E643A2022005A204F6642
:1004100066736574203A20007A5F6D61783A200037
:100420007A5F6D696E3A20005A204F666673657474
:10043000005A204F6666736574206F6B007A5F6D9B
:1004400061783A20007A5F6D696E3A2000795F6DBD
:1004500061783A2000795F6D696E3A2000785F6DAF
:1004600061783A2000785F6D696E3A2000205A3A30
:100470000020593A0020436F756E7420583A2000CE
:1004800020453A00205A3A0020593A00583A00468E
:1004900049524D574152455F4E414D453A4D61726B
:1004A0006C696E2056313B20537072696E746572B0
:1004B0002F6772626C206D617368757020666F7251
:1004C0002067656E36204649524D574152455F556B
:1004D000524C3A68747470733A2F2F676974687558
:1004E000622E636F6D2F4572696B5A616C6D2F4D73
:1004F00061726C696E2F2050524F544F434F4C5FC6
:1005000056455253494F4E3A312E30204D414348C3
:10051000494E455F545950453A4D656E64656C20AF
:1005200045585452554445525F434F554E543A3105
:1005300020555549443A30303030303030302D304D
:100540003030302D303030302D303030302D3030B4
:10055000303030303030303030300A0020423A0015
:1005600020453A00543A0020573A0020453A0054BA
:100570003A002042403A0020403A00202F003A0042
:10058000205400202F0020423A00202F006F6B20C3
:10059000543A002569206D696E2C20256920736509
:1005A00063000A00205A3A200020593A20002058BF
:1005B0003A20004265640050726F62696E67206481
:1005C0006F6E65210020643A200020623A200045C9
:1005D000716E20636F656666696369656E74733AF0
:1005E00020613A2000486F6D6520582F59206265C0
:1005F000666F7265205A00FFFF010000254300006E
:10060000394300002043000000000000000000000B
:100610002043000000000000000000000000000077
:10062000254300003943000020430000A0400000A3
:10063000A040000000400A00207A3A200020793AC9
:10064000200020783A2000426564005072696E7480
:1006500065722073746F70706564206475652074B2
:100660006F206572726F72732E20466978207468ED
:1006700065206572726F7220616E642075736520EB
:100680004D39393920746F20726573746172742E1C
:10069000202854656D706572617475726520697388
:1006A0002072657365742E2053657420697420610F
:1006B000667465722072657374617274696E6729FD
:1006C000006F6B004E6F204C696E65204E756D6239
:1006D0006572207769746820636865636B73756DF4
:1006E0002C204C617374204C696E653A20004E6F6B
:1006F00020436865636B73756D2077697468206C3F
:10070000696E65206E756D6265722C204C61737424
:10071000204C696E653A2000636865636B73756D84
:10072000206D69736D617463682C204C6173742053
:100730004C696E653A20004C696E65204E756D629D
:100740006572206973206E6F74204C617374204C45
:10075000696E65204E756D6265722B312C204C617F
:100760007374204C696E653A20004D3131300020A1
:1007700020506C616E6E6572427566666572427974
:100780007465733A20002046726565204D656D6F73
:1007900072793A20004E6F76203139203230313470
:1007A00000436F6D70696C65643A200028416C6588
:1007B0007068204F626A6563747320496E632C20F1
:1007C0004D696E692D3230313451342900207C203E
:1007D000417574686F723A20004E6F76203139206F
:1007E000323031342031313A32383A313300204C12
:1007F00061737420557064617465643A2000312E11
:10080000302E30004D61726C696E0020536F66743B
:100810007761726520526573657400205761746357
:1008200068646F67205265736574002042726F7749
:100830006E206F757420526573657400204578745E
:1008400065726E616C20526573657400506F7765D8
:10085000725570007374617274002200656E717558
:1008600065696E672022002200656E717565696E8C
:10087000672022006563686F3A0020746F6F206CF8
:100880006F6E6720657874727573696F6E20707211
:100890006576656E7465640020636F6C64206578AE
:1008A00074727573696F6E2070726576656E7465AB
:1008B000640045313A200045303A20005A3A200081
:1008C000593A2000583A20004D53312C4D533220D4
:1008D00050696E730A0024F404D9201BC40C5C0E0A
:1008E0009804C4095F0265077101F405F900FB046F
:1008F000B30048048700C10369005803550003038F
:100900004500BE023A008402310053022A00290247
:10091000250004022000E4011C00C8011900AF01F9
:100920001700980114008401130071011000610187
:10093000100051010E0043010D0036010B002B0188
:100940000B0020010B00150109000C010900030137
:100950000800FB000800F3000800EB000700E400BB
:100960000600DE000600D8000600D2000600CC001B
:100970000500C7000500C2000500BD000400B90065
:100980000400B5000400B1000400AD000400A9009B
:100990000400A5000300A20003009F0004009B00C8
:1009A00003009800030095000200930003009000EC
:1009B00003008D0002008B00030088000200860007
:1009C000020084000300810002007F0002007D001D
:1009D00002007B000200790002007700010076002F
:1009E00002007400020072000100710002006F003A
:1009F00002006D0001006C0002006A000100690045
:100A0000020067000100660001006500010064004B
:100A100002006200010061000100600001005F004F
:100A200002005D0001005C0001005B0001005A0053
:100A30000100590001005800010057000100560054
:100A40000100550001005400010053000000530054
:100A500001005200010051000100500001004F0050
:100A600001004E0000004E0001004D0001004C004E
:100A700001004B0000004B0001004A00010049004A
:100A80000100480000004800010047000100460046
:100A90000000460001004500000045000100440040
:100AA000010043000000430001004200000042003A
:100AB00001004100000041000100400001003F0032
:100AC00000003F0001003E0000003E0001003D002C
:100AD00000003D0001003C0000003C0000003C0024
:100AE00001003B0000003B0001003A0000003A001A
:100AF0000100390000003900010038000000380012
:100B00000000380001003700000037000100360007
:100B100000003600000036000100350000003500FE
:100B200000003500010034000000340000003400F3
:100B300001003300000033000000330001003200E8
:100B400000003200000032000100310000003100DE
:100B500000003100010030000000300000003000D3
:100B600001002F0000002F0000002F0000002F00C8
:100B700001002E0000002E0000002E0001002D00BC
:100B800000002D0000002D0000002D0001002C00B1
:100B900000002C0000002C0000002C0001002B00A5
:100BA00000002B0000002B0000002B0001002A0099
:100BB00000002A0000002A0000002A00010029008D
:100BC0000000290000002900000029000000290081
:100BD0000100280000002800000028000000280074
:100BE0000000280001002700000027000000270067
:100BF000000027000000270001002600000026005A
:100C0000000026000000260000002600010025004C
:100C10000000250000002500000025000000250040
:100C20000000250001002400000024000000240032
:100C30000000240000002400010023000000230025
:100C40000000230000002300000023000000230018
:100C5000000023000100220000002200000022000A
:100C600000002200000022000000220001002100FC
:100C700000002100000021000000210000002100F0
:100C800000002100000021000100200000002000E1
:100C900000002000000020000000200000002000D4
:100CA000000020000000200001001F0000001F00C5
:100CB00000001F0000001F0000001F0000001F00B8
:100CC00000001F0001001E0000001E0000001E00AA
:100CD00000001E00000024F4D43050C38E20C2A2B5
:100CE0004017828B7011127A910D816CD90AA8611C
:100CF000E108C7586607615143061E4B5D05C145B3
:100D0000A7041A411104093D980371393103403693
:100D1000DB0265339102D4305402802E1D02632C15
:100D2000EE01752AC501B028A001102781018F2589
:100D300064012B244B01E0223401AC211F018D20E2
:100D40000D01801FFC00841EED00971DDF00B81C04
:100D5000D200E61BC600201BBC00641AB200B21908
:100D6000A8000A19A0006A189900D117910040172D
:100D70008B00B516840031167E00B31579003A1544
:100D80007300C7146F0058146A00EE1366008813CE
:100D9000630025135E00C7125B006C12570015122A
:100DA0005400C111510070114F0021114B00D61099
:100DB00049008D1047004610440002104200C00F49
:100DC0004000800F3E00420F3C00060F3B00CB0E60
:100DD0003800930E37005C0E3500270E3400F30DFB
:100DE0003200C10D3100900D3000600D2E00320D2B
:100DF0002D00050D2C00D90C2B00AE0C2900850C04
:100E000029005C0C2700350C27000E0C2600E80B8F
:100E10002400C40B2400A00B23007D0B23005A0BDD
:100E20002100390B2100180B2000F80A1F00D90AF5
:100E30001E00BB0A1E009D0A1D00800A1D00630AD9
:100E40001C00470A1B002C0A1B00110A1A00F70994
:100E50001A00DD091900C4091900AB09190092092B
:100E600017007B091800630917004C0916003609A2
:100E70001600200916000A091500F5081500E008FB
:100E80001400CC081400B8081400A408140090083A
:100E900013007D0812006B08130058081200460862
:100EA0001200340811002308110012081100010873
:100EB0001100F0071000E0071000D0071000C00775
:100EC0001000B0070F00A107100091070E00830764
:100ED0000F0074070F0065070E0057070E00490743
:100EE0000E003B070D002E070E0020070D00130714
:100EF0000D0006070D00F9060C00ED060D00E006DA
:100F00000C00D4060C00C8060C00BC060C00B00691
:100F10000C00A4060B0099060C008D060B0082063F
:100F20000B0077060B006C060B0061060A005706E3
:100F30000B004C060A0042060A0038060A002E067C
:100F40000A0024060A001A060A001006090007060D
:100F50000A00FD050900F4050900EB050900E2059A
:100F60000900D9050900D0050900C7050900BE051B
:100F70000900B5050800AD050800A50509009C0598
:100F80000800940508008C050800840508007C050D
:100F90000800740508006C050700650508005D057C
:100FA0000700560508004E050700470507004005E5
:100FB000080038050700310507002A05070023054A
:100FC00007001C050600160507000F0507000805A9
:100FD000060002050700FB040600F5040700EE0406
:100FE0000600E8040600E2040700DB040600D5045E
:100FF0000600CF040600C9040600C3040600BD04B1
:101000000600B7040600B1040500AC040600A604FF
:101010000600A00405009B0406009504050090044A
:1010200006008A04050085040500800406007A0491
:10103000050075040500700405006B0405006604D6
:101040000500610405005C04050057040500520416
:1010500005004D04050048040500430405003E0456
:1010600004003A04050035040500300404002C0493
:10107000050027040400230405001E0404001A04CC
:10108000040016040500110404000D040400090402
:1010900005000404040000040400FC030400F80339
:1010A0000400F4030400F0030400EC030400E8036C
:1010B0000400E4030400E0030400DC030400D8039C
:1010C0000400D4030400D0030400CC030400C803CC
:1010D0000300C50303006563686F3A00205A3A00B5
:1010E00020593A0020583A00656E6473746F70732B
:1010F000206869743A20004572726F723A00546534
:101100006D7065726174757265206865617465647F
:1011100020626564207377697463686564206F6614
:10112000662E204D415854454D50207472696767B2
:1011300065726564202121003A20457874727564D7
:101140006572207377697463686564206F66662EC4
:10115000204D494E54454D50207472696767657241
:1011600065642021003A20457874727564657220A8
:101170007377697463686564206F66662E204D41DD
:101180005854454D502074726967676572656420D4
:101190002100202D20496E76616C69642065787489
:1011A0007275646572206E756D6265722021001023
:1011B00000AD0330016A0150022B0170030A019057
:1011C00004F500B005E500D006D800F007CE001009
:1011D00009C500300ABE00500BB700700CB100907A
:1011E0000DAB00B00EA600D00FA200F0109D0010B5
:1011F000129900301395005014920070158E0090D3
:10120000168B00B0178700D0188400F019810010E9
:101210001B7E00301C7B00501D7900701E760090F4
:101220001F7300B0207000D0216E00F0226B001000
:101230002469003025660050266300702761009005
:10124000285E00B0295C00D02A5900F02B5600100F
:101250002D5400302E5100502F4E0070304B009016
:10126000314800B0324500D0334200F0343E001027
:10127000363B00303737005038330070392E00903D
:101280003A2900B03B2300D03C1B00F03D11001078
:101290003F0100F03F0000504944204175746F74D5
:1012A000756E652066696E69736865642120507586
:1012B0007420746865204B702C204B6920616E642B
:1012C000204B6420636F6E7374616E747320696E5B
:1012D000746F20436F6E66696775726174696F6EB3
:1012E0002E6800504944204175746F74756E6520F6
:1012F0006661696C6564212074696D656F75740041
:1013000020403A006F6B20543A006F6B20423A0045
:10131000504944204175746F74756E65206661692B
:101320006C6564212054656D7065726174757265B9
:1013300020746F6F206869676800204B643A200052
:10134000204B693A2000204B703A200020436C610A
:101350007369632050494420002054753A200020CE
:101360004B753A2000206D61783A2000206D696E3F
:101370003A200020643A200020626961733A20001C
:101380001000C90210012C01400122017001180156
:10139000B0010E01F00104015002FA00B002F000A9
:1013A0003003E600D003DC009004D2007005C800D2
:1013B000A006BE000008B400B009AA00D00BA0002F
:1013C000600E960060118C000015820020197800D4
:1013D000C01D6E00A0226400B0275A00902C50005F
:1013E00000314600E0343C0010383200903A2800CA
:1013F000603C1E00A03D1400803E0A00203F00001B
:101400000A0020000A00207A3A200020793A2000C1
:1014100020783A200000002100240027002A002D17
:10142000003000330001010000040107010A01003F
:10143000002200250028002B002E0031003400027D
:10144000010000050108010B010000200023002617
:101450000029002C002F00320000010000030106CB
:10146000010901050505050705080808080202022B
:10147000020A0A080804040404010101010101012F
:10148000010303030303030303040707070C0C0C06
:101490000C0C0C0C0C0202020206060606060606DE
:1014A000060B0B0B0B0B0B0B0B07070A0A0A0A0A9E
:1014B0000A05050504040408080102102020080894
:1014C00010204010204080020102010804020101A6
:1014D000020408102040808040201008040201808F
:1014E00004020180402010080402010804020101E6
:1014F00002040810204080010204081020408010DF
:10150000080408801020400440801020400480001F
:1015100000090A02080B0C0D070603040100000075
:1015200000000000000000000000000000000000BB
:10153000000000000000000000000011100F00007B
:10154000000000000000000000000000000000009B
:10155000000000000000000000000000000000008B
:101560000000000000494E46494E4954594E414E34
:10157000CDCCCC3D0AD7233C17B7D13877CC2B3212
:101580009595E6241FB14F0A000020410000C84293
:1015900000401C4620BCBE4CCA1B0E5AAEC59D74F2
:1015A000291B791DD89211241FBECFEFD1E2DEBFD7
:1015B000CDBF00E00CBF14E0A0E0B2E0EEE5FBE33D
:1015C00001E00BBF02C007900D92AA3AB107D9F70C
:1015D0001BBE1EE0AAEAB4E001C01D92A23EB10704
:1015E000E1F715E1C6EAD5E104C02297FE010E94A9
:1015F000679DC03AD107C9F70E9401980C94AD9D30
:101600000C940000CF93DF93BC018230910510F45D
:1016100062E070E0A091DE0EB091DF0EED0140E0DF
:1016200050E0E0E0F0E021C08881998186179707BB
:1016300069F48A819B81309719F09383828304C077
:101640009093DF0E8093DE0EFE0134C06817790799
:1016500038F44115510519F08417950708F4AC01C9
:10166000FE018A819B819C01E9012097E9F64115E1
:101670005105A9F1CA01861B970B049708F4BA011A
:10168000E0E0F0E02AC08D919C91119784179507B6
:10169000F9F46417750781F412968D919C91139754
:1016A000309719F09383828304C09093DF0E809368
:1016B000DE0EFD0132964CC0CA01861B970BFD0160
:1016C000E80FF91F6193719302978D939C9340C02B
:1016D000FD01828193819C01D9011097A1F680912F
:1016E000DC0E9091DD0E892B41F480917D03909169
:1016F0007E039093DD0E8093DC0E40917F0350912A
:1017000080034115510541F44DB75EB780917B03CD
:1017100090917C03481B590B2091DC0E3091DD0E1B
:10172000CA01821B930B8617970780F0AB014E5FAF
:101730005F4F8417950750F0420F531F5093DD0EF3
:101740004093DC0EF9016193719302C0E0E0F0E098
:10175000CF01DF91CF910895CF93DF93009709F4E4
:1017600050C0EC0122971B821A82A091DE0EB0912C
:10177000DF0E109709F140E050E0AC17BD0708F10B
:10178000BB83AA83FE0121913191E20FF31FAE17B3
:10179000BF0779F48D919C911197280F391F2E5F07
:1017A0003F4F3983288312968D919C9113979B8389
:1017B0008A834115510571F4D093DF0EC093DE0E7C
:1017C00020C012968D919C911397AD01009711F056
:1017D000DC01D3CFFA01D383C28321913191E20F8F
:1017E000F31FCE17DF0769F488819981280F391F0D
:1017F0002E5F3F4FFA01318320838A819B8193833F
:101800008283DF91CF910895A0E0B0E0EAE0FCE0B0
:101810000C947C9DEC015B016115710519F0FB01D5
:1018200091838083F9908F2D90E00E946B9D892B8E
:10183000C9F7FDE2FF1621F4F990EE24E39405C008
:101840002BE2F21609F4F990EE248E0101501040BB
:10185000C80165E675E143E050E062D2892BF9F4F6
:101860008E010E5F1F4FC80168E675E145E050E04C
:1018700057D2892B19F48E01095F1F4FA114B104AF
:1018800019F0F50111830083E0FC04C070E090E0E2
:1018900080E813C070E090E080E86FEF07C1C801F6
:1018A0006DE675E143E050E03BD2892B69F4A11469
:1018B000B10429F470E090E080EC6FE7F7C0229665
:1018C000F501D183C083F6CF8824992440E050E00D
:1018D00060E070E0EF2DE053EA30A0F5F2E0EF2A8F
:1018E0008E2D90E09C0128703070E2FE06C0232B04
:1018F00079F50894811C911C2BC0232B19F00894B6
:1019000081089108DB01CA0112E0880F991FAA1F04
:10191000BB1F1A95D1F7480F591F6A1F7B1F440F31
:10192000551F661F771F4E0F511D611D711D4839D0
:1019300029E9520729E9620729E1720748F084E0A2
:10194000E82A06C0EE3F31F4E3FC39C098E0E92A0A
:10195000F990C0CFE53311F0E53189F529912D32A9
:1019600019F4E0E1EE2A05C02B3219F081E090E095
:1019700003C0299182E090E0E22FE053EA3018F0B2
:10198000C81BD90B1CC020E030E0FCE020383F072A
:101990005CF4C901880F991F880F991F280F391F00
:1019A000220F331F2E0F311DE991E053EA3068F307
:1019B000E4FE03C0309521953F4F820E931ECE2C3E
:1019C000DD24E1FE07C0A114B10421F02197F50147
:1019D000D183C083CB01BA010E94D0997B018C01D5
:1019E000F3E0CF22DD2423E0C216D10421F417FB5B
:1019F000109517F9109557016801C801B70120E04B
:101A000030E040E050E00E943099882309F44AC059
:101A100097FE0DC024E8E22E25E1F22E90948194E9
:101A200091089394C0E2D0E000E010E012C09CE97D
:101A3000E92E95E1F92EF6CFF701259135914591E3
:101A40005491C601B5010E94109C5B016C018C1A77
:101A50009D0A8C169D0684F7D595C7950F5F1F4F7D
:101A60000630110529F08CEF9FEFE80EF91EF1CF3B
:101A7000C501D6017C018D018C2D880F8D2D881F0D
:101A80008F3F51F0C601B50120E030E040E050E06A
:101A90000E943099882331F482E290E09093E10E25
:101AA0008093E00E7E2D9F2D802F612F272F392FC1
:101AB000482F562FB901CA01CDB7DEB7ECE00C9420
:101AC000989D2F923F925F926F927F928F929F92FA
:101AD000AF92BF92CF92DF92EF92FF920F931F933C
:101AE000CF93DF938C011B01EA016115710519F099
:101AF000FB0191838083209749F0CE010297839761
:101B000028F020E030E040E050E0F6C0F801A1907D
:101B10008F018A2D90E00E946B9D892BB9F7FDE221
:101B2000AF1631F4F801A1908F015524539407C0EA
:101B3000FBE2AF1619F4F801A1908F01552420970C
:101B400019F0C031D105C1F4F0E3AF1679F4F80112
:101B50008081883711F0883549F4F801A1800E5F43
:101B60001F4FF2E05F2AC0E1D0E006C0209721F4C9
:101B700080E3A816E9F427C0C830D10531F1C93097
:101B8000D10524F4C230D10531F50CC0CA30D105DD
:101B900089F0C031D105F9F4C12CD12CE12CB8E089
:101BA000FB2E28C0C12CD12CE12CA0E4FA2E22C09F
:101BB000CAE0D0E0FCECCF2EFCECDF2EFCECEF2EEC
:101BC000FCE0FF2E17C0C8E0D0E0C12CD12CE12CE6
:101BD000E0E1FE2E0FC09E01442737FD4095542FB3
:101BE00060E070E080E090E80E94289DC901DA0181
:101BF0006C017D0120E030E040E050E060E03E011B
:101C0000882477FC8094982C70EDB72EBA0CE9E00C
:101C1000EB1570F48A2D81548A3118F499ECB92EA1
:101C200006C08A2D81568A3150F589EAB82EBA0C41
:101C30008B2D90E08C179D0714F56F3FE1F0C216D5
:101C4000D306E406F506B0F0CA01B901A401930178
:101C50000E94E29C9B01AC012B0D311D411D511DC9
:101C60002130F0E03F07F0E04F07F0E85F0710F4A5
:101C700061E001C06FEFF801A1908F01C5CF211481
:101C8000310481F0662331F001501040F1011183DD
:101C9000008308C051FE1AC002501040F1011183A8
:101CA000008314C067FF12C050FC05C02FEF3FEF48
:101CB0004FEF5FE704C020E030E040E050E882E210
:101CC00090E09093E10E8093E00E16C050FE08C0A5
:101CD00050954095309521953F4F4F4F5F4F0CC029
:101CE00057FF0AC082E290E09093E10E8093E00EED
:101CF0002FEF3FEF4FEF5FE7B901CA01DF91CF91BF
:101D00001F910F91FF90EF90DF90CF90BF90AF9019
:101D10009F908F907F906F905F903F902F9008954D
:101D2000FB01DC014150504088F08D9181341CF062
:101D30008B350CF4805E659161341CF06B350CF4CE
:101D4000605E861B611171F3990B0895881BFCCFAF
:101D5000FB0155915523A9F0BF01DC014D914517B9
:101D60004111E1F759F4CD010590002049F04D9162
:101D700040154111C9F3FB014111EFCF81E090E023
:101D800001970895FC018191861721F08823D9F7E6
:101D9000992708953197CF010895FB01DC018D91BA
:101DA000019080190110D9F3990B0895FB01DC0112
:101DB0004150504030F08D910190801919F400206D
:101DC000B9F7881B990B0895AEE0B0E0EAEEFEE0AB
:101DD0000C94849D0E891F898EE08C831A8309835D
:101DE0008FEF9FE79E838D839E01265E3F4FCE013E
:101DF0000196688D798DA9010AD02F813885020F4F
:101E0000131FF80110822E96E4E00C94A09DABE025
:101E1000B0E0EDE0FFE00C94769D3C012B015A010F
:101E2000FC0117821682838181FD03C06FEF7FEF73
:101E3000B9C19AE0892E1E010894211C311CF301BE
:101E40002381F20123FD859123FF81912F018823B6
:101E500009F4A5C1853239F423FD859123FF8191D1
:101E60002F01853221F490E0B301B7D1E8CF982F4C
:101E7000FF24EE249924FFE1FF15D0F09B3269F096
:101E80009C3228F4903259F0933291F40EC09D3276
:101E900049F0903369F441E024C052E0F52A84E02F
:101EA000F82A28C098E0F92A25C0E0E1FE2A22C0DD
:101EB000F7FC29C0892F80538A3070F4F6FE05C0E4
:101EC000989C902C1124980E15C0E89CE02C1124AD
:101ED000E80EF0E2FF2A0EC09E3229F4F6FC5FC144
:101EE00040E4F42A07C09C3619F450E8F52A02C0F1
:101EF000983649F4F20123FD959123FF91912F012A
:101F0000992309F0B8CF892F8554833018F0805277
:101F1000833038F444E050E0A40EB51E5FE35983EB
:101F20000FC0933631F0933779F0933509F052C0F2
:101F30001FC0F5018081898342E050E0A40EB51EE8
:101F4000610101E010E011C0F501C080D180F6FC14
:101F500003C06FEF7FEF02C0692D70E042E050E0F8
:101F6000A40EB51EC6012ED18C015FE7F52213C069
:101F7000F501C080D180F6FC03C06FEF7FEF02C097
:101F8000692D70E042E050E0A40EB51EC6010FD1ED
:101F90008C0150E8F52AF3FE06C018C080E290E0FC
:101FA000B3011BD1EA948E2D90E008171907B0F306
:101FB0000DC0F601F7FC8591F7FE81916F0190E06D
:101FC000B3010BD1E110EA94015010400115110545
:101FD00081F7E2C0943611F0993661F5F7FE08C03A
:101FE000F501208131814281538184E090E00AC073
:101FF000F501808191819C01442737FD4095542F44
:1020000082E090E0A80EB91E9FE6F92257FF09C0B2
:1020100050954095309521953F4F4F4F5F4FE0E8E9
:10202000FE2ACA01B901A1012AE030E002D1D82E6E
:10203000D2183FC0953729F41F2D1F7E2AE030E0CB
:102040001DC01F2D197F9F3661F0903720F4983501
:1020500009F0A5C00FC0903739F0983709F09FC03C
:1020600004C028E030E00AC0106114FD146020E1D3
:1020700030E004C014FD166020E132E017FF08C014
:10208000F501608171818281938144E050E008C054
:10209000F50180819181BC0180E090E042E050E058
:1020A000A40EB51EA101C5D0D82ED2188FE7F82EE8
:1020B000F122F6FE0BC05EEFF522D91438F4F4FEDF
:1020C00007C0F2FC05C08FEEF82202C01D2D01C032
:1020D000192DF4FE0DC0FE01ED0DF11D8081803340
:1020E00019F499EEF92208C01F5FF2FE05C003C083
:1020F0008F2D867809F01F5F0F2DF3FC13C0F0FEC3
:102100000EC01E1510F09D2C0AC09D2C9E0C911A1D
:102110001E2D05C080E290E0B3015FD01F5F1E1549
:10212000C8F304C01E1510F4E11A01C0EE2404FF28
:102130000EC080E390E0B30150D002FF1BC001FD50
:1021400003C088E790E00EC088E590E00BC0802FC8
:10215000867881F001FF02C08BE201C080E2F7FCCB
:102160008DE290E0B30139D005C080E390E0B30187
:1021700034D09A94D914C8F3DA94F101ED0DF11D1D
:10218000808190E0B30129D0DD20B1F705C080E265
:1021900090E0B30122D0EA94EE20C9F750CEF301CB
:1021A00066817781CB012B96E2E10C94929DFC0134
:1021B0000590615070400110D8F7809590958E0F72
:1021C0009F1F0895FC016150704001900110D8F7E5
:1021D000809590958E0F9F1F08950F931F93CF9317
:1021E000DF938C01EB018B8181FF1BC082FF0DC04F
:1021F0002E813F818C819D812817390764F4E88105
:10220000F9810193F983E88306C0E885F985802F79
:102210001995892B31F48E819F8101969F838E833E
:1022200002C00FEF1FEFC801DF91CF911F910F91F7
:102230000895FA01AA27283051F1203181F1E8945C
:102240006F936E7F6E5F7F4F8F4F9F4FAF4FB1E0A9
:102250003ED0B4E03CD0670F781F891F9A1FA11DA4
:10226000680F791F8A1F911DA11D6A0F711D811DA5
:10227000911DA11D20D009F468943F912AE0269F6A
:1022800011243019305D3193DEF6CF010895462FC9
:102290004770405D4193B3E00FD0C9F7F6CF462FAA
:1022A0004F70405D4A3318F0495D31FD4052419313
:1022B00002D0A9F7EACFB4E0A695979587957795D0
:1022C0006795BA95C9F700976105710508959B0157
:1022D000AC010A2E06945795479537952795BA95E0
:1022E000C9F7620F731F841F951FA01D0895DF9308
:1022F000CF93CDB7DEB766970FB6F894DEBF0FBEAB
:10230000CDBF8091000290910102A0910202B09194
:1023100003028F87988BA98BBA8BFE013F9644E608
:1023200050E08081F999FECF1FBA52BD41BD80BDFA
:102330000FB6F894FA9AF99A0FBE4F5F5F4F48367E
:10234000510511F03196EDCFE5ECF7E08081F99978
:10235000FECF1FBA52BD41BD80BD0FB6F894FA9AA8
:10236000F99A0FBE4F5F5F4F4837510511F0319614
:10237000EDCFE5EBF7E08081F999FECF1FBA52BDB2
:1023800041BD80BD0FB6F894FA9AF99A0FBE4F5F1F
:102390005F4F4838510511F03196EDCFE5EDF7E08C
:1023A0008081F999FECF1FBA52BD41BD80BD0FB6E5
:1023B000F894FA9AF99A0FBE4F5F5F4F483951056A
:1023C00011F03196EDCFE9EEF7E08081F999FECF7B
:1023D0001FBA52BD41BD80BD0FB6F894FA9AF99A62
:1023E0000FBE4F5F5F4F4C39510511F03196EDCF65
:1023F000EDEEF7E08081F999FECF1FBA52BD41BDE5
:1024000080BD0FB6F894FA9AF99A0FBE4F5F5F4FEE
:10241000403A510511F03196EDCFE5EEF7E08081BD
:10242000F999FECF1FBA52BD41BD80BD0FB6F894D9
:10243000FA9AF99A0FBE4F5F5F4F443A510511F077
:102440003196EDCFEDEFF7E08081F999FECF1FBA1D
:1024500052BD41BD80BD0FB6F894FA9AF99A0FBEED
:102460004F5F5F4F483A510511F03196EDCFE1EBE8
:10247000F7E08081F999FECF1FBA52BD41BD80BD02
:102480000FB6F894FA9AF99A0FBE4F5F5F4F4C3A25
:10249000510511F03196EDCFE1EFF7E08081F99928
:1024A000FECF1FBA52BD41BD80BD0FB6F894FA9A57
:1024B000F99A0FBE4F5F5F4F403B510511F03196C7
:1024C000EDCFE5EFF7E08081F999FECF1FBA52BD5D
:1024D00041BD80BD0FB6F894FA9AF99A0FBE4F5FCE
:1024E0005F4F443B510511F03196EDCFE9EFF7E036
:1024F0008081F999FECF1FBA52BD41BD80BD0FB694
:10250000F894FA9AF99A0FBE4F5F5F4F483B510516
:1025100011F03196EDCFE5E4F5E08081F999FECF39
:102520001FBA52BD41BD80BD0FB6F894FA9AF99A10
:102530000FBE4F5F5F4F443C510511F03196EDCF18
:1025400084EB90E09A83898386E490E09C838B837C
:102550002FEF30E03E832D8380EF90E098878F83CC
:1025600084E690E09A8789873C872B87FE01319625
:102570008081F999FECF1FBA52BD41BD80BD0FB613
:10258000F894FA9AF99A0FBE4F5F5F4F463C510597
:1025900071F7FE0133968081F999FECF1FBA52BDC3
:1025A00041BD80BD0FB6F894FA9AF99A0FBE4F5FFD
:1025B0005F4F483C510511F03196EDCFFE01359645
:1025C0008081F999FECF1FBA52BD41BD80BD0FB6C3
:1025D000F894FA9AF99A0FBE4F5F5F4F4A3C510543
:1025E00011F03196EDCFFE0137968081F999FECF3B
:1025F0001FBA52BD41BD80BD0FB6F894FA9AF99A40
:102600000FBE4F5F5F4F4C3C510511F03196EDCF3F
:10261000FE0139968081F999FECF1FBA52BD41BDA6
:1026200080BD0FB6F894FA9AF99A0FBE4F5F5F4FCC
:102630004E3C510511F03196EDCFFE013B96808165
:10264000F999FECF1FBA52BD41BD80BD0FB6F894B7
:10265000FA9AF99A0FBE4F5F5F4F403D510511F056
:102660003196EDCFE0E6F5E08081F999FECF1FBA13
:1026700052BD41BD80BD0FB6F894FA9AF99A0FBECB
:102680004F5F5F4F443D510511F03196EDCFE4E0CF
:10269000F4E08081F999FECF1FBA52BD41BD80BDE3
:1026A0000FB6F894FA9AF99A0FBE4F5F5F4F483D04
:1026B000510511F03196EDCFE8E0F4E08081F99911
:1026C000FECF1FBA52BD41BD80BD0FB6F894FA9A35
:1026D000F99A0FBE4F5F5F4F4C3D510511F0319697
:1026E000EDCFECE0F4E08081F999FECF1FBA52BD46
:1026F00041BD80BD0FB6F894FA9AF99A0FBE4F5FAC
:102700005F4F403E510511F03196EDCF80E290E0F1
:102710009E878D87FE013D968081F999FECF1FBA75
:1027200052BD41BD80BD0FB6F894FA9AF99A0FBE1A
:10273000413E510521F0319641EE50E0EDCF8091C0
:10274000040290910502A0910602B09107028B8BC2
:102750009C8BAD8BBE8BFE01739684E690E020814E
:10276000F999FECF1FBA92BD81BD20BD0FB6F89476
:10277000FA9AF99A0FBE8736910519F001963196AB
:10278000EECFEFE2F1E0949108C08091C00085FFA8
:10279000FCCF9093C600319694919923B1F7E9E369
:1027A000F3E0949108C08091C00085FFFCCF909326
:1027B000C600319694919923B1F78091C00085FFAE
:1027C000FCCF8AE08093C60066960FB6F894DEBF11
:1027D0000FBECDBFCF91DF910895DF93CF93CDB7DB
:1027E000DEB7E0970FB6F894DEBF0FBECDBFDE01B7
:1027F0001196E6E4F4E080E101900D928150E1F75A
:10280000DE015196E6E3F4E080E101900D92815003
:10281000E1F7DE019196E6E2F4E080E101900D92AD
:102820008150E1F789819A81AB81BC818093C50792
:102830009093C607A093C707B093C80789899A8960
:10284000AB89BC898093B5079093B607A093B7076F
:10285000B093B80789A19AA1ABA1BCA18093D50779
:102860009093D607A093D707B093D8078D819E8108
:10287000AF81B8858093C9079093CA07A093CB070F
:10288000B093CC078D899E89AF89B88D8093B907A5
:102890009093BA07A093BB07B093BC078DA19EA1EC
:1028A000AFA1B8A58093D9079093DA07A093DB076F
:1028B000B093DC0789859A85AB85BC858093CD076D
:1028C0009093CE07A093CF07B093D007898D9A8DB0
:1028D000AB8DBC8D8093BD079093BE07A093BF07BF
:1028E000B093C00789A59AA5ABA5BCA58093DD07C9
:1028F0009093DE07A093DF07B093E0078D859E8558
:10290000AF85B8898093D1079093D207A093D3075E
:10291000B093D4078D8D9E8DAF8DB8A18093C107E4
:102920009093C207A093C307B093C4078DA59EA53B
:10293000AFA5B8A98093E1079093E207A093E307BE
:10294000B093E4070E94C94E80E090E0AAEFB4E49F
:102950008093E9079093EA07A093EB07B093EC0705
:1029600080E090E8ABE3B5E48093ED079093EE0749
:10297000A093EF07B093F00720E030E040E050E094
:102980002093E5073093E6074093E7075093E80765
:1029900080E29EE4A0E0B0E08093B1079093B2079C
:1029A000A093B307B093B4072093FD073093FE07BD
:1029B0004093FF075093000880E090E0A0E4B1E46A
:1029C0008093F1079093F207A093F307B093F40775
:1029D0008DEC9CECACECBEE38093F5079093F6078E
:1029E000A093F707B093F80780E090E0A0E2B1E48D
:1029F0008093F9079093FA07A093FB07B093FC0725
:102A000020934D0530934E0540934F05509350054C
:102A10002093490530934A0540934B0550934C054C
:102A2000209345053093460540934705509348054C
:102A30008AE999E9A9EBBFE380936005909361056A
:102A4000A0936205B09363058CEE91E5A6EEB1E428
:102A50008093040490930504A0930604B0930704A4
:102A600061EE7AE784EF9FE30E94AB8260930804F3
:102A70007093090480930A0490930B046FE175E04E
:102A800089ED92E40E94B78260930C0470930D0468
:102A900080930E0490930F040E94A58180E090E043
:102AA000A0E8BFE38093100490931104A093120454
:102AB000B0931304EFE2F1E0949108C08091C0005C
:102AC00085FFFCCF9093C600319694919923B1F77E
:102AD000E5E3F1E0949108C08091C00085FFFCCF50
:102AE0009093C600319694919923B1F78091C000DC
:102AF00085FFFCCF8AE08093C600E0960FB6F8947D
:102B0000DEBF0FBECDBFCF91DF910895CF93DF938E
:102B1000CFE2D1E0FE01949108C08091C00085FF12
:102B2000FCCF9093C600319694919923B1F7E9E2D6
:102B3000F3E0949108C08091C00085FFFCCF909392
:102B4000C600319694919923B1F78091C00085FF1A
:102B5000FCCF8AE08093C600FE019491EFE2F1E0A1
:102B600008C08091C00085FFFCCF9093C6003196CD
:102B700094919923B1F74091C5075091C607609190
:102B8000C7077091C80781E293E00E940921409134
:102B9000C9075091CA076091CB077091CC078EE1AD
:102BA00093E00E9409214091CD075091CE0760919A
:102BB000CF077091D0078BE193E00E9409214091EB
:102BC000D1075091D2076091D3077091D40788E163
:102BD00093E00E940921E8E0F2E007C08091C00084
:102BE00085FFFCCF31969093C60090819923B1F771
:102BF0008091C00085FFFCCF8AE08093C600FE0173
:102C00009491EFE2F1E008C08091C00085FFFCCF15
:102C10009093C600319694919923B1F7EEEFF2E0CC
:102C2000949108C08091C00085FFFCCF9093C600AE
:102C3000319694919923B1F78091C00085FFFCCF24
:102C40008AE08093C600FE019491EFE2F1E008C0B3
:102C50008091C00085FFFCCF9093C600319694917F
:102C60009923B1F74091B5075091B6076091B70726
:102C70007091B80785EF92E00E9409214091B90751
:102C80005091BA076091BB077091BC0782EF92E048
:102C90000E9409214091BD075091BE076091BF0776
:102CA0007091C0078FEE92E00E9409214091C10708
:102CB0005091C2076091C3077091C4078CEE92E0F7
:102CC0000E940921E8E0F2E007C08091C00085FF82
:102CD000FCCF31969093C60090819923B1F78091F3
:102CE000C00085FFFCCF8AE08093C600FE0194916E
:102CF000EFE2F1E008C08091C00085FFFCCF909327
:102D0000C600319694919923B1F7EEECF2E09491DC
:102D100008C08091C00085FFFCCF9093C60031961B
:102D200094919923B1F78091C00085FFFCCF8AE090
:102D30008093C600FE019491EFE2F1E008C080911B
:102D4000C00085FFFCCF9093C600319694919923E3
:102D5000B1F74091D5075091D6076091D707709190
:102D6000D80785EC92E00E941B214091D907509131
:102D7000DA076091DB077091DC0782EC92E00E9439
:102D80001B214091DD075091DE076091DF077091B4
:102D9000E0078FEB92E00E941B214091E1075091E8
:102DA000E2076091E3077091E4078CEB92E00E94E8
:102DB0001B21E8E0F2E007C08091C00085FFFCCF56
:102DC00031969093C60090819923B1F78091C0000D
:102DD00085FFFCCF8AE08093C600FE019491EFE26C
:102DE000F1E008C08091C00085FFFCCF9093C60041
:102DF000319694919923B1F7E7E8F2E0949108C0F5
:102E00008091C00085FFFCCF9093C60031969491CD
:102E10009923B1F78091C00085FFFCCF8AE08093B1
:102E2000C600FE019491EFE2F1E008C08091C0007D
:102E300085FFFCCF9093C600319694919923B1F70A
:102E40004091E9075091EA076091EB077091EC0718
:102E50008EE792E00E9409214091ED075091EE0724
:102E60006091EF077091F0078BE792E00E940921D3
:102E7000E8E0F2E007C08091C00085FFFCCF31960A
:102E80009093C60090819923B1F78091C00085FF8F
:102E9000FCCF8AE08093C600FE019491EFE2F1E05E
:102EA00008C08091C00085FFFCCF9093C60031968A
:102EB00094919923B1F7E8ECF1E0949108C08091E6
:102EC000C00085FFFCCF9093C60031969491992362
:102ED000B1F78091C00085FFFCCF8AE08093C600E7
:102EE000FE019491EFE2F1E008C08091C00085FFFF
:102EF000FCCF9093C600319694919923B1F74091FD
:102F0000E5075091E6076091E7077091E8078FEBBE
:102F100091E00E9409214091FD075091FE076091C8
:102F2000FF07709100088CEB91E00E94092140910D
:102F3000B1075091B2076091B3077091B40789EB64
:102F400091E00E941B214091F1075091F20760919E
:102F5000F3077091F40786EB91E00E9409214091FC
:102F6000F5075091F6076091F7077091F80783EB2A
:102F700091E00E9409214091F9075091FA07609170
:102F8000FB077091FC0780EB91E00E940921E8E0CB
:102F9000F2E007C08091C00085FFFCCF319690938E
:102FA000C60090819923B1F78091C00085FFFCCFC6
:102FB0008AE08093C600FE019491EFE2F1E008C040
:102FC0008091C00085FFFCCF9093C600319694910C
:102FD0009923B1F7EEE9F1E0949108C08091C00027
:102FE00085FFFCCF9093C600319694919923B1F759
:102FF0008091C00085FFFCCF8AE08093C600FE016F
:103000009491EFE2F1E008C08091C00085FFFCCF11
:103010009093C600319694919923B1F7409145055C
:1030200050914605609147057091480585E991E00A
:103030000E9409214091490550914A0560914B0534
:1030400070914C0582E991E00E94092140914D0563
:1030500050914E0560914F05709150058FE891E0B9
:103060000E940921E8E0F2E007C08091C00085FFDE
:10307000FCCF31969093C60090819923B1F780914F
:10308000C00085FFFCCF8AE08093C600FE019491CA
:10309000EFE2F1E008C08091C00085FFFCCF909383
:1030A000C600319694919923B1F7E1E8F1E094914B
:1030B00008C08091C00085FFFCCF9093C600319678
:1030C00094919923B1F78091C00085FFFCCF8AE0ED
:1030D0008093C600FE019491EFE2F1E008C0809178
:1030E000C00085FFFCCF9093C60031969491992340
:1030F000B1F7409104045091050460910604709169
:10310000070487E791E00E9409216091080470910B
:10311000090480910A0490910B040E94B182AB01D2
:10312000BC0184E791E00E94092160910C04709138
:103130000D0480910E0490910F040E94BD82AB019A
:10314000BC0181E791E00E940921E8E0F2E007C0BC
:103150008091C00085FFFCCF31969093C60090818E
:103160009923B1F78091C00085FFFCCF8AE080935E
:10317000C600DF91CF9108950F931F93DF93CF93F4
:10318000CDB7DEB766970FB6F894DEBF0FBECDBFE2
:103190008091040290910502A0910602B09107026D
:1031A0008B8B9C8BAD8BBE8BFE013F9604E610E0B3
:1031B000F999FECF12BD01BDF89A80B580830F5FEB
:1031C0001F4F0836110511F03196F2CFCE0143960C
:1031D000BE01615F7F4F43E050E00E94D60E009732
:1031E00009F096C1E5ECF7E0F999FECF12BD01BDFB
:1031F000F89A80B580830F5F1F4F0837110511F0D3
:103200003196F2CFE5EBF7E0F999FECF12BD01BDA3
:10321000F89A80B580830F5F1F4F0838110511F0B1
:103220003196F2CFE5EDF7E0F999FECF12BD01BD81
:10323000F89A80B580830F5F1F4F0839110511F090
:103240003196F2CF0E94C94EE9EEF7E0F999FECF30
:1032500012BD01BDF89A80B580830F5F1F4F0C39F6
:10326000110511F03196F2CFEDEEF7E0F999FECFAE
:1032700012BD01BDF89A80B580830F5F1F4F003AE1
:10328000110511F03196F2CFE5EEF7E0F999FECF96
:1032900012BD01BDF89A80B580830F5F1F4F043ABD
:1032A000110511F03196F2CFEDEFF7E0F999FECF6D
:1032B00012BD01BDF89A80B580830F5F1F4F083A99
:1032C000110511F03196F2CFE1EBF7E0F999FECF5D
:1032D00012BD01BDF89A80B580830F5F1F4F0C3A75
:1032E000110511F03196F2CFE1EFF7E0F999FECF39
:1032F00012BD01BDF89A80B580830F5F1F4F003B60
:10330000110511F03196F2CFE5EFF7E0F999FECF14
:1033100012BD01BDF89A80B580830F5F1F4F043B3B
:10332000110511F03196F2CFE9EFF7E0F999FECFF0
:1033300012BD01BDF89A80B580830F5F1F4F083B17
:10334000110511F03196F2CFE5E4F5E0F999FECFE1
:1033500012BD01BDF89A80B580830F5F1F4F043CFA
:10336000110511F03196F2CFFE013196F999FECF99
:1033700012BD01BDF89A80B580830F5F1F4F063CD8
:10338000110599F7FE013396F999FECF12BD01BDE3
:10339000F89A80B580830F5F1F4F083C110511F02C
:1033A0003196F2CFFE013596F999FECF12BD01BDDF
:1033B000F89A80B580830F5F1F4F0A3C110511F00A
:1033C0003196F2CFFE013796F999FECF12BD01BDBD
:1033D000F89A80B580830F5F1F4F0C3C110511F0E8
:1033E0003196F2CFFE013996F999FECF12BD01BD9B
:1033F000F89A80B580830F5F1F4F0E3C110511F0C6
:103400003196F2CFFE013B96F999FECF12BD01BD78
:10341000F89A80B580830F5F1F4F003D110511F0B2
:103420003196F2CFE0E6F5E0F999FECF12BD01BD8D
:10343000F89A80B580830F5F1F4F043D110511F08E
:103440003196F2CFE4E0F4E0F999FECF12BD01BD70
:10345000F89A80B580830F5F1F4F083D110511F06A
:103460003196F2CFE8E0F4E0F999FECF12BD01BD4C
:10347000F89A80B580830F5F1F4F0C3D110511F046
:103480003196F2CFECE0F4E0F999FECF12BD01BD28
:10349000F89A80B580830F5F1F4F003E110511F031
:1034A0003196F2CFFE013D96F999FECF12BD01BDD6
:1034B000F89A80B58083013E110521F0319601EE26
:1034C00010E0F2CF0E94A581EFE2F1E0949108C0F4
:1034D0008091C00085FFFCCF9093C60031969491F7
:1034E0009923B1F7E7E5F1E0949108C08091C0001D
:1034F00085FFFCCF9093C600319694919923B1F744
:103500008091C00085FFFCCF8AE08093C60001C097
:1035100064D9FCDA66960FB6F894DEBF0FBECDBF55
:10352000CF91DF911F910F9108951F920F920FB6C7
:103530000F920BB60F9211242F933F934F938F93BB
:103540009F93EF93FF934091C600E0912A05F0917D
:103550002B0531969F012F773070319780912C0584
:1035600090912D052817390739F0E655FB4F408318
:1035700030932B0520932A05FF91EF919F918F9116
:103580004F913F912F910F900BBE0F900FBE0F9058
:103590001F9018959A01AB01203081EE380780E02A
:1035A000480780E0580749F182E08093C00060E05E
:1035B00079E08DE390E00E944A9D215030404040E8
:1035C0005040CA01B90122E030E040E050E00E94E2
:1035D0004A9D3093C5002093C4008091C100806152
:1035E0008093C1008091C10088608093C100809168
:1035F000C10080688093C10008951092C00020E14E
:1036000030E0E7CF20912C0530912D0580912A05DF
:1036100090912B058217930719F42FEF3FEF0EC0FF
:10362000F901E655FB4F80812F5F3F4F2F773070B8
:1036300030932D0520932C05282F30E0C9010895E3
:1036400080912C0590912D0590932B0580932A0550
:10365000089508952F923F924F925F926F927F92BA
:103660008F929F92AF92BF92CF92DF92EF92FF9292
:103670000F931F93DF93CF93CDB7DEB7A0970FB60D
:10368000F894DEBF0FBECDBF1C016A017B0141155E
:1036900051056105710541F440E350E060E070E0E0
:1036A00020E030E08BD055C0882499245401422E6C
:1036B00055246624772401E010E00C0F1D1F080D2F
:1036C000191DC701B601A30192010E94289DF801AE
:1036D00060830894811C911CA11CB11CC701B60118
:1036E000A30192010E94289DC901DA016C017D01AC
:1036F000C114D104E104F104F1F681E0E82EF12CCB
:10370000EC0EFD1EE80CF91C3E010894611C711CB6
:10371000D501C4010197A109B1096C01C818D908E4
:1037200015C0F601EE0DFF1D40814A3010F4405DDA
:1037300001C0495C552747FD5095652F752FC10184
:1037400020E030E03BD00894E108F1086E147F04DB
:1037500041F7A0960FB6F894DEBF0FBECDBFCF9154
:10376000DF911F910F91FF90EF90DF90CF90BF906E
:10377000AF909F908F907F906F905F904F903F9011
:103780002F9008952115310539F48091C00085FFEF
:10379000FCCF4093C60008955DCFEF92FF920F9348
:1037A0001F939A01E62EFF2400E010E0B801A70164
:1037B000E9DF1F910F91FF90EF900895EF92FF9234
:1037C0000F931F93CF93DF93EC017A018B012115A7
:1037D000310539F48091C00085FFFCCFE092C6002E
:1037E00019C02A303105A9F477FF0FC04DE250E02F
:1037F00060E070E020E030E0E1DF10950095F094AB
:10380000E094E11CF11C011D111DCE01B801A701BE
:103810002AE020DFDF91CF911F910F91FF90EF9071
:103820000895EF92FF920F931F937B019A01002757
:10383000F7FC0095102FB801A701C0DF1F910F9171
:10384000FF90EF9008950F931F938C014DE050E08F
:1038500060E070E020E030E0B1DFC8014AE050E015
:1038600060E070E020E030E0A9DF1F910F91089543
:10387000CF92DF92EF92FF920F931F938C019A01E8
:103880006B01EE24FF24B701A6017CDFC801DBDF5A
:103890001F910F91FF90EF90DF90CF9008959F922E
:1038A000AF92BF92CF92DF92EF92FF920F931F934E
:1038B000CF93DF93EC017A018B01922ECB01BA01F9
:1038C00020E030E040E050E00E943099882364F42A
:1038D000CE014DE250E060E070E020E030E06EDFCD
:1038E00017FB109517F9109520E030E040E05FE3FA
:1038F000AA240BC0CA01B90120E030E040E251E443
:103900000E9437999B01AC01A394A91498F3C801B4
:10391000B7010E9457987B018C010E94A4995B011A
:103920006C010E94D0999B01AC01C801B7010E94B3
:1039300056987B018C01CE01B601A5012AE030E04A
:1039400021DF992099F1E9E0F2E007C08091C00001
:1039500085FFFCCF31969093C60090819923B1F7F3
:1039600025C0C801B70120E030E040E251E40E94E8
:10397000109C7B018C010E949F995B016C01CC24FF
:10398000B7FCC094DC2CCE01B601A5012AE030E0E2
:1039900015DFC601B5010E94D2999B01AC01C80197
:1039A000B7010E9456987B018C019A949920C9F620
:1039B000DF91CF911F910F91FF90EF90DF90CF900B
:1039C000BF90AF909F9008956ACF0895EF92FF92B5
:1039D0000F931F93CF93DF93EC01E0909B03F09044
:1039E0009C0300919D0310919E03688179818A81D7
:1039F0009B81A80197010E943E9B181624F4E8823F
:103A0000F9820A831B83E0909F03F090A00300914A
:103A1000A1031091A2036C817D818E819F81A801F9
:103A200097010E943E9B181624F4EC82FD820E83BF
:103A30001F83E090A303F090A4030091A5031091CD
:103A4000A603688579858A859B85A80197010E94D0
:103A50003E9B181624F4E886F9860A871B87DF91B7
:103A6000CF911F910F91FF90EF9008958091720573
:103A7000089567707070E82FF0E0E15FFA4E84916E
:103A80008B3028F48830A0F4863090F106C08E3058
:103A9000D0F08F50833060F521C08091B100887FD5
:103AA0008093B1008091B100862B8093B10008957E
:103AB00080919100887F8093910080919100862B66
:103AC0008093910008958091A100887F8093A10048
:103AD0008091A100862B8093A100089580912101FF
:103AE000887F8093210180912101862B8093210181
:103AF000089583E795E00C9492470E948E8280910E
:103B00007205882309F036C081E0809372058091A8
:103B1000780590917905A0917A05B0917B05809305
:103B20007C0590937D05A0937E05B0937F05EFE41F
:103B3000F3E0949108C08091C00085FFFCCF909382
:103B4000C600319694919923B1F7E6E5F3E094919C
:103B500008C08091C00085FFFCCF9093C6003196CD
:103B600094919923B1F78091C00085FFFCCF8AE042
:103B70008093C6000895F8940E948E82179A10923E
:103B80005D05169A10925E05159A10925F05149ABB
:103B900084E060E00E940F96EFE4F3E0949108C0A7
:103BA0008091C00085FFFCCF9093C6003196949120
:103BB0009923B1F7ECECF3E0949108C08091C00038
:103BC00085FFFCCF9093C600319694919923B1F76D
:103BD0008091C00085FFFCCF8AE08093C600FFCFB4
:103BE0000E944695609382057093830580938405B7
:103BF00090938505EBEEF3E0949108C08091C000AE
:103C000085FFFCCF9093C600319694919923B1F72C
:103C10008091C00085FFFCCF8AE08093C6000895A4
:103C20006F927F928F929F92AF92BF92CF92DF92CC
:103C3000EF92FF920F931F93F82E60918A05709177
:103C40008B0580918C0590918D0520918E0530918A
:103C50008F0540919005509191050E944B9B3B012F
:103C60004C0100D000D00DB71EB70F5F1F4F609101
:103C7000910370919203882777FD8095982F0E9479
:103C8000D2992091BE033091BF034091C00350915F
:103C9000C1030E94109C20E030E040E752E40E9403
:103CA000379920E030E048EC52E40E9437995B01FC
:103CB0006C01F8016082718282829382F482809129
:103CC0006405858385E395E066E975E04AE855E09B
:103CD00020E001E032E0E32E0E940B4A809196053D
:103CE00090919705A0919805B0919905809335051D
:103CF00090933605A0933705B093380580919A05C7
:103D000090919B05A0919C05B0919D0580933905EC
:103D100090933A05A0933B05B0933C0580919E0596
:103D200090919F05A091A005B091A10580933D05BC
:103D300090933E05A0933F05B09340058091A20566
:103D40009091A305A091A405B091A505809341058C
:103D500090934205A0934305B09344058DB79EB759
:103D600006960FB6F8949EBF0FBE8DBF0E94469573
:103D700060938205709383058093840590938505F5
:103D80001F910F91FF90EF90DF90CF90BF90AF9079
:103D90009F908F907F906F9008954F925F926F9257
:103DA0007F928F929F92AF92BF92CF92DF92EF92CB
:103DB000FF920F931F93DF93CF9300D00F92CDB755
:103DC000DEB7E0909B03F0909C0300919D0310915F
:103DD0009E0360919605709197058091980590914A
:103DE0009905A80197010E943E9B181644F4E092A1
:103DF0009605F09297050093980510939905E09029
:103E00009F03F090A0030091A1031091A203609181
:103E10009A0570919B0580919C0590919D05A80144
:103E200097010E943E9B181644F4E0929A05F09286
:103E30009B0500939C0510939D05E090A303F090D3
:103E4000A4030091A5031091A60360919E057091B3
:103E50009F058091A0059091A105A80197010E945E
:103E60003E9B181644F4E0929E05F0929F05009345
:103E7000A0051093A1050E9446956093820570935A
:103E80008305809384059093850580919605909194
:103E90009705A0919805B091990589839A83AB8382
:103EA000BC836091350570913605809137059091FE
:103EB000380529813A814B815C810E9430998823A1
:103EC00009F09EC040909A0550909B0560909C051B
:103ED00070909D056091390570913A0580913B0580
:103EE00090913C05A30192010E943099882309F02A
:103EF00087C00F920F92CDB6DEB60894C11CD11CBC
:103F0000E0909E05F0909F050091A0051091A105FD
:103F10006091BE037091BF038091C0039091C10373
:103F200020E030E040E752E40E9437994B015C0109
:103F300084E695E0D6018D939C9369817A818B818B
:103F40009C81A3019201E2EACE2EE5E0DE2E0E94E2
:103F500025550F900F908091960590919705A0910F
:103F60009805B09199058093350590933605A093F7
:103F70003705B093380580919A0590919B05A091E3
:103F80009C05B0919D058093390590933A05A093C7
:103F90003B05B0933C0580919E0590919F05A091B3
:103FA000A005B091A10580933D0590933E05A09397
:103FB0003F05B09340058091A2059091A305A09183
:103FC000A405B091A5058093410590934205A09367
:103FD0004305B09344050F900F900F900F90CF9131
:103FE000DF911F910F91FF90EF90DF90CF90BF90E6
:103FF000AF909F908F907F906F905F904F900895BB
:104000000F920F92CDB6DEB60894C11CD11C409021
:104010009A0550909B0560909C0570909D05E090DE
:104020009E05F0909F050091A0051091A10560915B
:10403000910370919203882777FD8095982F0E94B5
:10404000D2992091BE033091BF034091C00350919B
:10405000C1030E94109C20E030E040E752E40E943F
:10406000379920E030E048EC52E40E9437994B0148
:104070005C0184E695E0F601918380835ECF8EE259
:1040800095E0DEDAEEEEF3E0949108C08091C00096
:1040900085FFFCCF9093C600319694919923B1F798
:1040A000409178055091790560917A0570917B0572
:1040B0004F5F5F4F6F4F7F4F8EE295E02AE030E019
:1040C0007DDB8091C00085FFFCCF8AE08093C60035
:1040D00087CD4F925F926F927F928F929F92AF9215
:1040E000BF92CF92DF92EF92FF920F931F93409077
:1040F000BE035090BF036090C0037090C1030F2EA9
:10410000F0E0AF2EF0EABF2EFCE8CF2EF6E4DF2E73
:10411000F02DA092BE03B092BF03C092C003D09214
:10412000C1036093350570933605809337059093EE
:1041300038052093390530933A0540933B05509359
:104140003C05E0923D05F0923E0500933F0510933B
:1041500040050F920F92E4E6F5E0ADB7BEB71296B8
:10416000FC93EE931197F1E4CF2EF5E0DF2E0F2EA6
:10417000F0E08F2EF0E09F2EF6E9AF2EF3E4BF2E95
:10418000F02D0E9425550F900F900E94F6784092D6
:10419000BE035092BF036092C0037092C1031F918F
:1041A0000F91FF90EF90DF90CF90BF90AF909F90D6
:1041B0008F907F906F905F904F9008958091BE0395
:1041C0009091BF03A091C003B091C1038093AB0550
:1041D0009093AC05A093AD05B093AE05809191038B
:1041E00090919203909334058093330584E690E098
:1041F00090939203809391030E9446956093820569
:1042000070938305809384059093850581E00C94D9
:104210002D76FC01949108C08091C00085FFFCCFF1
:104220009093C600319694919923B1F78EE295E070
:1042300022E030E0C9CBFC01949108C08091C0001D
:1042400085FFFCCF9093C600319694919923B1F7E6
:104250008EE295E02AE030E095CA4091B105509198
:10426000B20520E630E0B901469F9001479F300D2E
:10427000569F300D1124682F772767FD7095C9016F
:104280008D549A4F0E94C20E9C019093B00580936A
:10429000AF0580E0232B09F081E008952F923F9233
:1042A0004F925F926F927F928F929F92AF92BF9246
:1042B000CF92DF92EF92FF920F931F93DF93CF93F2
:1042C000CDB7DEB76C970FB6F894DEBF0FBECDBF8B
:1042D0009E838D838330910508F04AC2FC01E9502A
:1042E000FA4FB4904C01880C991C880C991CF4016D
:1042F000EB5CFA4F80E090E0A0E0B0E08083918337
:10430000A283B3836091350570913605809137059E
:10431000909138052091390530913A0540913B053F
:1043200050913C05E0903D05F0903E0500913F0521
:1043300010914005E1E4CE2EE5E0DE2E0E94114F03
:10434000ED81FE81EE0FFF1FE955FC4F0190F081DA
:10435000E02DF7FD10C0CF01880F991F8E0F9F1F12
:104360002DEA33E0820E931ED4016D917C918D581D
:104370009A4F0E945B482D803E80220C331C220CF9
:10438000331CF101E650FA4FE590F5900591149138
:104390006B2D772767FD7095882777FD8095982F7F
:1043A0000E94D29969837A838B839C83F101EA56B8
:1043B000FA4FFC8FEB8FC801B70120E030E040ECF2
:1043C0005FE30E94109C29813A814B815C810E94AD
:1043D000109CAB8DBC8D6D937D938D939C931397A7
:1043E000F101EF57FC4FF887EF8360817181828183
:1043F00093816093BE037093BF038093C003909337
:10440000C1030F920F92CDB6DEB60894C11CD11C29
:10441000409096055090970560909805709099058A
:1044200020919A0530919B0540919C0550919D05E6
:1044300029873A874B875C87E0909E05F0909F051F
:104440000091A0051091A10520E030E040E752E482
:104450000E9437994B015C01E4E6F5E0D601ED934B
:10446000FC93C301B20129853A854B855C85B2EA8C
:10447000CB2EB5E0DB2E0E9425550F900F900E94A9
:10448000F67891012B5C3A4F3E872D8780E090E0D3
:10449000A0E0B0E0F90180839183A283B3836091AF
:1044A000350570913605809137059091380520913A
:1044B000390530913A0540913B0550913C05E0901B
:1044C0003D05F0903E0500913F0510914005A1E4A7
:1044D000CA2EA5E0DA2E0E94114FF101E65DF94FD8
:1044E0004590559065907490C301B2019058298110
:1044F0003A814B815C810E94109CAB8DBC8D6D9389
:104500007D938D939C9313970F920F92CDB6DEB649
:104510000894C11CD11C20919605309197054091BB
:104520009805509199052F87388B498B5A8B80912C
:104530009A0590919B05A0919C05B0919D058B8B50
:104540009C8BAD8BBE8BE0909E05F0909F050091FB
:10455000A0051091A1056091BE037091BF038091E9
:10456000C0039091C10320E030E040E752E40E9494
:1045700037994B015C01E4E6F5E0D601ED93FC933D
:104580006F85788989899A892B893C894D895E89CB
:10459000F2EACF2EF5E0DF2E0E9425550F900F9006
:1045A0000E94F678C301B201A30192010E945798BC
:1045B00029813A814B815C810E94109CAB8DBC8D1E
:1045C0006D937D938D939C931397EF81F885608114
:1045D00071818281938120E030E040E05FE30E94BE
:1045E000109C6093BE037093BF038093C0039093AD
:1045F000C1030F920F92CDB6DEB60894C11CD11C38
:104600004090960550909705609098057090990598
:1046100020919A0530919B0540919C0550919D05F4
:104620002F8B388F498F5A8FE0909E05F0909F0511
:104630000091A0051091A10520E030E040E752E490
:104640000E9437994B015C01E4E6F5E0D601ED9359
:10465000FC93C301B2012F89388D498D5A8DE2EA4E
:10466000CE2EE5E0DE2E0E9425550F900F900E9481
:10467000F678F101EA5FF94F659175918591949112
:10468000F101EB5BFA4FA080B180C280D380A6011C
:1046900095010E9457987B018C01CB01D801ED85D3
:1046A000FE8580839183A283B383F101EE5EF94F8F
:1046B000659175918591949121E5822E25E0922E48
:1046C000820C931CA60195010E945798D4016D930A
:1046D0007D938D939C931397F101E25EF94F659161
:1046E000759185919491EBE9F3E02E0E3F1EA601A2
:1046F00095010E945798D1016D937D938D939C9362
:104700001397C701D801EB8DFC8D80839183A28321
:10471000B38320E030E040E050E02093BE033093CC
:10472000BF034093C0035093C1030E942676ED81DE
:10473000FE81E35AFA4F81E08083AD81BE81AA0FEA
:10474000BB1FFD01E955FC4F0190F081E02DF7FD05
:104750000FC0CF01880F991F8E0F9F1FAA0FBB1F7D
:10476000A155BC4F6D917C918D589A4F0E945B482A
:104770006C960FB6F894DEBF0FBECDBFCF91DF9120
:104780001F910F91FF90EF90DF90CF90BF90AF906F
:104790009F908F907F906F905F904F903F902F9061
:1047A00008950F931F93CF93DF93C7EAD3E00FEAE7
:1047B00013E02881398137FD0CC0C901880F991F8A
:1047C000820F931FF801608171818D589A4F0E946A
:1047D0005B4822960C5F1F4FF3E0CD3ADF0749F7A5
:1047E000DF91CF911F910F9108952F923F924F9299
:1047F0005F926F927F928F929F92AF92BF92CF9271
:10480000DF92EF92FF920F931F93DF93CF93CDB779
:10481000DEB72E970FB6F894DEBF0FBECDBF83EC88
:1048200093E00E949C8F6091890370918A0380912C
:104830008B0390918C036093BE037093BF038093AE
:10484000C0039093C1030F920F92CDB6DEB60894C9
:10485000C11CD11CE0903505F0903605009137055C
:10486000109138054090390550903A0560903B050D
:1048700070903C05B1E42B2EB5E03B2E20E030E0FB
:1048800040E752E40E9437994B015C01E4E6F5E011
:10489000D601ED93FC93C801B701A30192010F2E3D
:1048A000F0E0EF2EF0E0FF2EF0E20F2FF1EC1F2FE3
:1048B000F02D61010E9425550F900F900E94F6780F
:1048C00082E00E9493764B015C0160913505709106
:1048D0003605809137059091380520913905309142
:1048E0003A0540913B0550913C05850174010E94B9
:1048F000114F22E336E0F90185919591A591B4918C
:1049000089839A83AB83BC83C501B40129813A8131
:104910004B815C810E9457986D837E838F8398873B
:104920000F920F92CDB6DEB60894C11CD11CE09058
:104930003505F09036050091370510913805409007
:10494000390550903A0560903B0570903C056091A8
:10495000BE037091BF038091C0039091C10320E01A
:1049600030E040E752E40E9437994B015C01E4E6F5
:10497000F5E0D601ED93FC93C801B701A3019201C4
:10498000ED80FE800F81188561010E9425550F90F2
:104990000F900E94F6786091890370918A0380914C
:1049A0008B0390918C0320E030E040E252E40E94BF
:1049B00037995B016C016093BE037093BF038093D2
:1049C000C0039093C1030F920F928DB79EB70196CB
:1049D0009E878D874090350550903605609037054D
:1049E000709038058091390590913A05A0913B056A
:1049F000B0913C0589879A87AB87BC8769817A81AA
:104A00008B819C8120E030E040E050EC0E94109CC3
:104A10009B01AC016D817E818F8198850E945798A2
:104A20007B018C01C601B50120E030E040E752E493
:104A30000E9437994B015C01E4E6F5E0AD85BE8547
:104A4000ED93FC93C301B20129853A854B855C85C2
:104A500061010E9425550F900F900E94F67882E028
:104A60000E9493767B018C0160933D0570933E0517
:104A700080933F0590934005609135057091360510
:104A800080913705909138052091390530913A058C
:104A900040913B0550913C050E94114F2E960FB658
:104AA000F894DEBF0FBECDBFCF91DF911F910F9164
:104AB000FF90EF90DF90CF90BF90AF909F908F903E
:104AC0007F906F905F904F903F902F9008956F92DE
:104AD0007F928F929F92AF92BF92CF92DF92EF928E
:104AE000FF920F931F935B016C0139014A016091A2
:104AF00035057091360580913705909138052091E4
:104B0000390530913A0540913B0550913C05E1DA79
:104B1000E0903D05F0903E0500913F051091400565
:104B2000C601B501A4019301D4DA2091AB03309101
:104B3000AC0337FD0DC0C901880F991F820F931F69
:104B40006091B5037091B6038D589A4F0E945B48EF
:104B50004CDE10913D0500913E05F0903F05E09040
:104B600040052091AB033091AC0337FD0DC0C90166
:104B7000880F991F820F931F6091B7037091B8033C
:104B80008D589A4F0E945B48E7E4F6E0949108C084
:104B90008091C00085FFFCCF9093C6003196949120
:104BA0009923B1F7E2E4F6E0949108C08091C00047
:104BB00085FFFCCF9093C600319694919923B1F76D
:104BC0008EE295E0B601A50122E030E00E94E41CEF
:104BD000EDE3F6E0949108C08091C00085FFFCCF22
:104BE0009093C600319694919923B1F78EE295E0A7
:104BF000B401A30122E030E00E94E41CE8E3F6E007
:104C0000949108C08091C00085FFFCCF9093C600AE
:104C1000319694919923B1F78EE295E0212F302FB0
:104C2000EF2DFE2DA901BF0122E030E00E94E41C1F
:104C3000E6E3F6E0949108C08091C00085FFFCCFC8
:104C40009093C600319694919923B1F7212F302F7C
:104C50004F2D5E2DB901CA011F910F91FF90EF906A
:104C6000DF90CF90BF90AF909F908F907F906F908C
:104C700008958091AF059091B005019660E070E0D5
:104C80004AE050E00C94610D8091AF059091B00521
:104C9000019660E070E00C94040CCF93DF93EC017C
:104CA000809164058093770584E5D7DA882309F439
:104CB00081C0EADF0E94A499262F609377056623BE
:104CC00009F478C0E9E4F3E0949108C08091C00051
:104CD00085FFFCCF9093C600319694919923B1F74C
:104CE000CD36D105C1F0CE36D10544F4C836D10554
:104CF000C1F0C936D10509F04DC010C0CA3DD1057B
:104D000039F0CD3DD10509F045C0EBE0F2E03FC000
:104D1000E2E2F2E031C0E9E3F2E023C0E0E5F2E0F4
:104D200015C0E7E6F2E007C08091C00085FFFCCF28
:104D300031969093C60090819923B1F72BC0809152
:104D4000C00085FFFCCF31969093C60090819923D7
:104D5000B1F720C08091C00085FFFCCF31969093C1
:104D6000C60090819923B1F715C08091C00085FFDE
:104D7000FCCF31969093C60090819923B1F70AC079
:104D80008091C00085FFFCCF31969093C600908142
:104D90009923B1F78EE295E0622F40E050E00E9447
:104DA000CD1B8091C00085FFFCCF8AE08093C600B8
:104DB00081E001C080E0DF91CF910895AF92BF9272
:104DC000CF92DF92EF92FF920F931F93CF93DF93D7
:104DD00065E3E62E65E0F62EC6E9D5E000E010E0DA
:104DE000F801EA5AFB4F808138DA882331F14CDF31
:104DF0005B016C01F801E15DFA4F8081882311F0BD
:104E000061E002C06091A60570E0882777FD80957B
:104E1000982F0E94D299F7012081318142815381DC
:104E20000E94109C9B01AC01C601B5010E945798DD
:104E3000688379838A839B8309C0F701808191818C
:104E4000A281B38188839983AA83BB830F5F1F4F9D
:104E500084E090E0E80EF91E24960430110509F074
:104E6000BFCF86E4FAD98823D9F00EDF7B018C010D
:104E70006093A7057093A8058093A9059093AA0550
:104E800020E030E040E050E00E943E9B181644F4E1
:104E9000E092BE03F092BF030093C0031093C103DE
:104EA000DF91CF911F910F91FF90EF90DF90CF9006
:104EB000BF90AF90089582DF89E4CFD9882351F065
:104EC000E3DE60938A0570938B0580938C05909345
:104ED0008D050CC080E090E0A0E0B0E080938A05F2
:104EE00090938B05A0938C05B0938D058AE4B5D97A
:104EF000882351F0C9DE60938E0570938F058093EF
:104F0000900590939105089580E090E0A0E0B0E0D6
:104F100080938E0590938F05A0939005B093910593
:104F200008958F929F92AF92BF92CF92DF92EF92AD
:104F3000FF920F931F93CF93DF93E0E6CE2ED12CF9
:104F4000EBE4F6E0A4907AE0972EE1ECF6E0B49082
:104F50008824839421C22D3071F02A3321F480916A
:104F60003407882341F080913507909136078F35BB
:104F700091050CF4EDC1E0913507F09136073097BB
:104F800019F41092340741C2A0913707B091380745
:104F9000AC9D8001AD9D100DBC9D100D1124E00F46
:104FA000F11FED54FA4F108280913407882309F0E5
:104FB000CAC110923407A75CB84F1C92E801CD54C7
:104FC000DA4FCE016EE470E00E94C20E9C010097A1
:104FD00009F4F7C09093B0058093AF052F5F3F4F62
:104FE0002C1B3D0B200F311FC9018D549A4F60E0DF
:104FF00070E04AE050E00E94610D60933D077093BD
:105000003E0780933F0790934007E0907805F0902B
:10501000790500917A0510917B05A80197012F5F12
:105020003F4F4F4F5F4F621773078407950709F48F
:10503000D2C180913707909138079C012C9DC00107
:105040002D9D900D3C9D900D11248D549A4F6AE634
:1050500077E00E94A80E892B09F0BDC1EFE4F3E0D0
:10506000949108C08091C00085FFFCCF9093C6004A
:10507000319694919923B1F7E7E3F7E0949108C052
:105080008091C00085FFFCCF9093C600319694912B
:105090009923B1F78EE295E0B801A7012AE030E04C
:1050A0000E94DE1B8091C00085FFFCCF73C01E27CD
:1050B0004F5FFC01E40FF11DED54FA4FE081EA323D
:1050C000B1F73093B0052093AF05C901019660E0B8
:1050D00070E00E94040C0E949F99212F30E0261757
:1050E000370709F45DC0EFE4F3E0949108C08091C4
:1050F000C00085FFFCCF9093C60031969491992310
:10510000B1F7E8E1F7E0949108C08091C00085FF15
:10511000FCCF9093C600319694919923B1F74091BA
:1051200078055091790560917A0570917B058EE242
:1051300095E02AE030E00E94DE1B8091C00085FFF0
:10514000FCCF28C0EFE4F3E0949108C08091C00048
:1051500085FFFCCF9093C600319694919923B1F7C7
:10516000EEEEF6E0949108C08091C00085FFFCCF80
:105170009093C600319694919923B1F78EE295E011
:10518000B801A7012AE030E00E94DE1B8091C00038
:1051900085FFFCCF8AE08093C6000E943F204AC072
:1051A00080913D0790913E07A0913F07B091400745
:1051B0008093780590937905A0937A05B0937B0549
:1051C0003EC0CE016AE270E00E94C20E009709F470
:1051D00036C0EFE4F3E0949108C08091C00085FFF1
:1051E000FCCF9093C600319694919923B1F7E4ECEB
:1051F000F6E0949108C08091C00085FFFCCF9093A9
:10520000C600319694919923B1F740917805509159
:10521000790560917A0570917B058EE295E02AE030
:1052200030E00E94DE1B8091C00085FFFCCF8AE049
:105230008093C6001092360710923507E6C0809121
:105240003707909138078C9D80018D9D100D9C9D96
:10525000100D1124E801CD54DA4FCE0167E470E05F
:105260000E94C20E9C01009709F441C09093B005C2
:105270008093AF052F5F3F4F2C1B3D0B200F311F3D
:10528000C9018D549A4F60E070E00E94040C0E94A6
:105290009F996430710558F580917205882399F4BF
:1052A0009B2DE1ECF6E008C08091C00085FFFCCFAB
:1052B0009093C600319694919923B1F78091C000E4
:1052C00085FFFCCF12C09A2DEBE4F6E008C0809178
:1052D000C00085FFFCCF9093C6003196949199232E
:1052E000B1F78091C00085FFFCCF9092C6008091FD
:1052F0003707909138079C012C9DC0012D9D900D82
:105300003C9D900D11248D549A4F6EE772E00E94DF
:10531000CD0E009711F40E94BB1D8091370790912C
:105320003807019664E070E00E94159D909338075D
:105330008093370780918005909181050196909325
:10534000810580938005109236071092350724C09E
:105350002B3311F480923407809134078823E1F4D1
:1053600020913507309136078091370790913807A3
:105370008C9DF0018D9DF00D9C9DF00D1124E20F90
:10538000F31FED54FA4F8091330780832F5F3F4F17
:10539000309336072093350780912A0590912B058D
:1053A00020912C0530912D05821B930B8F779070E7
:1053B000892B59F1809180059091810504972CF5F6
:1053C0008EE295E00E94021B282F809333078A30DB
:1053D00009F0C1CDD0CD80913707909138078C9DD1
:1053E000E0018D9DD00D9C9DD00D1124CE018D54DA
:1053F0009A4F6AE270E00E94C20E9C01009709F485
:10540000A1CE40E010E0CE0154CEDF91CF911F91AC
:105410000F91FF90EF90DF90CF90BF90AF909F9053
:105420008F900895EF92FF920F931F9380918005C4
:105430009091810503970CF474DD0E944695E090ED
:105440008605F090870500918805109189052091C7
:105450008205309183054091840550918505621B3A
:10546000730B840B950BE616F7060807190738F43B
:10547000E114F1040105110511F00E94BB1D80919A
:10548000BA039091BB03A091BC03B091BD030097F8
:10549000A105B10559F10E944695209182053091F0
:1054A00083054091840550918505621B730B840B25
:1054B000950B2091BA033091BB034091BC035091EE
:1054C000BD03261737074807590780F49091320D1E
:1054D0008091330D981751F4179A10925D05169A22
:1054E00010925E05159A10925F05149A0E9402525E
:1054F0001F910F91FF90EF9008952F923F924F923E
:105500005F926F927F928F929F92AF92BF92CF9253
:10551000DF92EF92FF920F931F93DF93CF93CDB75C
:10552000DEB7CB5CD0400FB6F894DEBF0FBECDBF68
:1055300087E40E942D21882311F40C94E933A4DB25
:105540000E949F996C31710509F493C06D3171050A
:105550009CF462307105C9F16330710524F477233E
:105560004CF50C946B4563307105C1F164307105E5
:1055700011F00C946B453EC06A35710511F40C9422
:105580007A336B35710554F46D31710509F485C4B6
:105590006E31710511F00C946B45DAC76B357105EE
:1055A00011F40C947E336C35710511F00C946B453D
:1055B0000C94833380917205882311F00C946B4511
:1055C000FDDB0E94CD1E0C948E45809172058823D0
:1055D00011F00C946B456FDC81E008C0809172057E
:1055E000882311F00C946B4566DC80E00E94101E4D
:1055F0000C948E4580E50E942D21882321F4EE2411
:10560000FF24870105C040DB0E94A4997B018C0127
:1056100083E50E942D21882359F036DB20E030E01D
:105620004AE754E40E94109C0E94A4997B018C01DB
:105630000E94F6780E9446955B016C01AE0CBF1C7F
:10564000C01ED11E0E94469560938205709383050B
:10565000809384059093850503C00E94E286E2DE74
:105660000E9446956A157B058C059D05B0F30C9448
:105670006B4583EC93E00E949C8F84E190E09093D3
:10568000FE038093FD038091BE039091BF03A09120
:10569000C003B091C1038093AB059093AC05A09378
:1056A000AD05B093AE0580919103909192039093D4
:1056B00034058093330584E690E0909392038093C1
:1056C00091030E94469560938205709383058093B1
:1056D00084059093850581E00E942D7680913505A3
:1056E00090913605A0913705B091380580939605C5
:1056F00090939705A0939805B093990580913905EB
:1057000090913A05A0913B05B0913C0580939A0594
:1057100090939B05A0939C05B0939D0580913D05BA
:1057200090913E05A0913F05B091400580939E0564
:1057300090939F05A093A005B093A105809141058A
:1057400090914205A0914305B09144058093A20534
:105750009093A305A093A405B093A50580E090E0E5
:10576000A0E0B0E08093BE039093BF03A093C0037A
:10577000B093C10388E50E942D21882361F489E557
:105780000E942D21882339F48AE50E942D21882347
:1057900011F481E001C080E08093C203882329F4E2
:1057A0008AE50E942D21882321F082E090E00E946A
:1057B0004E218091C203882361F488E50E942D2147
:1057C000882309F483C289E50E942D21882309F4E6
:1057D0007DC280E090E0A0E0B0E08093350590933A
:1057E0003605A0933705B09338058093390590931B
:1057F0003A05A0933B05B0933C05F7EF6F2EF5E01B
:105800007F2EF3018490E0903D05F0903E050091DD
:105810003F0510914005BC01CD019B01AC01E1E4C5
:10582000CE2EE5E0DE2E0E94114FBAEF4B2EB5E0F2
:105830005B2EF201659175918591949120E030E0A5
:1058400040EC5FE30E94109C7B018C01992487FC53
:105850009094AA2497FCA094BA2CC501B4010E948C
:10586000D2999B01AC01C801B7010E94109C6093C2
:105870009605709397058093980590939905A4E0F9
:105880008A2E912C840C951CF4016591759185915B
:1058900094910894611C711CF301D49020E030E0D5
:1058A00040EC5FE30E94109C7B018C016D2D7727FB
:1058B00067FD7095872F972F0E94D2999B01AC01AD
:1058C000C801B7010E94109C60939A0570939B05D4
:1058D00080939C0590939D052091810330918203D4
:1058E00040918303509184032093BE033093BF0300
:1058F0004093C0035093C103E0908503F09086036A
:105900000091870310918803C801B7010E94309964
:10591000882344F4E092BE03F092BF030093C003D7
:105920001093C103F201A590B590C590D490F401F5
:10593000E590F59005911491C601B501A801970174
:105940000E943E9B18162CF4C801B701A6019501D0
:1059500004C0C601B501A80197010E9437999B01B7
:10596000AC010E94109C9B01AC01CA0120E030E018
:1059700040E85FE30E9457980E947D9C9B01AC0128
:105980006091BE037091BF038091C0039091C103E9
:105990000E94109C6093BE037093BF038093C0036A
:1059A0009093C1030F920F92CDB6DEB60894C11C3E
:1059B000D11C409096055090970560909805709086
:1059C000990580919A0590919B05A0919C05B091B5
:1059D0009D05C054DF4F88839983AA83BB83C05C35
:1059E000D040E0909E05F0909F050091A005109199
:1059F000A1056091BE037091BF038091C003909197
:105A0000C10320E030E040E752E40E9437994B01A7
:105A10005C01F4E62F2EF5E03F2ED6012D923C924C
:105A2000C301B201C054DF4F288139814A815B81B3
:105A3000C05CD040E2EACE2EE5E0DE2E0E94255585
:105A40000F900F900E94F678E6E0F6E06591759170
:105A500085919491209145053091460540914705E7
:105A6000509148050E9457983B014C0160933505C1
:105A7000709336058093370590933805E2E1F6E0A0
:105A800065917591859194912091450530914605D8
:105A900040914705509148050E94579860935105E1
:105AA000709352058093530590935405EEE1F6E010
:105AB00065917591859194912091450530914605A8
:105AC00040914705509148050E94579860939B0369
:105AD00070939C0380939D0390939E03EAE0F6E00D
:105AE00065917591859194912091490530914A0570
:105AF00040914B0550914C050E9457985B016C01F9
:105B00006093390570933A0580933B0590933C056B
:105B1000E6E1F6E0659175918591949120914905B2
:105B200030914A0540914B0550914C050E94579881
:105B300060935505709356058093570590935805CB
:105B4000E2E2F6E065917591859194912091490585
:105B500030914A0540914B0550914C050E94579851
:105B600060939F037093A0038093A1039093A2037B
:105B7000E0903D05F0903E0500913F0510914005F5
:105B8000C401B301A6019501B1E4CB2EB5E0DB2E33
:105B90000E94114F8091350590913605A0913705EF
:105BA000B0913805CC53DF4F88839983AA83BB8398
:105BB000C45CD0408093960590939705A093980578
:105BC000B09399054090390550903A0560903B0597
:105BD00070903C0540929A0550929B0560929C05FE
:105BE00070929D050F920F92CDB6DEB60894C11C3F
:105BF000D11CE0909E05F0909F050091A0051091AA
:105C0000A1056091BE037091BF038091C003909184
:105C1000C10320E030E040E752E40E9437994B0195
:105C20005C01D6012D923C92CC53DF4F6881798183
:105C30008A819B81C45CD040A3019201A2EACA2E52
:105C4000A5E0DA2E0E94255580E090E0A0E0B0E0CB
:105C50008093BE039093BF03A093C003B093C1038E
:105C60000F900F900E94F6780E94267680919605FC
:105C700090919705A0919805B0919905809335056D
:105C800090933605A0933705B093380580919A0517
:105C900090919B05A0919C05B0919D05809339053D
:105CA00090933A05A0933B05B0933C0580919E05E7
:105CB00090919F05A091A005B091A10580933D050D
:105CC00090933E05A0933F05B09340058091C20399
:105CD000882329F488E50E942D21882321F080E083
:105CE00090E00E944E218091C203882329F489E527
:105CF0000E942D21882321F081E090E00E944E2116
:105D000088E50E942D218823D9F00E94392661154B
:105D1000710581059105A1F00E9444262091450559
:105D20003091460540914705509148050E9457988B
:105D30006093350570933605809337059093380549
:105D400089E50E942D218823D9F00E94392661150A
:105D5000710581059105A1F00E9444262091490515
:105D600030914A0540914B0550914C050E9457983F
:105D70006093390570933A0580933B0590933C05F9
:105D80008AE50E942D218823D9F00E9439266115C9
:105D9000710581059105A1F00E94442620914D05D1
:105DA00030914E0540914F05509150050E945798F3
:105DB00060933D0570933E0580933F0590934005A9
:105DC0008091C203882329F48AE50E942D2188232B
:105DD000D1F060913D0570913E0580913F05909115
:105DE0004005209160053091610540916205509118
:105DF00063050E94579860933D0570933E0580931C
:105E00003F0590934005609135057091360580916E
:105E10003705909138052091390530913A05409128
:105E20003B0550913C05E0903D05F0903E0500910A
:105E30003F0510914005F1E4CF2EF5E0DF2E0E94E2
:105E4000114F8091AB059091AC05A091AD05B0913B
:105E5000AE058093BE039093BF03A093C003B0939D
:105E6000C103809133059091340590939203809300
:105E700091030E94469560938205709383058093F9
:105E80008405909385050E94267682E390E09093A6
:105E9000FE038093FD030C946B4584E190E09093A6
:105EA000FE038093FD0380915D05882321F080919E
:105EB0005E05882329F5E9E4F3E0949108C0809118
:105EC000C00085FFFCCF9093C60031969491992332
:105ED000B1F7E5EEF5E0949108C08091C00085FF30
:105EE000FCCF9093C600319694919923B1F780919D
:105EF000C00085FFFCCF8AE08093C6000C946B4500
:105F00000E94F67883EC93E00E949C8FCE010D9660
:105F10000E940D506D857E858F859889609335052B
:105F200070933605809337059093380529893A890F
:105F30004B895C892093390530933A0540933B05A2
:105F400050933C05ED88FE880F89188DE0923D0541
:105F5000F0923E0500933F0510934005E1E4CE2EFC
:105F6000E5E0DE2E0E94114F0E94DE208091890321
:105F700090918A03A0918B03B0918C038093BE0310
:105F80009093BF03A093C003B093C103C354DF4FEA
:105F90001882CD5BD04022243324E0EAF0E0C754DD
:105FA000DF4FF983E883C95BD040C554DF4F1982C6
:105FB0001882CB5BD040C254DF4F19821882CE5B6F
:105FC000D04028C0C354DF4FF881CD5BD040FF23C1
:105FD00091F421E0C354DF4F2883CD5BD04080EAA9
:105FE000282E312C80E69FEFC754DF4F998388839A
:105FF000C95BD0400FC0C354DF4F1882CD5BD04087
:1060000022243324A0EAB0E0C754DF4FB983A88329
:10601000C95BD040C254DF4F88819981CE5BD040AC
:10602000880F991F880F991FE1E3F0E0EC0FFD1F27
:10603000E80FF91FCB54DF4FF983E883C55BD040ED
:106040001FE5412E512C4C0E5D1E480E591EC254A8
:10605000DF4F28813981CE5BD040CD54DF4F39836B
:106060002883C35BD040C954DF4F19821882C75BB5
:10607000D040C554DF4F88819981CB5BD040AA279F
:1060800097FDA095BA2FC853DF4F88839983AA83C1
:10609000BB83C85CD040CD54DF4FA881B981C35BBE
:1060A000D040AB2B29F4EE24FF2400EA10E410C00A
:1060B00060913D0570913E0580913F0590914005AE
:1060C00020E030E040EA50E40E9457987B018C01C8
:1060D000B101882777FD8095982F0E94D2993B01C6
:1060E0004C01C853DF4F688179818A819B81C85CEC
:1060F000D0400E94D2995B016C01C401B301A6019A
:1061000095010E946725CB54DF4FE881F981C55B7B
:10611000D0406193719381939193CB54DF4FF98376
:10612000E883C55BD040D2016D927D928D929C92A6
:106130001397F201A08AB18AC28AD38A80E090E0E4
:10614000A0E8BFE380A391A3A2A3B3A3CD54DF4FE4
:1061500028813981C35BD0402F5F3F4FCD54DF4F43
:1061600039832883C35BD040C954DF4F888199812C
:10617000C75BD0400196C954DF4F99838883C75BC2
:10618000D040A4E0B0E04A0E5B1E029749F0C7542D
:10619000DF4FE881F981C95BD0402E0E3F1E7BCFD7
:1061A000C254DF4F28813981CE5BD0402E5F3F4FF4
:1061B000C254DF4F39832883CE5BD040C554DF4FB4
:1061C00088819981CB5BD04080569F4FC554DF4F6B
:1061D00099838883CB5BD0402430310509F0F2CE1F
:1061E0008091AB059091AC05A091AD05B091AE0545
:1061F0008093BE039093BF03A093C003B093C103E9
:10620000809133059091340590939203809391038C
:106210000E94469560938205709383058093840560
:106220009093850584E090E063E070E0AE01415A10
:106230005F4F9E012F5C3F4F0E9477754C01EFEC42
:10624000F5E0949108C08091C00085FFFCCF909349
:10625000C600319694919923B1F7D4014D915D9187
:106260006D917C918EE295E022E030E00E94E41C8A
:10627000EAECF5E0949108C08091C00085FFFCCF66
:106280009093C600319694919923B1F7F40144811B
:106290005581668177818EE295E022E030E00E94B0
:1062A000E41CE5ECF5E0949108C08091C00085FF06
:1062B000FCCF9093C600319694919923B1F7D40105
:1062C00018964D915D916D917C911B978EE295E0B2
:1062D00022E030E00E94E41C8091C00085FFFCCFEA
:1062E0008AE08093C600B9E1AB2EB12CAC0EBD1E86
:1062F000F40140815181628173817058048115815C
:10630000268137813058C5010F2EF0E0CF2EF0E006
:10631000DF2EF0E8EF2EFFE3FF2EF02D0E94218EFE
:10632000C50163E872E00E946390AFE8AA2EB12C29
:10633000AC0EBD1EC501C98CDA8CEB8CFC8C0D8DAE
:106340001E8D2F8D38A149A15AA16BA17CA10E945D
:106350007491A3ECB3E0F50184E201900D928150B9
:10636000E1F7CE0185960E940D506DA17EA18FA10F
:1063700098A5609335057093360580933705909303
:10638000380529A53AA54BA55CA52093390530937E
:106390003A0540933B0550933C05E0906005F09032
:1063A00061050091620510916305E0923D05F09250
:1063B0003E0500933F0510934005F1E4CF2EF5E034
:1063C000DF2E0E94114FC4010E94AC0B0E94F67890
:1063D00082E00E9481760E94D2992091CD0730916F
:1063E000CE074091CF075091D0070E9437997B018B
:1063F0008C0160913505709136058091370590913B
:10640000380520E030E040E050E00E945798698372
:106410007A838B839C836091390570913A058091D2
:106420003B0590913C0520E030E040E050E00E94C8
:1064300057986D837E838F83988780913D059091D7
:106440003E05A0913F05B091400589879A87AB87AB
:10645000BC872DB73EB72A5230400FB6F8943EBFE6
:106460000FBE2DBFEDB7FEB731969F0143EC53E051
:1064700084E2DA010D90AD01D9010D929D018150A8
:10648000C1F7CE01019695A384A3CE01059697A3EB
:1064900086A3CE01099691A780A70E94288F6985BF
:1064A0007A858B859C85A80197010E94569820913A
:1064B0003D0530913E0540913F05509140050E94B9
:1064C00057987B018C01CB01D80180933D059093B7
:1064D0003E05A0933F05B0934005EDB7FEB7BA96D1
:1064E0000FB6F894FEBF0FBEEDBF609135057091F9
:1064F0003605809137059091380520913905309106
:106500003A0540913B0550913C05E1E4CE2EE5E093
:10651000DE2E0E94114F82E390E09093FE03809361
:10652000FD03E7EBF5E0949108C08091C00085FF82
:10653000FCCF9093C600319694919923B1F7809146
:10654000C00085FFFCCF8AE08093C6000C946B45A9
:106550002091AB033091AC0337FD0DC0C901880F0A
:10656000991F820F931F6091B5037091B6038D58E8
:106570009A4F0E945B480E94F6780E94DE2080912C
:10658000890390918A03A0918B03B0918C0380932F
:10659000BE039093BF03A093C003B093C1030E94B6
:1065A000F523E3EBF5E0949108C08091C00085FFEE
:1065B000FCCF9093C600319694919923B1F7EEEAFF
:1065C000F5E0949108C08091C00085FFFCCF9093C6
:1065D000C600319694919923B1F7409135055091B9
:1065E000360560913705709138058EE295E022E01E
:1065F00030E00E94E41CE9EAF5E0949108C0809143
:10660000C00085FFFCCF9093C600319694919923EA
:10661000B1F74091390550913A0560913B05709171
:106620003C058EE295E022E030E00E94E41CE4EAC2
:10663000F5E0949108C08091C00085FFFCCF909355
:10664000C600319694919923B1F740913D05509140
:106650003E0560913F05709140058EE295E022E095
:1066600030E00E94E41CE2EAF5E0949108C08091D9
:10667000C00085FFFCCF9093C6003196949199237A
:10668000B1F78091AB059091AC05A091AD05B091AB
:10669000AE058093BE039093BF03A093C003B09355
:1066A000C1038091330590913405909392038093B8
:1066B00091030E94469560938205709383058093B1
:1066C0008405909385052091AB033091AC0337FF8F
:1066D00002C00C946B45C901880F991F820F931F4C
:1066E0006091B7037091B8038D589A4F0E945B4830
:1066F0000C946B451092A6050C946B4581E0809339
:10670000A6050C946B4585E40E942D21882311F485
:106710000E94F678A5E38A2EA5E09A2EF5E46F2E66
:10672000F5E07F2EAA24BB24F501EA5AFB4F8081B5
:106730000E942D218823E9F1F3E0AF1669F40E944D
:106740004426D4016D937D938D939C93139781E49C
:1067500095E00E94F44E2DC00E944426F301208152
:106760003181428153810E945798D4016D937D936A
:106770008D939C93139760913505709136058091A8
:106780003705909138052091390530913A054091AF
:106790003B0550913C05E0903D05F0903E05009191
:1067A0003F0510914005E1E4CE2EE5E0DE2E0E948B
:1067B000114F0894A11CB11CE4E0F0E08E0E9F1E66
:1067C0006E0E7F1EF4E0AF16B10409F0ADCF0C944D
:1067D0006B458DE40E942D21882311F40C948D4487
:1067E0000E9444260E949F99683C710511F40C9404
:1067F000023E693C71050CF08CC06936710509F4E4
:1068000072C26A3671050CF041C06135710509F438
:10681000C1C662357105DCF46F31710509F436C10A
:106820006032710554F46131710509F429C1623196
:10683000710511F00C946B45CBC66A32710509F4F1
:10684000D3C16035710511F00C946B459FC664355A
:10685000710509F4BDC66535710554F462357105DD
:1068600009F4ADC66335710511F00C946B45ABC6E8
:106870006C35710509F420C76836710509F4FEC14D
:106880006535710511F00C946B45FBC663377105D6
:1068900009F49BC764377105DCF46D36710509F4A2
:1068A00046C36E36710554F46A36710509F431C673
:1068B0006B36710511F00C946B455CC66037710541
:1068C00009F4FCC16237710511F00C946B459FC748
:1068D0006837710511F40C94FC3C6937710554F468
:1068E0006537710509F481C76737710511F00C949C
:1068F0006B45C3C06C38710509F4E4C16E3B71058A
:1069000009F4FEC46937710511F00C946B450C94C1
:10691000013D21E06033720711F40C946A4131E0CB
:10692000613373070CF051C06C3D710511F40C9488
:10693000593F6D3D710504F56C3C710511F40C94E3
:10694000BD3E6D3C710564F4693C710511F40C9415
:106950007C3E6B3C710511F00C946B450C949F3E92
:106960006D3C710511F40C94DD3E6E3C710511F027
:106970000C946B450C943B3F81E06831780711F42F
:106980000C94E53F91E06931790764F46D3D710540
:1069900011F40C94683F623E710511F00C946B4544
:1069A0000C948F3FA1E06E327A0711F40C941842D8
:1069B000B1E06F327B0714F00C9427426D527140A6
:1069C00011F00C946B450C949240F1E0643F7F070A
:1069D00011F40C94904221E0653F720724F531E0F8
:1069E0006039730711F40C94674281E061397807CC
:1069F0006CF491E06E35790711F40C94D0436F5527
:106A0000714011F00C946B450C941044B1E0613965
:106A10007B0711F40C946A426259714011F00C9496
:106A20006B450C947D42F1E0673F7F0711F40C94B5
:106A3000994221E0683F72076CF431E0653F7307CB
:106A400011F40C949342665F714011F00C946B4505
:106A50000C94964293E06B38790711F40C94A1439F
:106A6000A3E0673E7A0711F40C94784463557340B1
:106A700011F00C946B450C949C42EFE8F2E0CDC70A
:106A800017981698159814980C946B450E94469583
:106A900060936E0570936F058093700590937105F8
:106AA00020916A0530916B0540916C0550916D0500
:106AB000621B730B840B950B28EE33E040E050E033
:106AC0000E94289DF22EE32ED42EC52EEDB7FEB7E0
:106AD00038970FB6F894FEBF0FBEEDBF0DB71EB7C7
:106AE0000F5F1F4FCE018F5B9F4F9283818383E99E
:106AF00095E0D80113969C938E931297622F732F73
:106B0000842F952F2CE330E040E050E00E94289D38
:106B1000F801358324836F2D7E2D8D2D9C2D2CE344
:106B200030E040E050E00E94289DD80117967C9309
:106B30006E9316970E94E40EE9E4F3E094912DB76A
:106B40003EB7285F3F4F0FB6F8943EBF0FBE2DBF34
:106B500008C08091C00085FFFCCF9093C60031969D
:106B600094919923B1F7FE01EF5BFF4F07C080912D
:106B7000C00085FFFCCF31969093C6009081992389
:106B8000B1F78091C00085FFFCCF8AE08093C600FA
:106B900080912108882311F40C946B4510922108F0
:106BA00080916405082F10E0000F111F0955124F46
:106BB000D8016D917C91882777FD8095982F0E9450
:106BC000D2992091EB033091EC034091ED03509169
:106BD000EE030E943E9B181614F00C946B45F801CE
:106BE000118210820C946B4583E50E942D2188232D
:106BF00011F40C946B450E9444260E949F997B01DE
:106C00008C016B0180E50E942D21882369F0F7FC3F
:106C10000BC0FFEFEF16F10409F034F40E94442694
:106C20000E949F998B0102C00DE010E0EAE5F4E0BC
:106C3000808191818017910711F40C946B453296F5
:106C400024E0E239F207A1F70830110529F4D092C7
:106C50006705C092660504C017FF02C00C946B451F
:106C6000802F61E00E940F96802F6C2D0E94C296AB
:106C7000802FB6010E9423970C946B4588E690E024
:106C80000E944D26882311F00C946B4583E50E94E9
:106C90002D21882379F00E94442620917705022F28
:106CA00010E0000F111F0955124F0E949F99D80143
:106CB0006D937C930E948D820C946B450E94BB1D4A
:106CC0000C946B4583E50E942D21882311F40C94CC
:106CD0006B450E9444260E949F997093AA0D609371
:106CE000A90D0C946B4589E690E00E944D268823FF
:106CF00011F00C946B45EDE8F5E0949108C080919B
:106D0000C00085FFFCCF9093C600319694919923E3
:106D1000B1F7E0917705F0E0EE0FFF1FEE0FFF1FD8
:106D2000E355F24F40815181628173818EE295E09B
:106D300021E030E00E94E41CEAE8F5E0949108C00C
:106D40008091C00085FFFCCF9093C600319694914E
:106D50009923B1F7E0917705F0E0EE0FFF1FE955B9
:106D6000F24F60817181882777FD8095982F0E946E
:106D7000D299AB01BC018EE295E021E030E00E94A7
:106D8000E41CE6E8F5E0949108C08091C00085FF1E
:106D9000FCCF9093C600319694919923B1F740911E
:106DA000B30D5091B40D6091B50D7091B60D8EE29A
:106DB00095E021E030E00E94E41CE3E8F5E09491E6
:106DC00008C08091C00085FFFCCF9093C60031962B
:106DD00094919923B1F76091A90D7091AA0D88271C
:106DE00077FD8095982F0E94D299AB01BC018EE26D
:106DF00095E021E030E00E94E41CE0E8F5E09491A9
:106E000008C08091C00085FFFCCF9093C6003196EA
:106E100094919923B1F78EE295E060E070E04AE04A
:106E200050E00E94111CEEE7F5E0949108C08091BB
:106E3000C00085FFFCCF9093C600319694919923B2
:106E4000B1F74091AD0D5091AE0D6091AF0D7091C5
:106E5000B00D8EE295E021E030E00E94E41CEBE70B
:106E6000F5E0949108C08091C00085FFFCCF90931D
:106E7000C600319694919923B1F76091A70D709156
:106E8000A80D882777FD8095982F0E94D299AB0195
:106E9000BC018EE295E021E030E00E94E41CE7E7CF
:106EA000F5E0949108C08091C00085FFFCCF9093DD
:106EB000C600319694919923B1F7809177050E948D
:106EC000D281BC018EE295E04AE050E00E94111CA4
:106ED000E2E7F5E0949108C08091C00085FFFCCF07
:106EE0009093C600319694919923B1F78FEF9FEF5D
:106EF0000E94D281BC018EE295E04AE050E00E94FF
:106F0000111CE8EAF2E007C08091C00085FFFCCFC9
:106F100031969093C60090819923B1F78091C0007B
:106F200085FFFCCF8AE08093C6000C948E458DE6E9
:106F300090E00E944D26882311F00C946B4510922E
:106F4000210883E50E942D21882399F00E94442680
:106F500020917705022F10E0000F111F0955124FE5
:106F60000E949F99F8017183608381E08093B90347
:106F700016C082E50E942D21882389F00E944426B4
:106F800020917705022F10E0000F111F0955124FB5
:106F90000E949F99D8016D937C931092B90383E569
:106FA0000E942D21882351F00E9444266093EB0318
:106FB0007093EC038093ED039093EE0382E40E94C0
:106FC0002D21882351F00E9444266093E70370939B
:106FD000E8038093E9039093EA0386E40E942D215D
:106FE000882369F00E9444266093EF037093F003B6
:106FF0008093F1039093F20381E0809321080E9433
:107000008D820E9446954B015C0120917705022FED
:1070100010E010927605000F111FF801E955F24FAC
:1070200060817181882777FD8095982F0E94D29981
:10703000000F111F0355124FF80120813181428149
:1070400053810E943E9B18161CF481E080937605C4
:10705000CC24CA94DC2C7601EFE6F5E05490EBE604
:10706000F5E06490E7E6F5E074906AE0462E3BC1F7
:10707000952DEFE6F5E008C08091C00085FFFCCFBC
:107080009093C600319694919923B1F7E0917705DA
:10709000F0E0EE0FFF1FEE0FFF1FE355F24F4081B0
:1070A0005181628173818EE295E021E030E00E949F
:1070B000E41C962DEBE6F5E008C08091C00085FF4A
:1070C000FCCF9093C600319694919923B1F76091CB
:1070D00077058EE295E070E04AE050E00E94111CD6
:1070E000972DE7E6F5E008C08091C00085FFFCCF52
:1070F0009093C600319694919923B1F7F7FE03C09F
:10710000E9EAF2E02CC00E9446956C197D098E09CF
:107110009F090E94D0999B01AC0160E070E08AEF6A
:1071200093E40E94569820E030E04AE754E40E943D
:1071300037990E94A499AB01BC018EE295E02AE048
:1071400030E00E94C21B8091C00085FFFCCF0EC0C2
:107150008091C00085FFFCCF31969093C60090814E
:107160009923B1F78091C00085FFFCCF4092C60003
:107170000E9446954B015C010E94E2860E94122A01
:10718000FFEFCF16FFEFDF06FFEFEF06FFEFFF0683
:1071900009F052C080917605E0917705882331F19E
:1071A000F0E08F01000F111F000F111F0355124F48
:1071B000EE0FFF1FE955F24F60817181882777FD3F
:1071C0008095982F0E94D29920E030E040E251E46F
:1071D0000E9456989B01AC01D8016D917D918D91D3
:1071E0009C910E943E9B87FF58C05EC0F0E08F01DB
:1071F000000F111F000F111F0355124FEE0FFF1F3D
:10720000E955F24F60817181882777FD8095982F2D
:107210000E94D29920E030E040E251E40E94579869
:107220009B01AC01F80160817181828193810E9490
:107230003099181694F538C0F7FC36C0E091770500
:10724000F0E08F01000F111F000F111F0355124FA7
:10725000EE0FFF1FE955F24F60817181882777FD9E
:107260008095982F0E94D2999B01AC01D8016D9115
:107270007D918D919C910E9456980E949F9997FFB5
:1072800007C090958095709561957F4F8F4F9F4F68
:107290006B307105810591053CF00E944695AC016B
:1072A000CB01DA016C017D01BFEFCB16BFEFDB062E
:1072B000BFEFEB06BFEFFB06B1F0F7FE02C00C9488
:1072C0006E450E9446956C197D0980E090E00E9411
:1072D000D09920E030E04AEF53E40E9430998823AF
:1072E00014F00C946E450E944695681979098A0934
:1072F0009B09695E73408040904008F0B9CE3CCF56
:1073000083E50E942D21882361F00E9444260E947B
:107310009F997093AA0D6093A90D81E08093B903A2
:107320000FC082E50E942D21882351F00E9444263F
:107330000E949F997093AA0D6093A90D1092B903B2
:107340000E9446957B018C01109276056091A90DF3
:107350007091AA0D882777FD8095982F0E94D29969
:107360002091B30D3091B40D4091B50D5091B60DF3
:107370000E943E9B18160CF080C081E08093760539
:107380007CC00E9446956E197F09800B910B695E47
:1073900073408040904008F46BC0E0916405F0E0D9
:1073A000EE0FFF1FEE0FFF1FE355F24F408151819B
:1073B000628173819B2DE4E6F5E008C08091C000F6
:1073C00085FFFCCF9093C600319694919923B1F735
:1073D0008EE295E022E030E00E94E41C9C2DE0E685
:1073E000F5E008C08091C00085FFFCCF9093C600F7
:1073F000319694919923B1F7609164058EE295E0FE
:1074000070E04AE050E00E94111C9D2DECE5F5E093
:1074100008C08091C00085FFFCCF9093C6003196D4
:1074200094919923B1F74091B30D5091B40D6091AF
:10743000B50D7091B60D8EE295E021E030E00E942E
:10744000E41CE8EAF2E007C08091C00085FFFCCFB1
:1074500031969093C60090819923B1F78091C00036
:1074600085FFFCCFA092C6000E9446957B018C014F
:107470000E94E2860E94122A0BC0E4E6F5E0B49076
:10748000E0E6F5E0C490ECE5F5E0D4907AE0A72ED4
:10749000809176052091A90D3091AA0D8823A9F03D
:1074A000B901882777FD8095982F0E94D299209165
:1074B000B30D3091B40D4091B50D5091B60D0E94B1
:1074C0003E9B18160CF45DCF18C0B901882777FDD4
:1074D0008095982F0E94D2992091B30D3091B40DD0
:1074E0004091B50D5091B60D0E94309988232CF42F
:1074F0008091B903882309F444CF0E944695609394
:1075000082057093830580938405909385050C9480
:107510006B4583E50E942D21882321F10E9444269A
:1075200020E030E040E050E00E94309988231CF4D5
:1075300060E070E011C00E94442620E030E04FE798
:1075400053E40E943E9B18161CF46FEF70E004C0D9
:107550000E9444260E949F99709367056093660578
:107560000C946B458FEF90E09093670580936605D0
:107570000C946B4510926505109267051092660594
:1075800010926905109268050C946B459D9AA59818
:107590000C946B450E948E820E94F678149A0E9489
:1075A0000279109267051092660568EE73E080E03C
:1075B00090E00E9454959D9AA59A0C946B45109268
:1075C00032050C946B4581E0809332050C946B4539
:1075D00083E50E942D218823A1F00E94442620E00B
:1075E00030E04AE754E40E94109C0E94A499609302
:1075F000BA037093BB038093BC039093BD030C94B8
:107600006B4588E50E942D21882311F00C94834559
:1076100089E50E942D21882311F00C9483458AE589
:107620000E942D21882311F00C94834585E40E944B
:107630002D21882311F00C9483450E94F678149A2A
:107640000E9402790C946B45179A10925D0589E5AA
:107650000E942D21882319F0169A10925E058AE562
:107660000E942D21882319F0159A10925F0585E458
:107670000E942D21882311F40C946B45149A0C94CC
:107680006B4583E50E942D21882311F40C946B45F2
:107690000E94442620E030E04AE754E40E94109C17
:1076A0000E94A4996093860570938705809388054E
:1076B000909389050C946B4565EC662E67E0762EF9
:1076C00055EB252E57E0352E41E0442E48E0542E50
:1076D00088249924F401EA5AFB4F80810E942D21CD
:1076E000882309F460C023E0821609F054C00E9488
:1076F00044265B016C0120E030E040EA51E40E9446
:10770000309988230CF041C0D3016D917D918D910A
:107710009C91A60195010E9437997B018C01609193
:10772000F9077091FA078091FB079091FC07A80177
:1077300097010E94109C6093F9077093FA07809359
:10774000FB079093FC07F101608171818281938135
:10775000A80197010E94109CD1016D937D938D9398
:107760009C931397F20160817181828193810E94C1
:10777000D099A80197010E94109C0E94A499D2015F
:107780006D937D938D939C931397F301A082B182A7
:10779000C282D38208C00E944426D3016D937D9398
:1077A0008D939C9313970894811C911CE4E0F0E066
:1077B0006E0E7F1E2E0E3F1E4E0E5F1EF4E08F16C5
:1077C000910409F087CF0C946B45EFE8F4E09491B5
:1077D00008C08091C00085FFFCCF9093C600319611
:1077E00094919923B1F70C946B458091AF059091DA
:1077F000B00505966AE270E00E94C20EFC01009797
:1078000011F40C946B45319710820C946B45ECE8A5
:10781000F4E0949108C08091C00085FFFCCF909364
:10782000C600319694919923B1F740913505509156
:10783000360560913705709138058EE295E022E0BB
:1078400030E00E94E41CE8E8F4E0949108C08091E4
:10785000C00085FFFCCF9093C60031969491992388
:10786000B1F74091390550913A0560913B0570910F
:107870003C058EE295E022E030E00E94E41CE4E862
:10788000F4E0949108C08091C00085FFFCCF9093F4
:10789000C600319694919923B1F740913D055091DE
:1078A0003E0560913F05709140058EE295E022E033
:1078B00030E00E94E41CE0E8F4E0949108C080917C
:1078C000C00085FFFCCF9093C60031969491992318
:1078D000B1F7409141055091420560914305709187
:1078E00044058EE295E022E030E00E94E41CE5E7EA
:1078F000F4E0949108C08091C00085FFFCCF909384
:10790000C600319694919923B1F780E00E94817668
:107910000E94D2992091C5073091C6074091C707B0
:107920005091C8070E943799AB01BC018EE295E0E7
:1079300022E030E00E94E41CE1E7F4E0949108C00A
:107940008091C00085FFFCCF9093C6003196949142
:107950009923B1F781E00E9481760E94D29920910B
:10796000C9073091CA074091CB075091CC070E94BC
:107970003799AB01BC018EE295E022E030E00E9435
:10798000E41CEDE6F4E0949108C08091C00085FF0E
:10799000FCCF9093C600319694919923B1F782E081
:1079A0000E9481760E94D2992091CD073091CE0716
:1079B0004091CF075091D0070E943799AB01BC018D
:1079C0008EE295E022E030E00E94E41CE8EAF2E07A
:1079D00007C08091C00085FFFCCF31969093C60010
:1079E00090819923B1F78091C00085FFFCCF8AE098
:1079F0008093C6000C946B4580E00E942D760C9419
:107A00006B4581E00E942D760C946B458091C000FF
:107A100085FFFCCF31969093C60090819923B1F7F2
:107A20008091C00085FFFCCF8AE08093C600E5E628
:107A3000F4E0949108C08091C00085FFFCCF909342
:107A4000C600319694919923B1F71E9B03C0EBEACF
:107A5000F2E00AC0E0EBF2E007C08091C00085FFD1
:107A6000FCCF31969093C60090819923B1F7809115
:107A7000C00085FFFCCF8AE08093C600EDE5F4E00E
:107A8000949108C08091C00085FFFCCF9093C60000
:107A9000319694919923B1F7379B03C0EBEAF2E05A
:107AA0000AC0E0EBF2E007C08091C00085FFFCCF88
:107AB00031969093C60090819923B1F78091C000D0
:107AC00085FFFCCF8AE08093C600E5E5F4E0949161
:107AD00008C08091C00085FFFCCF9093C60031960E
:107AE00094919923B1F71D9B03C0EBEAF2E00AC021
:107AF000E0EBF2E007C08091C00085FFFCCF31963B
:107B00009093C60090819923B1F78091C00085FFC2
:107B1000FCCF8AE08093C600EDE4F4E0949108C0C5
:107B20008091C00085FFFCCF9093C6003196949160
:107B30009923B1F7029B03C0EBEAF2E00AC0E0EB45
:107B4000F2E007C08091C00085FFFCCF3196909392
:107B5000C60090819923B1F78091C00085FFFCCFCA
:107B60008AE08093C600E5E4F4E0949108C0809137
:107B7000C00085FFFCCF9093C60031969491992365
:107B8000B1F71C9B03C0EBEAF2E00AC0E0EBF2E0C5
:107B900007C08091C00085FFFCCF31969093C6004E
:107BA00090819923B1F78091C00085FFFCCF8AE0D6
:107BB0008093C600EDE3F4E0949108C08091C0008A
:107BC00085FFFCCF9093C600319694919923B1F72D
:107BD000019B03C0EBEAF2E00AC0E0EBF2E007C071
:107BE0008091C00085FFFCCF31969093C6009081B4
:107BF0009923B1F78091C00085FFFCCF8AE0809384
:107C0000C60069C784E40E942D21882309F463C754
:107C10000E94442620E030E040E05FE30E94109C98
:107C20007B018C0120E030E040E050E00E94309980
:107C3000882359F40F2EF0E0CF2EF0E0DF2EF0E88D
:107C4000EF2EFFE3FF2EF02D11C0C801B701A801F0
:107C500097010E94109C9B01AC01CA012BED3FE0F3
:107C600049E450E40E94109C6B017C018091640502
:107C70008093770584E50E942D21882321F10E94BD
:107C800044260E94A499609377056623E1F0E9E415
:107C9000F3E0949108C08091C00085FFFCCF9093E1
:107CA000C600319694919923B1F7EAEBF2E007C050
:107CB0008091C00085FFFCCF31969093C6009081E3
:107CC0009923B1F708C780917705082F10E0000FBE
:107CD000111F000F111F09561C4F60E070E080E873
:107CE0009FE3A70196010E943799D8016D937D9378
:107CF0008D939C931397EFC606E514E025EDE22ED5
:107D000027E0F22EF80180810E942D21882351F076
:107D10000E9444260E94A499D7016D937D938D9370
:107D20009C9313970F5F1F4FE4E0F0E0EE0EFF1EF1
:107D3000F4E00A351F0731F70E94C94ECCC606E5AC
:107D400014E095EBE92E97E0F92ED8018C910E9472
:107D50002D21882339F00E944426F7016083718326
:107D6000828393830F5F1F4F24E030E0E20EF31E07
:107D700034E00A35130749F7AEC683E50E942D218A
:107D8000882351F00E9444266093E9077093EA0724
:107D90008093EB079093EC0784E50E942D218823C4
:107DA00009F499C60E9444266093ED077093EE078C
:107DB0008093EF079093F0078EC683E50E942D21F4
:107DC000882351F00E9444266093E5077093E607EC
:107DD0008093E7079093E80784E50E942D2188238C
:107DE00051F00E9444266093FD077093FE07809334
:107DF000FF079093000882E40E942D21882361F000
:107E00000E9444260E94A4996093B1077093B20720
:107E10008093B3079093B40788E50E942D218823AF
:107E200051F00E9444266093F1077093F20780930B
:107E3000F3079093F4078AE50E942D21882351F0DF
:107E40000E9444266093F5077093F6078093F70726
:107E50009093F80785E40E942D21882309F43BC6FE
:107E60000E9444266093F9077093FA078093FB07FA
:107E70009093FC0730C606E514E085E4E82E85E023
:107E8000F82ED8018C910E942D21882339F00E9470
:107E90004426F70160837183828393830F5F1F4FB2
:107EA00024E030E0E20EF31E34E00935130749F711
:107EB00012C683E50E942D21882309F40CC60E9476
:107EC00044260E949F99709392036093910303C686
:107ED00083E50E942D21882309F4FDC50E944426D4
:107EE0000E949F997B018C0184E50E942D218823AB
:107EF00089F08DED90E00E944D26882309F0EBC5B6
:107F0000E0917705F0E0EE0FFF1FEB56FC4FF1829A
:107F1000E082E1C5F0929403E0929303DCC580E532
:107F20000E942D21882309F4D6C50E9444260E9470
:107F30009F997B0183E50E942D21882319F40FEF7F
:107F40001FEF05C00E9444260E949F998B01C80123
:107F50000196039708F0BFC5EAE5F4E080819181BE
:107F60008E159F0509F4B7C5329684E0E239F8070B
:107F7000A9F7F7FCB0C50E94F678DE2C8E2D60E0E4
:107F80000E940F960115110541F00130110579F09D
:107F90009FEF0F3F190791F403C000E010E00EC0FF
:107FA0008E2D0E94F49600E010E0892B39F401E058
:107FB00010E004C00E94E2860E94122A8D2D0E94C9
:107FC000F49680179107B1F786C580E50E942D21B0
:107FD000882319F40FEF1FEF05C00E9444260E946A
:107FE0009F998B0183E50E942D21882309F446C0C7
:107FF0000E9444260115110551F40E949F999B018E
:10800000AC0183E795E0B9010E945B4864C5E9E4EF
:10801000F3E0949108C08091C00085FFFCCF90935D
:10802000C600319694919923B1F7E1EDF2E007C0D3
:108030008091C00085FFFCCF31969093C60090815F
:108040009923B1F78EE295E0B8014AE050E00E9432
:10805000111CE8EDF2E007C08091C00085FFFCCF65
:1080600031969093C60090819923B1F78091C0001A
:1080700085FFFCCF8AE08093C6002DC517FD2BC578
:10808000E6EEF2E007C08091C00085FFFCCF31969C
:108090009093C60090819923B1F7E9EEF2E007C012
:1080A0008091C00085FFFCCF31969093C6009081EF
:1080B0009923B1F78EE295E0B8014AE050E00E94C2
:1080C000111CE1EFF2E007C08091C00085FFFCCFFA
:1080D00031969093C60090819923B1F7C801880F1B
:1080E000991F800F911F8D589A4F91D7BC018EE236
:1080F00095E04AE050E00E94111CE8EAF2E007C077
:108100008091C00085FFFCCF31969093C60090818E
:108110009923B1F78091C00085FFFCCF8AE080935E
:10812000C600D9C480E50E942D21882351F00E9409
:10813000442660930404709305048093060490938E
:10814000070489E40E942D21882361F00E944426BF
:108150000E94AB82609308047093090480930A0420
:1081600090930B0484E40E942D21882361F00E94E7
:1081700044260E94B78260930C0470930D04809390
:108180000E0490930F0483E40E942D21882351F064
:108190000E9444266093100470931104809312048B
:1081A000909313040E94A581E6EEF2E007C080914F
:1081B000C00085FFFCCF31969093C6009081992333
:1081C000B1F7E4EFF2E007C08091C00085FFFCCF7B
:1081D00031969093C60090819923B1F740910404A1
:1081E0005091050460910604709107048EE295E0B9
:1081F00022E030E00E94E41CE8EFF2E007C080914A
:10820000C00085FFFCCF31969093C60090819923E2
:10821000B1F7609108047091090480910A0490916B
:108220000B040E94B182AB01BC018EE295E022E01A
:1082300030E00E94E41CECEFF2E007C08091C00047
:1082400085FFFCCF31969093C60090819923B1F7BA
:1082500060910C0470910D0480910E0490910F04B4
:108260000E94BD82AB01BC018EE295E022E030E0CD
:108270000E94E41CE0E0F3E007C08091C00085FFAD
:10828000FCCF31969093C60090819923B1F740912D
:1082900010045091110460911204709113048EE245
:1082A00095E022E030E00E94E41CE8EAF2E007C03A
:1082B0008091C00085FFFCCF31969093C6009081DD
:1082C0009923B1F78091C00085FFFCCF8AE08093AD
:1082D000C60001C480E50E942D21882351F00E9430
:1082E00044266093140470931504809316049093AD
:1082F000170489E40E942D21882361F00E944426FE
:108300000E94AB82609318047093190480931A043E
:1083100090931B0484E40E942D21882361F00E9425
:1083200044260E94B78260931C0470931D048093BE
:108330001E0490931F040E94A581E6EEF2E007C0A0
:108340008091C00085FFFCCF31969093C60090814C
:108350009923B1F7E4EFF2E007C08091C00085FFF8
:10836000FCCF31969093C60090819923B1F740914C
:1083700014045091150460911604709117048EE254
:1083800095E022E030E00E94E41CE8EFF2E007C054
:108390008091C00085FFFCCF31969093C6009081FC
:1083A0009923B1F7609118047091190480911A040F
:1083B00090911B040E94B182AB01BC018EE295E05A
:1083C00022E030E00E94E41CECEFF2E007C0809174
:1083D000C00085FFFCCF31969093C6009081992311
:1083E000B1F760911C0470911D0480911E0490915E
:1083F0001F040E94BD82AB01BC018EE295E022E029
:1084000030E00E94E41CE8EAF2E007C08091C0007E
:1084100085FFFCCF31969093C60090819923B1F7E8
:108420008091C00085FFFCCF8AE08093C60053C3D3
:1084300083E50E942D21882329F460E070E080E02C
:1084400090E002C00E9444260E94C04E44C385E4CE
:108450000E942D21882319F4CC24DD2412C00E940F
:1084600044260E949F996B0177FF0BC00F2EF0E00E
:10847000EF2EF0E0FF2EFCE80F2FF2E41F2FF02D7F
:108480000AC00F2EF0E0EF2EF0E0FF2EF6E10F2FE6
:10849000F3E41F2FF02D83E50E942D21882321F086
:1084A0000E9444267B018C0183E40E942D218823B5
:1084B00019F425E030E005C00E9444260E949F99EF
:1084C0009B01C801B701A6010E94808904C30E94D4
:1084D000F67801C32091AB033091AC0337FDFBC2AA
:1084E000C901880F991F820F931F6091B503709186
:1084F000B6038D589A4FDFD5EEC22091AB03309171
:10850000AC0337FDE8C2C901880F991F820F931F82
:108510006091B7037091B8038D589A4FCCD5DBC2E8
:108520000E947711D8C20E94BC18D5C20E94ED13D8
:10853000D2C20E948615CFC28AE50E942D218823CF
:1085400009F4B8C00E9444267B018C0120E030E091
:1085500040E751EC0E943E9B88230CF44EC0C801BA
:10856000B70120E030E040EA50E40E94309918164C
:108570000CF443C0D801C701B058809360059093B4
:108580006105A0936205B0936305E9E4F3E094917B
:1085900008C08091C00085FFFCCF9093C600319643
:1085A00094919923B1F7E1E3F4E0949108C08091AC
:1085B000C00085FFFCCF9093C6003196949199231B
:1085C000B1F78091C00085FFFCCF8AE08093C600A0
:1085D000E8EAF2E007C08091C00085FFFCCF319649
:1085E0009093C60090819923B1F78091C00085FFD8
:1085F000FCCF8AE08093C6006EC2E9E4F3E0949178
:1086000008C08091C00085FFFCCF9093C6003196D2
:1086100094919923B1F7E8E2F4E0949108C0809135
:10862000C00085FFFCCF9093C600319694919923AA
:10863000B1F7E0E2F4E0949108C08091C00085FFBA
:10864000FCCF9093C600319694919923B1F78EE2B6
:1086500095E061EF7FEF4AE050E00E94111CE8E1F5
:10866000F4E0949108C08091C00085FFFCCF909306
:10867000C600319694919923B1F78EE295E065E0BA
:1086800070E04AE050E00E94111CE8EAF2E007C006
:108690008091C00085FFFCCF31969093C6009081F9
:1086A0009923B1F78091C00085FFFCCF8AE08093C9
:1086B000C60011C2E9E4F3E0949108C08091C000C3
:1086C00085FFFCCF9093C600319694919923B1F722
:1086D000ECE0F4E0949108C08091C00085FFFCCFED
:1086E0009093C600319694919923B1F78091C00080
:1086F00085FFFCCF8AE08093C600409160055091D1
:108700006105609162057091630570588EE295E095
:1087100022E030E00E94E41CE8EAF2E007C0809129
:10872000C00085FFFCCF31969093C60090819923BD
:10873000B1F78091C00085FFFCCF8AE08093C6002E
:10874000CAC188E50E942D21882351F00E94442649
:108750000E949F999B01AC0180E0B9010E942178A1
:108760008AE50E942D21882351F00E9444260E9410
:108770009F999B01AC0181E0B9010E94217885E4B9
:108780000E942D21882309F4A6C10E9444260E943C
:108790009F999B01AC0182E0B9010E9421789BC1A5
:1087A00083E50E942D21882319F400E010E00FC01A
:1087B00010E00E9444260E94A4999B01AC01812FE5
:1087C000622F0E94CC771F5F153099F7EECFF8012A
:1087D000EA5AFB4F80810E942D21882351F00E948C
:1087E00044260E94A4999B01AC01802F622F0E9415
:1087F000CC770F5F1F4F0430110549F782E40E94C8
:108800002D21882351F00E9444260E94A4999B01A7
:10881000AC0184E0622F0E94CC770E94B2765BC1EB
:1088200083E50E942D21882309F45FC00E9444261D
:108830000E949F996130710529F06230710509F03D
:1088400054C029C000E010E0F801EA5AFB4F8081D3
:108850000E942D21882359F00E9444260E949F994E
:108860009B01AC01802F622F4FEF0E948E770F5F2C
:108870001F4F0430110541F782E40E942D21882307
:10888000A1F10E9444260E949F999B01AC0184E0C3
:10889000622F4FEF28C000E010E0F801EA5AFB4FCA
:1088A00080810E942D21882359F00E9444260E9435
:1088B0009F999B01AC01802F6FEF422F0E948E7712
:1088C0000F5F1F4F0430110541F782E40E942D21F4
:1088D000882359F00E9444260E949F999B01AC0175
:1088E00084E06FEF422F0E948E770E94B276F3C031
:1088F0001092720580917C0590917D05A0917E0576
:10890000B0917F058093780590937905A0937A05BF
:10891000B0937B050E943F20DEC084E50E942D219C
:10892000882309F48DC00E9444260E94A499262F12
:10893000609377056623B9F1E9E4F3E0949108C008
:108940008091C00085FFFCCF9093C6003196949132
:108950009923B1F7E4E0F3E007C08091C00085FF00
:10896000FCCF31969093C60090819923B1F78EE2A7
:1089700095E0622F40E050E00E94CD1BE6E0F3E07E
:1089800007C08091C00085FFFCCF31969093C60050
:1089900090819923B1F78091C00085FFFCCF8AE0D8
:1089A0008093C60098C086E40E942D218823E1F0C0
:1089B0000E9444267B018C016093A7057093A80553
:1089C0008093A9059093AA0520E030E040E050E0B4
:1089D0000E943E9B181644F4E092BE03F092BF033F
:1089E0000093C0031093C103E9E4F3E0949108C03D
:1089F0008091C00085FFFCCF9093C6003196949182
:108A00009923B1F7E7E1F3E007C08091C00085FF4B
:108A1000FCCF31969093C60090819923B1F7609175
:108A200064058EE295E070E04AE050E00E94111C7F
:108A30008091C00085FFFCCF8AE08093C6004BC0C8
:108A4000E9E4F3E0949108C08091C00085FFFCCF79
:108A50009093C600319694919923B1F7E9EFF3E032
:108A6000949108C08091C00085FFFCCF9093C60010
:108A7000319694919923B1F72091B1053091B205C7
:108A800080E690E0289FF001299FF00D389FF00DBF
:108A90001124ED54FA4F07C08091C00085FFFCCF30
:108AA00031969093C60090819923B1F7E7EFF3E0F8
:108AB000949108C08091C00085FFFCCF9093C600C0
:108AC000319694919923B1F78091C00085FFFCCF36
:108AD0008AE08093C6000E94F01D20C00E94469547
:108AE00060936A0570936B0580936C0590936D0598
:108AF0000E94469560938205709383058093840558
:108B000090938505E8CF0E94F67888E50E942D2194
:108B1000882311F00C94243B0C94273BC553DF4F62
:108B20000FB6F894DEBF0FBECDBFCF91DF911F917E
:108B30000F91FF90EF90DF90CF90BF90AF909F90FC
:108B40008F907F906F905F904F903F902F900895FF
:108B50008091800590918105039714F40E949127DC
:108B60008091800590918105892BC1F00E947D2A1A
:108B70008091800590918105019790938105809364
:108B800080058091B1059091B205019664E070E096
:108B90000E94159D9093B2058093B1050E94E286D4
:108BA0000E94122A0C940781DF93CF930F920F92A9
:108BB000CDB7DEB79D9AA5988EE295E040E052ECE5
:108BC00061E070E00E94CA1AE4E5F8E0949108C000
:108BD0008091C00085FFFCCF9093C60031969491A0
:108BE0009923B1F78091C00085FFFCCF8AE0809384
:108BF000C60049E453E0FA01949108C08091C00096
:108C000085FFFCCF9093C600319694919923B1F7DC
:108C100084B7282F80FF15C0ECE4F8E0949108C0D9
:108C20008091C00085FFFCCF9093C600319694914F
:108C30009923B1F78091C00085FFFCCF8AE0809333
:108C4000C60021FF15C0ECE3F8E0949108C08091C4
:108C5000C00085FFFCCF9093C60031969491992374
:108C6000B1F78091C00085FFFCCF8AE08093C600F9
:108C700022FF15C0EBE2F8E0949108C08091C0009B
:108C800085FFFCCF9093C600319694919923B1F75C
:108C90008091C00085FFFCCF8AE08093C60023FF4F
:108CA00015C0EBE1F8E0949108C08091C00085FF09
:108CB000FCCF9093C600319694919923B1F780919F
:108CC000C00085FFFCCF8AE08093C60025FF15C059
:108CD000EBE0F8E0949108C08091C00085FFFCCFE4
:108CE0009093C600319694919923B1F78091C0007A
:108CF00085FFFCCF8AE08093C60014BEE4E0F8E074
:108D0000949108C08091C00085FFFCCF9093C6006D
:108D1000319694919923B1F7EEEFF7E0949108C062
:108D20008091C00085FFFCCF9093C600319694914E
:108D30009923B1F78091C00085FFFCCF8AE0809332
:108D4000C600FA019491E9E4F3E008C08091C00004
:108D500085FFFCCF9093C600319694919923B1F78B
:108D6000EEEEF7E0949108C08091C00085FFFCCF43
:108D70009093C600319694919923B1F7E9EDF7E00D
:108D8000949108C08091C00085FFFCCF9093C600ED
:108D9000319694919923B1F7EDECF7E0949108C0E6
:108DA0008091C00085FFFCCF9093C60031969491CE
:108DB0009923B1F7ECEAF7E0949108C08091C000E4
:108DC00085FFFCCF9093C600319694919923B1F71B
:108DD0008091C00085FFFCCF8AE08093C600E1EA65
:108DE000F7E0949108C08091C00085FFFCCF90937C
:108DF000C600319694919923B1F7E5E9F7E0949193
:108E000008C08091C00085FFFCCF9093C6003196CA
:108E100094919923B1F78091C00085FFFCCF8AE03F
:108E20008093C600FA019491E9E4F3E008C08091D0
:108E3000C00085FFFCCF9093C60031969491992392
:108E4000B1F7E6E8F7E0949108C08091C00085FF93
:108E5000FCCF9093C600319694919923B1F720915D
:108E6000DC0E3091DD0ECE0101962115310519F48D
:108E7000825E9E4002C0821B930B9A838983698124
:108E80007A818EE295E04AE050E00E94111CEFE604
:108E9000F7E0949108C08091C00085FFFCCF9093CB
:108EA000C600319694919923B1F78EE295E060E186
:108EB00075E04AE050E00E94111C8091C00085FFDF
:108EC000FCCF8AE08093C6001092390710923A07CF
:108ED00010923B0710923C070E94BC180E94E98543
:108EE0000E9468520E948B780E94D12380E197E211
:108EF00020E931E0F9013197F1F70197D9F7809135
:108F0000010188608093010186E062E80E94C296B8
:108F100086E062E870E00E9423970F900F90CF9157
:108F2000DF910895FC0180914107843290F48083A1
:108F30008F5F80934107815090E0FC01EE0FFF1F8F
:108F4000E80FF91FEE5BF84F88EB9BE0928381837B
:108F500008958FEF80830895FC0120812432B8F5B5
:108F60008181992787FD909548E850E0481B590B6F
:108F7000440F551F440F551F6417750784F08281F5
:108F8000992787FD909548E552E0481B590B440FFF
:108F9000551F440F551F641775070CF4AB01425061
:108FA0005040CA01AA2797FDA095BA2F880F991F94
:108FB000AA1FBB1F4FB7F89430E0F901EE0FFF1F57
:108FC000E20FF31FEE5BF84F928381834FBF08954A
:108FD000FC0180818F3F19F420E030E016C090E062
:108FE000FC01EE0FFF1FE80FF91FEE5BF84F218128
:108FF000328183E0220F331F8A95E1F7B4E0369582
:109000002795BA95E1F72E5F3F4FC9010895AF92BA
:10901000BF92CF92DF92EF92FF920F931F938C013A
:10902000D7DF00D00F920196AA2797FDA095BA2FFF
:10903000F8016181772767FD709528E830E0261BED
:10904000370B220F331F220F331F442737FD409564
:10905000542F6281772767FD7095E8E5EE2EE2E0F8
:10906000FE2EE61AF70AEE0CFF1CEE0CFF1C002782
:10907000F7FC0095102F64EBA62EB12CC12CD12C3F
:10908000EDB7FEB7A182B282C382D482BC01CD010A
:10909000AA24BB2465010E940F980F900F900F9097
:1090A0000F90CB011F910F91FF90EF90DF90CF9029
:1090B000BF90AF900895AF92BF92CF92DF92EF92A0
:1090C000FF920F931F93CF93DF93EC019B0182E0FC
:1090D000603278070CF048C077FF03C020E030E032
:1090E00005C0653B710514F024EB30E000D00F9211
:1090F000B901882777FD8095982F2981332727FD8F
:109100003095E8E8AE2EB12CA21AB30AAA0CBB1C0B
:10911000AA0CBB1CCC24B7FCC094DC2CEA81FF2732
:10912000E7FDF09528E532E02E1B3F0B220F331FA1
:10913000220F331F442737FD4095542FEDB7FEB75C
:10914000218332834383548320E030E040E050E0C9
:1091500004EBE02EF12C012D112D0E940F989B01A4
:109160000F900F900F900F90CE01B901F5DEDF91B7
:10917000CF911F910F91FF90EF90DF90CF90BF9014
:10918000AF900895EF92FF920F931F93CF93DF93C9
:109190008B017A01EC01DC01A255B84F8C9187FF5D
:1091A00004C0FB011182108237C0AE01440F551F6D
:1091B0004C0F5D1F440F551F440F551F2C91332733
:1091C00027FD3095240F351F8091410790E0281727
:1091D000390714F58C91992787FD9095840F951F79
:1091E000FC01EE0FFF1FE80FF91FEE5BF84F8081C7
:1091F00086FF12C08C91992787FD9095840F951F4B
:10920000FC01EE0FFF1FE80FF91FEE5BF84F8081A6
:109210008F7360E00E94C296DE01A255B84F8C9118
:109220008F5F8C93AE01440F551F4C0F5D1F440F91
:10923000551F440F551F2C91332727FD3095240FC0
:10924000351F8091410790E0281739070CF04DC079
:109250008C918C300CF049C0F801208131818C91C7
:10926000992787FD9095840F951FFC01EE0FFF1F36
:10927000E80FF91FEE5BF84F81819281280F391FAB
:10928000F701318320838C91992787FD9095840F76
:10929000951FFC01EE0FFF1FE80FF91FEE5BF84F63
:1092A000808186FF2AC08C91992787FD9095840F35
:1092B000951FFC01EE0FFF1FE80FF91FEE5BF84F43
:1092C00080818F7361E00E94C29617C080E49CE9A0
:1092D00004C0F801808191810496F7019183808315
:1092E000C255D84F8FEF888308C0F80180819181E3
:1092F000049680549C4950F3ECCFDF91CF911F919D
:109300000F91FF90EF9008951F920F920FB60F925A
:109310000BB60F9211242F933F934F935F936F934C
:109320007F938F939F93AF93BF93EF93FF9380E0CF
:1093300090E064E271E048E251E024DFFF91EF91B8
:10934000BF91AF919F918F917F916F915F914F915D
:109350003F912F910F900BBE0F900FBE0F901F905B
:1093600018951F920F920FB60F920BB60F92112401
:109370002F933F934F935F936F937F938F939F931D
:10938000AF93BF93EF93FF9382E090E064EA70E0C5
:1093900048EA50E0F7DEFF91EF91BF91AF919F91C6
:1093A0008F917F916F915F914F913F912F910F908E
:1093B0000BBE0F900FBE0F901F9018951F920F922B
:1093C0000FB60F920BB60F9211242F933F934F932A
:1093D0005F936F937F938F939F93AF93BF93EF931D
:1093E000FF9381E090E064E970E048E950E0CADE74
:1093F000FF91EF91BF91AF919F918F917F916F916D
:109400005F914F913F912F910F900BBE0F900FBE28
:109410000F901F9018952F923F924F925F926F92EC
:109420007F928F929F92AF92BF92CF92DF92EF92F4
:10943000FF920F931F93DF93CF93CDB7DEB7CD5538
:10944000D0400FB6F894DEBF0FBECDBF2F969FAFB2
:109450008EAF2F9761967FAF6EAF61972A016296AC
:109460002FAF629763960FAF63976496EFAE6497E2
:109470006896ACAEBDAECEAEDFAE6897E22EFF24EE
:10948000EE0CFF1CEE0CFF1C9A012E0D3F1D2D96BD
:109490003FAF2EAF2D97D9016D907D908D909C9010
:1094A000FC01EE0DFF1DC401B30120813181428119
:1094B00053810E94579869AF7AAF8BAF9CAF10E091
:1094C000000F111F000F111FF201E00FF11F2B966B
:1094D000FFAFEEAF2B97A080B180C280D3802F96D4
:1094E000EEADFFAD2F97E00FF11FC601B501208152
:1094F0003181428153810E9457986DAB7EAB8FAB17
:1095000098AF64962FAD6497E22FF0E0EE0FFF1F47
:10951000EE0FFF1F2F96AEADBFAD2F97AE0FBF1F43
:109520002D913D914D915C9129962CAF3DAF4EAF61
:109530005FAF299761964EAD5FAD6197E40FF51F60
:10954000608171818281938129962CAD3DAD4EADB4
:109550005FAD29970E94569869AB7AAB8BAB9CABF9
:109560006196AEADBFAD61971C968D919D910D90AA
:10957000BC91A02D25968CAF9DAFAEAFBFAF259708
:109580002F96AEADBFAD2F971C962D913D914D916D
:109590005C911F9721962CAF3DAF4EAF5FAF2197E7
:1095A000A401930150582DA73EA74FA758ABD60151
:1095B000C501B05889A79AA7ABA7BCA76196AEAD65
:1095C000BFAD6197EA0EFB1EF70160817181828158
:1095D000938129AD3AAD4BAD5CAD0E9456983B01ED
:1095E0004C0161962EAD3FAD6197020F131FD8015C
:1095F0006D917D918D919C912DA93EA94FA958AD5A
:109600000E9456985B016C016DA57EA58FA598A957
:10961000A60195010E94109C7B018C0169A57AA589
:109620008BA59CA5A40193010E94109C9B01AC01F9
:10963000C801B7010E9456981B012C016DA57EA59B
:109640008FA598A9A40193010E94109C7B018C0115
:1096500069A57AA58BA59CA5A60195010E94109CE1
:109660009B01AC01C801B7010E9457989B01AC0156
:10967000C201B1010E94CA985B016C0120E030E098
:1096800040E050E00E943099882354F4C601B501AF
:109690002BED3FE049EC50E40E9457985B016C01D0
:1096A000E8968FADE897882351F0C601B5012BED00
:1096B0003FE049EC50E40E9456985B016C01C60102
:1096C000B501E7962CAD3DAD4EAD5FADE7970E947D
:1096D000109C29A93AA94BA95CA95F770E944B9BD2
:1096E0007B018C012FE632E143E85AE30E94309976
:1096F00087FD0EC2C801B7010E940D9A0E94A4996D
:1097000078A76FA3672B21F4E1E0F0E0F8A7EFA3BF
:109710002FA138A5B90180E090E00E94D0997B018B
:109720008C01C601B501A80197010E9437996BA36E
:109730007CA38DA39EA369A97AA98BA99CA9A80142
:1097400097010E9437996F8F78A389A39AA32596D2
:109750006CAD7DAD8EAD9FAD259721962CAD3DAD09
:109760004EAD5FAD21970E945698A80197010E94C7
:1097700037996B8F7C8F8D8F9E8F6BA17CA18DA174
:109780009EA120E030E040E05FEB0E94109C2BA106
:109790003CA14DA15EA10E94109C20E030E040E879
:1097A0005FE30E9457986F8B788F898F9A8F6496AA
:1097B0003FAD6497E32FF0E0EE0FFF1FEE0FFF1FAA
:1097C0009E012F5F3F4FE20FF31F29968CAD9DAD99
:1097D000AEADBFAD299780839183A283B3832F96CB
:1097E000AEADBFAD2F971C964D915D916D917C9163
:1097F0001F974D875E876F87788B41E050E05A8BCB
:10980000498B662462969FAD6297892F90E0880FFE
:10981000991F880F991FD901A80FB91F6A96BFAF6A
:10982000AEAF6A9763963FAD6397232F30E0220F68
:10983000331F220F331F4C0F5D1F420F531F6C96B7
:109840005FAF4EAF6C976E96FFAFEEAF6E9726C1CF
:1098500058E156150CF446C06DA57EA58FA598A9B4
:109860002BA13CA14DA15EA10E94109C7B018C010B
:1098700069A57AA58BA59CA52F89388D498D5A8D10
:109880000E94109C9B01AC01C801B7010E9457982F
:109890007B018C016DA57EA58FA598A92F89388D98
:1098A000498D5A8D0E94109C5B016C0169A57AA5B7
:1098B0008BA59CA52BA13CA14DA15EA10E94109C53
:1098C0009B01AC01C601B5010E9456986DA77EA709
:1098D0008FA798AB6394C701D80189A79AA7ABA7B4
:1098E000BCA765C0A989BA89BD0180E090E00E944B
:1098F000D0992BA13CA14DA15EA10E94109C7B019F
:109900008C01C8010E9434996B8B7C8B8D8B9E8B54
:10991000B701C8010E94739C3B014C012D96EEAD2E
:10992000FFAD2D97E080F1800281138117FB109528
:1099300017F910952B96AEADBFAD2B972D903D909E
:109940004D905C90C801B7012B893C894D895E8997
:109950000E94109C5B016C01C201B101A401930142
:109960000E94109C9B01AC01C601B5010E94579852
:109970006DA77EA78FA798ABC801B701A40193017B
:109980000E94109C7B018C01C201B1012B893C8992
:109990004D895E890E94109C9B01AC01C801B701F2
:1099A0000E94569869A77AA78BA79CA7662469ADE1
:1099B0007AAD8BAD9CAD2DA53EA54FA558A90E94B3
:1099C00057986A96EEADFFAD6A9760837183828384
:1099D00093836DA97EA98FA998AD29A53AA54BA51A
:1099E0005CA50E9457986C96AEADBFAD6C976D9319
:1099F0007D938D939C9313976E96EEADFFAD6E970E
:109A000060817181828193812F8D38A149A15AA1F2
:109A10000E9457986E96AEADBFAD6E976D937D93D5
:109A20008D939C9313976D857E858F8598892B8D5B
:109A30003C8D4D8D5E8D0E9457986D877E878F87F8
:109A4000988BCE0101960E94E61C0F920F926981BD
:109A50007A818B819C812D813E814F815885E9845B
:109A6000FA840B851C85A8E7B0E0AC0FBD1FEDB7ED
:109A7000FEB7B283A183EDE0CE2ED12CCC0EDD1E3D
:109A800068968CAC9DACAEACBFAC6897DED7E9896C
:109A9000FA893196FA8BE98B0F900F9029893A89D0
:109AA0004FA158A52417350708F4D2CE0F920F9274
:109AB0006196AEADBFAD61976D917D918D919C9199
:109AC000139714962D913D914D915C91179718968F
:109AD000ED90FD900D911C911B971C966196BFAF68
:109AE000AEAF6197FE01E858FF4FADB7BEB7129613
:109AF000FC93EE9311976196CEACDFAC61976896BC
:109B00008CAC9DACAEACBFAC68979FD70F900F905C
:109B1000C35ADF4F0FB6F894DEBF0FBECDBFCF9153
:109B2000DF911F910F91FF90EF90DF90CF90BF904A
:109B3000AF909F908F907F906F905F904F903F90ED
:109B40002F9008953F924F925F926F927F928F92E3
:109B50009F92AF92BF92CF92DF92EF92FF920F93BC
:109B60001F93CF93DF9380912108882309F4F6C0D7
:109B70008090EB039090EC03A090ED03B090EE0387
:109B80006091A70D7091A80D882777FD8095982F7B
:109B90000E94D29920E030E040E050E40E945798C3
:109BA000A50194010E94309987FDD8C03090330DF3
:109BB0000F2EF0E04F2EF0E05F2EF0E06F2EF0E081
:109BC0007F2EF02DC1E5D0E058C0232D30E02C9F32
:109BD000F0012D9FF00D3C9FF00D1124EE5DF74F2D
:109BE00080819181A281B3810097A105B10581F4A3
:109BF00084819581A681B7810097A105B10541F4C3
:109C000080859185A285B3850097A105B10591F165
:109C10002C9F60012D9FD00C3C9FD00C112482E220
:109C200098E0C80ED91EF6016485758586859785EE
:109C30000E94D2997B018C01F60160897189828929
:109C400093890E94D0999B01AC01C801B7010E9481
:109C50003799F60122A133A144A155A10E94109C7D
:109C60007B018C01A30192010E943E9B181614F403
:109C7000270138013394FFE03F228091320D3816DE
:109C800009F0A3CFC301B2012091EF033091F0039B
:109C90004091F1035091F2030E94109C9B01AC0192
:109CA000C501B4010E9457987B018C01A501940164
:109CB0000E94309987FD02C0470158011091E703C7
:109CC0000091E803F090E903E090EA03C501B401D4
:109CD000212F302F4F2D5E2D0E943E9B181634F4FD
:109CE000812F902FAF2DBE2D4C015D0140904C0D6A
:109CF00050904D0D60904E0D70904F0DC301B2010C
:109D0000A50194010E943E9B1816C4F4C501B4013C
:109D100020E037ED43EA5CE30E94109C7B018C015C
:109D2000C301B20128E431EE4AE75FE30E94109CD0
:109D3000A80197010E9457984B015C0180924C0D3D
:109D400090924D0DA0924E0DB0924F0DC501B401F1
:109D50000E949F997093A80D6093A70DDF91CF91FA
:109D60001F910F91FF90EF90DF90CF90BF90AF9039
:109D70009F908F907F906F905F904F903F9008954D
:109D80006093F3037093F4038093F5039093F603C9
:109D900008950F931F93CF93DF93C0E0D0E08E011F
:109DA0000F5F174FFE01EB52F84F60817181828186
:109DB00093810E94D099FE01EB53F84F20813181AD
:109DC000428153810E94109C0E94A499F8016083F3
:109DD0007183828393832496C031D10501F7DF918B
:109DE000CF911F910F910895FC0160817181828153
:109DF00093812091D1073091D2074091D3075091A0
:109E0000D4070E94109C0E94E09B60931D087093F1
:109E10001E0880931F08909320088DE198E00C9411
:109E20007076AF92BF92CF92DF92EF92FF920F9334
:109E30001F93DF93CF93CDB7DEB72C970FB6F8946F
:109E4000DEBF0FBECDBF69837A838B839C832D8356
:109E50003E834F835887E986FA860B871C87560115
:109E60008DB79EB78A970FB6F8949EBF0FBE8DBF71
:109E7000EDB7FEB731969F0143EC53E084E2DA017F
:109E80000D90AD01D9010D929D018150C1F7CE0118
:109E9000019695A384A3CE01059697A386A3CE0130
:109EA000099691A780A70E94288FEDB7FEB7BA96B2
:109EB0000FB6F894FEBF0FBEEDBF69817A818B812A
:109EC0009C812091C5073091C6074091C7075091EA
:109ED000C8070E94109C0E94E09B31E1C32E38E02D
:109EE000D32E6093110870931208809313089093F7
:109EF00014086D817E818F8198852091C9073091EA
:109F0000CA074091CB075091CC070E94109C0E9439
:109F1000E09B24E0E22EF12CEC0CFD1C6093150874
:109F2000D70111967C93119712968C9312971396E2
:109F30009C9369857A858B859C852091CD0730918E
:109F4000CE074091CF075091D0070E94109C0E94ED
:109F5000E09B8601085F1F4F60931908F801718329
:109F600082839383D5016D917D918D919C912091F8
:109F7000D1073091D2074091D3075091D4070E9466
:109F8000109C0E94E09BF6013C9660931D08718333
:109F900082839383C601B701A8019F010E94367690
:109FA00080E090E0A0E0B0E08093340D9093350D18
:109FB000A093360DB093370D8093380D9093390DE3
:109FC000A0933A0DB0933B0D80933C0D90933D0DC3
:109FD000A0933E0DB0933F0D8093400D9093410DA3
:109FE000A093420DB093430D8093440D9093450D83
:109FF000A093460DB093470D2C960FB6F894DEBF94
:10A000000FBECDBFCF91DF911F910F91FF90EF90C9
:10A01000DF90CF90BF90AF9008952F923F924F92D4
:10A020005F926F927F928F929F92AF92BF92CF92E8
:10A03000DF92EF92FF920F931F93DF93CF93CDB7F1
:10A04000DEB7A4970FB6F894DEBF0FBECDBF1C01DC
:10A0500080E00E9493762B013C0181E00E94937680
:10A060004B015C0182E00E9493766B017C01C1018F
:10A07000B301A201950184010E94218E8DB79EB784
:10A0800084970FB6F8949EBF0FBE8DBFADB7BEB715
:10A090001196E3ECF3E084E201900D928150E1F738
:10A0A0008E010F5F1F4FC8010E94CA8F8DB79EB7E8
:10A0B00084960FB6F8949EBF0FBE8DBF84970FB6DF
:10A0C000F8949EBF0FBE8DBFADB7BEB71196F80115
:10A0D00084E201900D928150E1F7C1010E943B8E14
:10A0E0008DB79EB784960FB6F8949EBF0FBE8DBFF6
:10A0F000C101A4960FB6F894DEBF0FBECDBFCF91BD
:10A10000DF911F910F91FF90EF90DF90CF90BF9064
:10A11000AF909F908F907F906F905F904F903F9007
:10A120002F9008958F929F92AF92BF92CF92DF921D
:10A13000EF92FF920F931F93CF93DF93EC016B018C
:10A14000009709F45CC08FA9882309F058C0EEA0DD
:10A15000FFA008A519A5FB01B6A0A7A090A481A403
:10A16000C801B7012B2D3A2D492D582D0E94309949
:10A1700088230CF044C0C801B701A80197010E94D0
:10A18000109C7B018C016AA97BA98CA99DA9905880
:10A1900020E030E040E050EC0E94109C2EA53FA54E
:10A1A00048A959A90E94109C9B01AC01C801B701A4
:10A1B0000E9457980E947D9C7B018C016B2D7A2D0B
:10A1C000892D982D9701A8010E943099882324F4A5
:10A1D000EB2CFA2C092D182D6B2D7A2D892D982D0D
:10A1E0009701A8010E943099882349F0C701D8013E
:10A1F000F60186A397A3A0A7B1A781E086ABDF9164
:10A20000CF911F910F91FF90EF90DF90CF90BF9073
:10A21000AF909F908F900895EF92FF920F931F93AE
:10A22000CF93DF93F090330D00E010E020E030E0BA
:10A2300041E5E42E11C0FE9CE0011124CE5DD74F14
:10A24000C901B801AE016EDF8F2D8F5F803109F437
:10A2500080E0F82E98018E018091320DF81659F7A2
:10A26000C901B80140E050E05DDFDF91CF911F915F
:10A270000F91FF90EF900895AF92BF92CF92DF922F
:10A28000EF92FF920F931F93CF93DF93EB018A011D
:10A290006115710509F466C04115510509F462C0E4
:10A2A000DAA4CBA4BCA4ADA46EA17FA188A599A576
:10A2B0002D2D3C2D4B2D5A2D0E943099882309F4C9
:10A2C00051C08FA9882309F043C0F801E6A0F7A088
:10A2D00000A511A56D2D7C2D8B2D9A2DA801970120
:10A2E0000E943E9B1816A4F5C801B701A80197016A
:10A2F0000E94109C7B018C016AA97BA98CA99DA955
:10A30000905820E030E040E050EC0E94109C2EA5D8
:10A310003FA548A959A90E94109C9B01AC01C80106
:10A32000B7010E9457980E947D9C7B018C016D2D86
:10A330007C2D8B2D9A2D9701A8010E94309988239E
:10A3400024F4ED2CFC2C0B2D1A2DC701D80104C0D0
:10A350008D2D9C2DAB2DBA2D8EA39FA3A8A7B9A799
:10A3600081E08EABDF91CF911F910F91FF90EF9025
:10A37000DF90CF90BF90AF900895CF92DF92EF9291
:10A38000FF920F93DF93CF930F920F92CDB7DEB76B
:10A390008091320D8FB7F894F090330D8FBF80917C
:10A3A000320D90E040968F1991098F70907004974C
:10A3B000FCF00091320D03500F70CC24DD2440E0FE
:10A3C00050E061E5E62E12C0802F002309F480E101
:10A3D000082F01500E9DC00111248E5D974F9A8366
:10A3E0008983B60149DFA601C980DA800F1561F7BC
:10A3F0000F900F90CF91DF910F91FF90EF90DF9032
:10A40000CF900895DF92EF92FF920F931F93609188
:10A4100066059091330D8091320D9817B9F04091F7
:10A42000330D242F30E081E590E0289FF001299F33
:10A43000F00D389FF00D1124E659F74F608102C0EE
:10A440004F5F4F708091320D4817D1F7D62E66239B
:10A4500031F1E090480DF090490D00914A0D1091B6
:10A460004B0DE114F1040105110579F40E944695A4
:10A470006C597F4F8F4F9F4F6093480D7093490DDC
:10A4800080934A0D90934B0D07C00E9446956E1520
:10A490007F058007910758F4DD24DA9408C01092F4
:10A4A000480D1092490D10924A0D10924B0D88E004
:10A4B0006D2D70E00E94239788E06D2D70E00E9462
:10A4C000239740DB1F910F91FF90EF90DF9008954D
:10A4D0001092320D1092330D80E1E1E1F8E0DF01DE
:10A4E0001D928A95E9F780E090E0A0E0B0E08093CB
:10A4F000380D9093390DA0933A0DB0933B0D809396
:10A500003C0D90933D0DA0933E0DB0933F0D809375
:10A51000400D9093410DA093420DB093430D809355
:10A52000440D9093450DA093460DB093470D809335
:10A53000340D9093350DA093360DB093370D0895DB
:10A540002F923F924F925F926F927F928F929F9243
:10A55000AF92BF92CF92DF92EF92FF920F931F9331
:10A56000DF93CF93CDB7DEB766970FB6F894DEBF13
:10A570000FBECDBF9E8B8D8B6A017B0148015901B7
:10A58000DC01D8966D917D918D919C91DB970E9415
:10A59000D099698B7A8B8B8B9C8BA70196010E943B
:10A5A000109C0E941D990E94A4996D837E838F83C5
:10A5B000988769897A898B899C89A50194010E9471
:10A5C000109C0E941D990E94A49969837A838B83B1
:10A5D0009C832D813E814F81588528373105410567
:10A5E000510540F448E750E060E070E04D835E8341
:10A5F0006F83788769817A818B819C816837710547
:10A600008105910540F488E790E0A0E0B0E08983FF
:10A610009A83AB83BC83AD89BE89AC5BBF4FAD90E1
:10A62000BD90CD90DC901397A454B040BE8BAD8B01
:10A630006D817E818F8198850E94D0996D877E87FC
:10A640008F87988BC601B5010E94D2991B012C01FE
:10A6500020E030E040E050E00E943099882321F46F
:10A66000E0E070E060E028C069897A898B899C8984
:10A670009B01AC010E94109C7B018C016D857E8545
:10A680008F8598899B01AC010E94109C9B01AC01B5
:10A69000C801B7010E9456987B018C01C201B1012B
:10A6A000A20191010E9457989B01AC01C801B7011A
:10A6B0000E943799E62F692F2E2F372F482F562FBC
:10A6C000B901CA010E941D990E949F993B014C014A
:10A6D00069817A818B819C810E94D09969877A8770
:10A6E0008B879C8766277727CB016A197B098C09A2
:10A6F0009D090E94D2995B016C0120E030E040E0AE
:10A7000050E00E943099882321F4E0E070E060E09E
:10A7100028C069857A858B859C859B01AC010E9448
:10A72000109C7B018C0169897A898B899C899B01AA
:10A73000AC010E94109C9B01AC01C801B7010E94B2
:10A7400056987B018C01C601B501A60195010E94B6
:10A7500057989B01AC01C801B7010E943799E62FB9
:10A76000692F2E2F372F482F562FB901CA010E946B
:10A770000D9AED89FE89A088B188C288D3888601A8
:10A780007501E618F708080919090E949F99A801A0
:10A790009701261B370B480B590B57FF71C0C2019D
:10A7A000B10120E030E040E050E00E943099882381
:10A7B00021F4E0E070E060E044C0C201B101A20118
:10A7C00091010E9457987B018C01C601B5010E943E
:10A7D000D0999B01AC01C801B7010E94109C7B017C
:10A7E0008C016D857E858F8598899B01AC010E94C7
:10A7F000109C9B01AC01C801B7010E9456987B01D7
:10A800008C0169857A858B859C859B01AC010E94B2
:10A81000109C9B01AC01C801B7010E9457987B01B5
:10A820008C01C201B10120E030E040E850E40E9418
:10A83000109C9B01AC01C801B7010E943799E62F1B
:10A84000692F2E2F372F482F562FB901CA010E948A
:10A850001D990E949F99AC01CB01DA013C014D0189
:10A8600097FE03C06624772443016A147B048C049A
:10A870009D0410F03501460120E030E040E050E05A
:10A880009FB7F8946D897E89605B7F4FDB018C9167
:10A89000A055B040BE8BAD8B882321F5FD01648AA5
:10A8A000758A868A978A260D371D481D591D589628
:10A8B0002D933D934D935C935B972D813E814F810A
:10A8C0005885DC962D933D934D935C93DF97A05C68
:10A8D000BF4F29813A814B815C812D933D934D93EC
:10A8E0005C9313979FBF66960FB6F894DEBF0FBEBA
:10A8F000CDBFCF91DF911F910F91FF90EF90DF902F
:10A90000CF90BF90AF909F908F907F906F905F900F
:10A910004F903F902F9008954F925F927F928F9229
:10A920009F92AF92BF92CF92DF92EF92FF920F93DE
:10A930001F93CF93DF937090330DC0E0D0E071E5AB
:10A94000472E512C45C02097A9F18EA9882361F488
:10A95000849CF001859CF00D949CF00D1124EE5D1B
:10A96000F74F86A9882331F1EAA0FBA00CA11DA115
:10A970006EA17FA188A599A5A80197010E9437998A
:10A980005B016C01849CF001859CF00D949CF00DA2
:10A990001124EE5DF74F66A177A180A591A5A801CE
:10A9A00097010E9437998B019C01CE01B601A50148
:10A9B000C7DD1EAA739480E1781609F47724849C7D
:10A9C000E001859CD00D949CD00D1124CE5DD74F15
:10A9D000872C992487FC90948091320D90E0881602
:10A9E000990609F0B0CF2097E9F0EAA0FBA00CA1EE
:10A9F0001DA16EA17FA188A599A5A80197010E941C
:10AA000037995B016C016DEC7CEC8CE49DE3A80153
:10AA100097010E9437998B019C01CE01B601A501D7
:10AA20008FDD1EAADF91CF911F910F91FF90EF90C4
:10AA3000DF90CF90BF90AF909F908F907F905F906E
:10AA40004F9008959ADCE8DB67CF2F923F924F92A8
:10AA50005F926F927F928F929F92AF92BF92CF92AE
:10AA6000DF92EF92FF920F931F93DF93CF93CDB7B7
:10AA7000DEB7CA5AD0400FB6F894DEBF0FBECDBFC6
:10AA800069A37AA38BA39CA32DA33EA34FA358A78E
:10AA9000E9A6FAA60BA71CA78601C955DF4F888235
:10AAA000C75AD040C855DF4F9882C85AD040C755C2
:10AAB000DF4FA882C95AD040C655DF4FB882CA5A64
:10AAC000D0408091320D8F5F803109F480E0282FD3
:10AAD000332727FD30953CAF2BAF04C00E94E286A0
:10AAE0000E94122A8091330D90E04BAD5CAD84172B
:10AAF0009507A1F36DB77EB76A5270400FB6F89410
:10AB00007EBF0FBE6DBFEDB7FEB731969F0143EC20
:10AB100053E084E2DA010D90AD01D9010D929D015F
:10AB20008150C1F7CE01819695A384A3CE0185966D
:10AB300097A386A3CE01899691A780A70E94288F0C
:10AB40002091C5073091C6074091C7075091C807AB
:10AB5000CF57DF4F288339834A835B83C158D04066
:10AB60004DB75EB7465D5F4F0FB6F8945EBF0FBE40
:10AB70004DBFCF57DF4F688179818A819B81C15852
:10AB8000D04029A13AA14BA15CA10E94109C0E9437
:10AB9000E09BCF56DF4F6883C159D040CE56DF4F80
:10ABA0007883C259D040CD56DF4F8883C359D040F7
:10ABB000CC56DF4F9883C459D0406091C90770913B
:10ABC000CA078091CB079091CC07C358DF4F6883A9
:10ABD00079838A839B83CD57D0402DA13EA14FA17D
:10ABE00058A50E94109C0E94E09BCB56DF4F6883C3
:10ABF000C559D040CA56DF4F7883C659D040C95690
:10AC0000DF4F8883C759D040C856DF4F9883C85953
:10AC1000D0408091CD079091CE07A091CF07B09101
:10AC2000D007ED968CAF9DAFAEAFBFAFED97BC0137
:10AC3000CD0129A53AA54BA55CA50E94109C0E94B8
:10AC4000E09BC756DF4F6883C959D040C656DF4FD7
:10AC50007883CA59D040C556DF4F8883CB59D0403E
:10AC6000C456DF4F9883CC59D0402091D107309102
:10AC7000D2074091D3075091D407E9962CAF3DAF4E
:10AC80004EAF5FAFE997CA01B901D8012D913D914F
:10AC90004D915C910E94109C0E94E09BC356DF4F37
:10ACA0006883CD59D040C256DF4F7883CE59D0400B
:10ACB000C156DF4F8883CF59D040C056DF4F9883AD
:10ACC000C05AD04080911D0890911E08A0911F0885
:10ACD000B0912008C356DF4F288139814A815B81BA
:10ACE000CD59D040281739074A075B0709F4B8C087
:10ACF000E0916405F0E0EE0FFF1FEE0FFF1FE3553C
:10AD0000F24F60817181828193812091F3033091B0
:10AD1000F4034091F5035091F6030E943099882383
:10AD20000CF033C0C356DF4F488159816A817B8163
:10AD3000CD59D04040931D0850931E0860931F08C2
:10AD400070932008E4E7F8E0949108C08091C00077
:10AD500085FFFCCF9093C600319694919923B1F76B
:10AD6000E8E9F8E0949108C08091C00085FFFCCF2D
:10AD70009093C600319694919923B1F78091C000C9
:10AD800085FFFCCF8AE08093C60080911D089091DA
:10AD90001E08A0911F08B0912008C356DF4F2881DC
:10ADA00039814A815B81CD59D040281B390B4A0B30
:10ADB0005B0BCA01B90157FF07C09095809570954C
:10ADC00061957F4F8F4F9F4F0E94D2997B018C01DD
:10ADD000E9966CAD7DAD8EAD9FADE99720E030E09A
:10ADE0004FEA53E40E94109C9B01AC01C801B701DB
:10ADF0000E943E9B18160CF033C0C356DF4F4881AB
:10AE000059816A817B81CD59D04040931D08509370
:10AE10001E0860931F0870932008E4E7F8E09491FF
:10AE200008C08091C00085FFFCCF9093C60031968A
:10AE300094919923B1F7EAE7F8E0949108C08091E2
:10AE4000C00085FFFCCF9093C60031969491992362
:10AE5000B1F78091C00085FFFCCF8AE08093C600E7
:10AE60008091320D682F70E0E5967FAF6EAFE59769
:10AE700081E590E0689FF001699FF00D789FF00DEB
:10AE80001124EE5DF74FE05BFF4F1082E055F0407C
:10AE90008091110890911208A0911308B0911408A4
:10AEA000E3968CAF9DAFAEAFBFAFE397CF56DF4F0A
:10AEB000288139814A815B81C159D040281B390BD7
:10AEC0004A0B5B0BAF962CAF3DAF4EAF5FAFAF976A
:10AED000208331834283538357FF0DC0DA01C901B8
:10AEE000B095A095909581959F4FAF4FBF4F8083B0
:10AEF0009183A283B3834091150850911608609105
:10AF0000170870911808AB964CAF5DAF6EAF7FAF6E
:10AF1000AB97CB56DF4F88819981AA81BB81C559F8
:10AF2000D040841B950BA60BB70BA7968CAF9DAF9B
:10AF3000AEAFBFAFA79781E590E0E596AEADBFADF0
:10AF4000E597A89FF001A99FF00DB89FF00D11247F
:10AF5000EE5DF74FA7962CAD3DAD4EAD5FADA7971B
:10AF6000248335834683578357FF0DC0DA01C90117
:10AF7000B095A095909581959F4FAF4FBF4F84831B
:10AF80009583A683B7834091190850911A08609160
:10AF90001B0870911C08A3964CAF5DAF6EAF7FAFDE
:10AFA000A397C756DF4F88819981AA81BB81C95970
:10AFB000D040841B950BA60BB70B6F968CAF9DAF43
:10AFC000AEAFBFAF6F9781E590E0E596AEADBFAD98
:10AFD000E597A89FF001A99FF00DB89FF00D1124EF
:10AFE000EE5DF74F6F962CAD3DAD4EAD5FAD6F97FB
:10AFF000208731874287538757FF0DC0DA01C90187
:10B00000B095A095909581959F4FAF4FBF4F80878A
:10B010009187A287B38740911D0850911E086091C7
:10B020001F08709120084DAB5EAB6FAB78AFC35675
:10B03000DF4F88819981AA81BB81CD59D040841B83
:10B04000950BA60BB70B89AB9AABABABBCABE09146
:10B050006405F0E0EE0FFF1FEE0FFF1FE956FC4FF7
:10B0600020813181428153816B962CAF3DAF4EAF31
:10B070005FAF6B97409193035091940367965FAFD6
:10B080004EAF6797BC01CD0197FF07C090958095A3
:10B09000709561957F4F8F4F9F4F0E94D2996B960D
:10B0A0002CAD3DAD4EAD5FAD6B970E94109C0E94E4
:10B0B0009F996796AEADBFAD67979D01442737FD59
:10B0C0004095542F0E94E29C24E630E040E050E09E
:10B0D0000E944A9D81E590E0E5966EAD7FADE597D3
:10B0E000689FF001699FF00D789FF00D1124EE5DCF
:10B0F000F74FDF011C96248711963C931197129607
:10B100004C93129713965C934080518062807380B9
:10B11000A480B580C680D780E084F1840285138541
:10B12000C901DA018E159F05A007B10714F4D801F3
:10B13000C7018A159B05AC05BD0514F4D601C501F0
:10B140009C01AD0184159505A605B70514F4A3016E
:10B15000920181E590E0E596AEADBFADE597A89F81
:10B16000B001A99F700DB89F700D11246E5D774FCF
:10B17000FB01208B318B428B538B263031054105EF
:10B18000510510F40C941A62E85BFF4F809166053C
:10B1900090916705AA2797FDA095BA2F8083918388
:10B1A000A283B383FB01E45BFF4F8091680590911C
:10B1B0006905AA2797FDA095BA2F80839183A28362
:10B1C000B383DB0190961C92CF56DF4F28813981E3
:10B1D0004A815B81C159D040E3968CAD9DADAEAD47
:10B1E000BFADE397281739074A075B0724F481E0CE
:10B1F000DB0190968C93CB56DF4F288139814A81B1
:10B200005B81C559D040AB966CAD7DAD8EAD9FAD29
:10B21000AB97261737074807590794F481E590E064
:10B22000E596AEADBFADE597A89FF001A99FF00DE3
:10B23000B89FF00D1124EE5DF74F80A1826080A3CE
:10B24000C756DF4F288139814A815B81C959D04077
:10B25000A3966CAD7DAD8EAD9FADA3972617370736
:10B260004807590794F481E590E0E596AEADBFAD8F
:10B27000E597A89FF001A99FF00DB89FF00D11244C
:10B28000EE5DF74F80A1846080A3C356DF4F288115
:10B2900039814A815B81CD59D0406DA97EA98FA9A2
:10B2A00098AD261737074807590794F481E590E0D1
:10B2B000E596AEADBFADE597A89FF001A99FF00D53
:10B2C000B89FF00D1124EE5DF74F80A1886080A338
:10B2D00081E590E0E5962EAD3FADE597289FF00122
:10B2E000299FF00D389FF00D1124EE5DF74FC054EB
:10B2F000DF4FA881B981C05CD0408C9181A340818F
:10B3000051816281738165964CAF5DAF6EAF7FAF47
:10B310006597411551056105710509F0179881E59B
:10B3200090E0E5966EAD7FADE597689FF001699F6F
:10B33000F00D789FF00D1124EE5DF74F648075805D
:10B3400086809780611471048104910409F0169835
:10B3500081E590E0E596AEADBFADE597A89FF00121
:10B36000A99FF00DB89FF00D1124EE5DF74FA0845A
:10B37000B184C284D384A114B104C104D10409F0FE
:10B38000159881E590E0E5962EAD3FADE597289FB5
:10B39000F001299FF00D389FF00D1124EE5DF74F5D
:10B3A00084859585A685B7850097A105B10551F0DF
:10B3B00014982090E5073090E6074090E7075090FA
:10B3C000E80708C02090FD073090FE074090FF0777
:10B3D00050900008C955DF4F6881C75AD040C85502
:10B3E000DF4F7881C85AD040C755DF4F8881C95A8E
:10B3F000D040C655DF4F9881CA5AD040A201910172
:10B400000E94309987FD16C0C955DF4F8881C75A01
:10B41000D040C855DF4F9881C85AD040C755DF4F3C
:10B42000A881C95AD040C655DF4FB881CA5AD0400A
:10B430001C012D01AF966CAD7DAD8EAD9FADAF976C
:10B440000E94D299CF57DF4F288139814A815B8191
:10B45000C158D0400E943799C357DF4F6883CD58F9
:10B46000D040C257DF4F7883CE58D040C157DF4F0E
:10B470008883CF58D040C057DF4F9883C059D04001
:10B48000AC01CB01DA0189839A83AB83BC83A79695
:10B490006CAD7DAD8EAD9FADA7970E94D299C3587C
:10B4A000DF4F288139814A815B81CD57D0400E948E
:10B4B0003799C757DF4F6883C958D040C657DF4F09
:10B4C0007883CA58D040C557DF4F8883CB58D040C7
:10B4D000C457DF4F9883CC58D040AC01CB01DA0180
:10B4E0008D839E83AF83B8876F966CAD7DAD8EAD37
:10B4F0009FAD6F970E94D299ED962CAD3DAD4EADAC
:10B500005FADED970E943799CB57DF4F6883C558E1
:10B51000D040CA57DF4F7883C658D040C957DF4F55
:10B520008883C758D040C857DF4F9883C858D04049
:10B53000AC01CB01DA0189879A87AB87BC8769A9FF
:10B540007AA98BA99CA90E94D299E9962CAD3DAD10
:10B550004EAD5FADE9970E9437996B962CAD3DAD2E
:10B560004EAD5FAD6B970E94109C7B018C0167967E
:10B570004EAD5FAD6797BA01882777FD8095982F0C
:10B580000E94D2999B01AC01C801B7010E94109C96
:10B5900020E030E048EC52E40E9437999B01AC0176
:10B5A0006D877E878F87988B65966CAD7DAD8EADF0
:10B5B0009FAD659766307105810591051CF576E0B4
:10B5C0006716710481049104ECF486E0A816B104B6
:10B5D000C104D104BCF481E590E0E596AEADBFAD09
:10B5E000E597A89FF001A99FF00DB89FF00D1124D9
:10B5F000EE5DF74FDA01C901BF7786A797A7A0AB29
:10B60000B1AB6DC0C357DF4F2881CD58D040C25772
:10B61000DF4F3881CE58D040C157DF4F4881CF58D7
:10B62000D040C057DF4F5881C059D040B901CA013E
:10B630000E94C79C3B014C01C757DF4F2881C95866
:10B64000D040C657DF4F3881CA58D040C557DF4F6A
:10B650004881CB58D040C457DF4F5881CC58D04098
:10B66000B901CA010E94C79C5B016C01CB57DF4F37
:10B670002881C558D040CA57DF4F3881C658D040BE
:10B68000C957DF4F4881C758D040C857DF4F58814E
:10B69000C858D040B901CA010E94C79C7B018C01E7
:10B6A000C401B301A60195010E945798A801970112
:10B6B0000E9457980E947D9C21E530E0E5964EADB2
:10B6C0005FADE597429FF001439FF00D529FF00D53
:10B6D0001124EE5DF74F66A777A780AB91AB81E5AC
:10B6E00090E0E5966EAD7FADE597689FF001699FAC
:10B6F000F00D789FF00D1124EE5DF74F86A597A50C
:10B70000A0A9B1A961968CAF9DAFAEAFBFAF619755
:10B7100060E070E080E89FE361962CAD3DAD4EADFA
:10B720005FAD61970E9437999B01AC01C201B101E5
:10B730000E94109C2B013C018091320D9091330DA1
:10B74000A82FB0E05096A91BB109AF70B070BAAF86
:10B75000A9AFA230B1050CF451C05D01CC24B7FCF7
:10B76000C094DC2CC601B5010E94D29920E030E0E3
:10B7700040E051E40E94309988230CF03FC060E023
:10B7800074E284E799E4A30192010E9437990E9430
:10B79000E09B7B018C016091B1077091B2078091B1
:10B7A000B3079091B407E616F7060807190730F5B6
:10B7B0006E197F09800B910B660F771F881F991FE9
:10B7C000A60195010E94289DCA01B9010E94D09945
:10B7D0000E94E09B9B01AC012E0D3F1D401F511F9D
:10B7E000CA01B9010E94D0999B01AC0160E074E2EA
:10B7F00084E799E40E9437992B013C0181E590E0B0
:10B80000E596EEADFFADE597E89F8001E99F100D4D
:10B81000F89F100D11240E5D174F61966CAD7DAD34
:10B820008EAD9FAD6197A30192010E94109CD8013B
:10B8300092966D937D938D939C93959750966D9171
:10B840007D918D919C9153970E94D099A301920173
:10B850000E94109C0E941D990E94A499F80160AF5B
:10B8600071AF82AF93AFCF55DF4F1882C15AD0402E
:10B87000CE55DF4F1882C25AD04020E8222E9FE3D7
:10B88000392E88249924E1E0F0E0EC0FFD1FE80D4B
:10B89000F91DC301B20120813181428153810E948F
:10B8A000109CE1E1F0E0EC0FFD1FE80DF91D608355
:10B8B0007183828393835B016C01E894D7F8F40170
:10B8C000EB54F84FE080F18002811381C601B5018D
:10B8D000A80197010E943E9B1816CCF4C801B7013D
:10B8E000A60195010E9437996B017C01CF55DF4F6E
:10B8F0006881C15AD040CE55DF4F7881C25AD040BE
:10B90000C101A70196010E94309988236CF4CF559C
:10B91000DF4F8881C15AD040CE55DF4F9881C25A3F
:10B92000D040D1016C017D0124E030E0820E931EF5
:10B9300030E18316910471F0D701C601CF55DF4F76
:10B94000C882C15AD040CE55DF4F9883C25AD040EA
:10B950001D0199CFC701B60120E030E040E85FE368
:10B960000E94309988230CF04CC08E010F5E1F4F4F
:10B9700081E2A82EB12CAC0EBD1ED8016D917D9137
:10B980008D919C91A70196010E94109CF8016193F2
:10B990007193819391938F01EA15FB0571F781E50E
:10B9A00090E0E5962EAD3FADE597289F8001299F59
:10B9B000100D389F100D11240E5D174FD80192966F
:10B9C0006D917D918D919C919597A70196010E9413
:10B9D000109CF80162A373A384A395A360AD71AD1D
:10B9E00082AD93AD0E94D099A70196010E94109C50
:10B9F0000E94A499D801D8966D937D938D939C93C2
:10BA0000DB9781E590E0E596EEADFFADE597E89F29
:10BA10008001E99F100DF89F100D11240E5D174F46
:10BA2000D80150966D917D918D919C9153970E9474
:10BA3000D099F80126A537A540A951A90E943799A8
:10BA40001B012C01F80180819181A281B3810097B3
:10BA5000A105B10549F584819581A681B78100973B
:10BA6000A105B10509F580859185A285B38500976B
:10BA7000A105B105C9F4C201B1012091ED073091D2
:10BA8000EE074091EF075091F0070E94109C0E9432
:10BA90001D990C5B1F4F0E94A499D8016D937D9353
:10BAA0008D939C93139771C1C201B1012091E90755
:10BAB0003091EA074091EB075091EC070E94109CEF
:10BAC0000E941D990E94A49921E530E0E596EEAD13
:10BAD000FFADE597E29F6001E39FD00CF29FD00C91
:10BAE000112422E238E0C20ED31EB4E46B2E712C76
:10BAF0006C0C7D1CD3016D937D938D939C93139758
:10BB00008090010890900208A0900308B09004086B
:10BB10000E94D0997B018C01F60160817181828144
:10BB200093810E94D2999B01AC01C801B7010E9488
:10BB3000109C7B018C01D60150966D917D918D9169
:10BB40009C9153970E94D0999B01AC01C801B70109
:10BB50000E9437997B018C01C501B4010E94D099E4
:10BB60009B01AC01C801B7010E943E9B18162CF442
:10BB7000F30180829182A282B38280900508909026
:10BB80000608A0900708B090080881E590E0E596C7
:10BB90002EAD3FADE597289F6001299FD00C389FBF
:10BBA000D00C112442E258E0C40ED51EA4E46A2E43
:10BBB000712C6C0C7D1CD3016D917D918D919C91AC
:10BBC0000E94D0997B018C01F60164817581868188
:10BBD00097810E94D2999B01AC01C801B7010E94D4
:10BBE000109C7B018C01D60150966D917D918D91B9
:10BBF0009C9153970E94D0999B01AC01C801B70159
:10BC00000E9437997B018C01C501B4010E94D09933
:10BC10009B01AC01C801B7010E943E9B18162CF491
:10BC2000F30180829182A282B38280900D0890906D
:10BC30000E08A0900F08B090100881E590E0E596FE
:10BC40002EAD3FADE597289F6001299FD00C389F0E
:10BC5000D00C112442E258E0C40ED51EF4E46F2E3D
:10BC6000712C6C0C7D1CD3016D917D918D919C91FB
:10BC70000E94D0997B018C01F601648575858685CB
:10BC800097850E94D2999B01AC01C801B7010E941F
:10BC9000109C7B018C01D60150966D917D918D9108
:10BCA0009C9153970E94D0999B01AC01C801B701A8
:10BCB0000E9437997B018C01C501B4010E94D09983
:10BCC0009B01AC01C801B7010E943E9B18162CF4E1
:10BCD000F30180829182A282B382809009089090C1
:10BCE0000A08A0900B08B0900C0881E590E0E5965A
:10BCF0002EAD3FADE597289F6001299FD00C389F5E
:10BD0000D00C112442E258E0C40ED51EE4E46E2E9D
:10BD1000712C6C0C7D1CD3016D917D918D919C914A
:10BD20000E94D0997B018C01F60160857185828526
:10BD300093850E94D2999B01AC01C801B7010E9472
:10BD4000109C7B018C01D60150966D917D918D9157
:10BD50009C9153970E94D0999B01AC01C801B701F7
:10BD60000E9437997B018C01C501B4010E94D099D2
:10BD70009B01AC01C801B7010E943E9B18162CF430
:10BD8000F30180829182A282B38281E590E0E59600
:10BD90002EAD3FADE597289F6001299FD00C389FBD
:10BDA000D00C112442E258E0C40ED51EF601EC5B23
:10BDB000FF4F60817181828193810E94D0997B01C4
:10BDC0008C01A20191010E943799D601D2966D9300
:10BDD0007D938D939C93D597C801B7012DEB37E3E5
:10BDE00046E051E40E94109C0E949F99F601648FE6
:10BDF000758F868F978F6090F1077090F207809013
:10BE0000F3079090F407C401B30120E030E040E074
:10BE10005FE30E94109C5B016C01298D3A8D4B8D74
:10BE20005C8D2D962CAF3DAF4EAF5FAF2D974091FF
:10BE3000F5075091F6076091F7077091F80729967A
:10BE40004CAF5DAF6EAF7FAF2997CB01BA0120E059
:10BE500030E040E05FE30E94109C7B018C012D9656
:10BE60006CAD7DAD8EAD9FAD2D979F77A8019701ED
:10BE70000E943E9B181644F4C601B501A801970123
:10BE80000E943099882314F4860175016D8D7E8D92
:10BE90008F8D98A125966CAF7DAF8EAF9FAF259704
:10BEA0008091F9079091FA07A091FB07B091FC07E8
:10BEB00021968CAF9DAFAEAFBFAF2197BC01CD0136
:10BEC00020E030E040E05FE30E94109C1B012C0169
:10BED00025966CAD7DAD8EAD9FAD25979F77A20168
:10BEE00091010E943E9B181644F4C801B701A201BB
:10BEF00091010E943099882314F41701280181E5EB
:10BF000090E0E596AEADBFADE597A89FF001A99F83
:10BF1000F00DB89FF00D1124EE5DF74F22A133A173
:10BF200044A155A12DA73EA74FA758ABC201B1010F
:10BF30000E94309987FD04C02DA43EA44FA458A8A8
:10BF400049AD5AAD423051050CF411C15091340D38
:10BF5000CD55DF4F5883C35AD0406091350DCC5535
:10BF6000DF4F6883C45AD0407091360DCB55DF4FF8
:10BF70007883C55AD0408091370DCA55DF4F8883EA
:10BF8000C65AD040652FCC55DF4F7881C45AD04077
:10BF9000CB55DF4F8881C55AD040CA55DF4F9881B5
:10BFA000C65AD04027E137EB41ED58E30E943E9B53
:10BFB00018160CF0DCC069897A898B899C892091DC
:10BFC000380D3091390D40913A0D50913B0D0E9442
:10BFD00056989B01AC010E94109C7B018C016D89DD
:10BFE0007E898F89988D20913C0D30913D0D409137
:10BFF0003E0D50913F0D0E9456989B01AC010E944E
:10C00000109C9B01AC01C801B7010E9457980E9487
:10C010007D9C7B018C01A40193010E943E9B18161C
:10C020005CF00F2EF0E06F2EF0E07F2EF0E88F2E08
:10C03000FFE39F2EF02D08C0C401B301A8019701B2
:10C040000E9437993B014C012D966CAD7DAD8EADB4
:10C050009FAD2D972091400D3091410D4091420DA3
:10C060005091430D0E9456987B018C01E89417F97A
:10C07000C801B70129962CAD3DAD4EAD5FAD2997F6
:10C080000E943E9B1816A4F429966CAD7DAD8EAD32
:10C090009FAD2997A80197010E9437995B016C0118
:10C0A000C401B301A60195010E943099882314F4BC
:10C0B0006401530125966CAD7DAD8EAD9FAD259786
:10C0C0002091440D3091450D4091460D5091470D02
:10C0D0000E9456987B018C01E89417F9C801B701BA
:10C0E00021962CAD3DAD4EAD5FAD21970E943E9B9C
:10C0F0001816A4F421966CAD7DAD8EAD9FAD219741
:10C10000A80197010E9437997B018C01C601B501F6
:10C11000A80197010E943099882314F486017501C3
:10C120006DA57EA58FA598A9A80197010E94109CD6
:10C130007B018C01CD55DF4F6881C35AD040CC556F
:10C14000DF4F7881C45AD040CB55DF4F8881C55A24
:10C15000D040CA55DF4F9881C65AD040A8019701F8
:10C160000E94309987FD19C0D801C70102C0D201D1
:10C17000C101CD55DF4F8883C35AD040CC55DF4F26
:10C180009883C45AD040CB55DF4FA883C55AD040BE
:10C19000CA55DF4FB883C65AD04081E590E0E59696
:10C1A000AEADBFADE597A89F8001A99F100DB89FC8
:10C1B000100D11240E5D174FCD55DF4F8881C35AE6
:10C1C000D040CC55DF4F9881C45AD040CB55DF4F7B
:10C1D000A881C55AD040CA55DF4FB881C65AD04051
:10C1E000F80182A793A7A4A7B5A762A973A984A9F8
:10C1F00095A9905820E030E040E050EC0E94109C5F
:10C20000D8019E962D913D914D915C91D1970E94C0
:10C21000109C2BE037ED43E25BE30E9457980E94AD
:10C220007D9CF62EE72ED82EC92ECD55DF4F688186
:10C23000C35AD040CC55DF4F7881C45AD040CB553B
:10C24000DF4F8881C55AD040CA55DF4F9881C65A02
:10C25000D0402F2D3E2D4D2D5C2D0E94309987FD15
:10C2600014C0CD55DF4FF882C35AD040CC55DF4FB4
:10C27000E882C45AD040CB55DF4FD882C55AD0404F
:10C28000CA55DF4FC882C65AD04081E590E0E59696
:10C29000EEADFFADE597E89F8001E99F100DF89F97
:10C2A000100D11240E5D174FCD55DF4F8881C35AF5
:10C2B000D040CC55DF4F9881C45AD040CB55DF4F8A
:10C2C000A881C55AD040CA55DF4FB881C65AD04060
:10C2D000F80186A397A3A0A7B1A762A173A184A127
:10C2E00095A12F2D3E2D4D2D5C2D0E9430991816B5
:10C2F0002CF081E0D801D7968C9302C0F80117AAE0
:10C3000081E590E0E5962EAD3FADE597289FF001E1
:10C31000299FF00D389FF00D1124EE5DF74F81E05D
:10C3200086ABA8E3BDE0FE01719680E101900D921D
:10C330008150E1F781E590E0E5964EAD5FADE59780
:10C34000489F6001499FD00C589FD00C112462E295
:10C3500078E0C60ED71ED6019296ED90FD900D9115
:10C360001C919597E092340DF092350D0093360DA7
:10C370001093370D96966D917D918D919C91999723
:10C38000A80197010E9437994B015C01C201B101DC
:10C39000A80197010E9437998B019C01C601B50144
:10C3A000A4010E94A052BBADB093320DC356DF4F23
:10C3B000288139814A815B81CD59D04020931D0865
:10C3C00030931E0840931F0850932008C756DF4F34
:10C3D000488159816A817B81C959D04040931908AD
:10C3E00050931A0860931B0870931C08CB56DF4FBC
:10C3F000688179818A819B81C559D04060931508F5
:10C40000709316088093170890931808CF56DF4F43
:10C4100088819981AA81BB81C159D040809311083C
:10C4200090931208A0931308B09314080E94225509
:10C430000E943076C655DF4F0FB6F894DEBF0FBEB0
:10C44000CDBFCF91DF911F910F91FF90EF90DF90C3
:10C45000CF90BF90AF909F908F907F906F905F90A4
:10C460004F903F902F9008952F923F924F925F925E
:10C470006F927F928F929F92AF92BF92CF92DF92F4
:10C48000EF92FF920F931F93DF93CF9300D000D0D2
:10C49000CDB7DEB71C017C836B836A01FA01E080B3
:10C4A000F18002811381C801B70120E030E040E053
:10C4B00050E00E943E9B87FF04C017FB109517F9C0
:10C4C0001095C101880F991F880F991F9A8389833E
:10C4D00026016624772443C0F401A080B180C28085
:10C4E000D380C601B50120E030E040E050E00E947A
:10C4F0003E9B88231CF0A601950103C0A60195016F
:10C500005058C801B7010E94309988239CF4C60195
:10C51000B50120E030E040E050E00E943E9B8823DF
:10C520001CF08601750106C08601750117FB109588
:10C5300017F910958D819E8101969E838D83E4E08D
:10C54000F0E08E0E9F1E8D819E818215930524F250
:10C550000894611C711CE981FA814E0E5F1E8B816B
:10C560009C816816790624F442011E821D82EBCF5D
:10C57000B701C80126960FB6F894DEBF0FBECDBF37
:10C58000CF91DF911F910F91FF90EF90DF90CF90AF
:10C59000BF90AF909F908F907F906F905F904F90E3
:10C5A0003F902F9008952F923F924F925F926F92FB
:10C5B0007F928F929F92AF92BF92CF92DF92EF9233
:10C5C000FF920F931F93DF93CF93CDB7DEB72A97D8
:10C5D0000FB6F894DEBF0FBECDBF98878F834A0198
:10C5E0005B013901181619060CF063C1CB01BA01C1
:10C5F00020E030E040E050E00E943099882309F4C8
:10C6000058C10130110529F421E0C216D10419F4F2
:10C6100060C017FD03C020E030E00DC081E090E075
:10C620004F815885841B950B089F9001099F300D01
:10C63000189F300D1124D7FC03C060E070E00DC0DE
:10C6400081E090E0EF81F8858E1B9F0BC89EB001C2
:10C65000C99E700DD89E700D1124CC0CDD1CCC0C25
:10C66000DD1C1B01220C331C220C331C2E0C3F1C26
:10C670002801440C551C440C551C7901EE0CFF1C80
:10C68000EE0CFF1CE60CF71C00E010E0C501B40145
:10C69000F70120813181428153810E94109C9B01CE
:10C6A000AC01F10160817181828193810E94579870
:10C6B000F10160837183828393830F5F1F4F2C0C82
:10C6C0003D1CE40CF51C2F81388502171307F4F28A
:10C6D000F0C00F81188503701070670123012224B8
:10C6E00033241CC0C501B401F20121913191419163
:10C6F00051912F010E94109C9B01AC01F6016081B9
:10C700007181828193810E945798F60161937193A0
:10C71000819391936F010894211C311C20163106DE
:10C720000CF3C801880F991F880F991F1701280E55
:10C73000391E9301280F391F3E832D830F5F1F4F32
:10C74000C801880F991F880F991F2701480E591E8D
:10C75000A301480F591F5C834B830F5F1F4FC80114
:10C76000880F991F880F991F6701C80ED91EF30102
:10C77000E80FF91FFA83E9830F5F1F4FC801880F85
:10C78000991F880F991F035010409701280F391FD8
:10C790003A8729877301E80EF91E85C0C501B401E7
:10C7A000ED81FE8120813181428153810E94109C64
:10C7B0009B01AC01F10160817181828193810E94B2
:10C7C0005798F1016083718382839383C501B4011B
:10C7D000EB81FC8120813181428153810E94109C38
:10C7E0009B01AC01F20160817181828193810E9481
:10C7F0005798F2016083718382839383C501B401EA
:10C80000E981FA8120813181428153810E94109C0B
:10C810009B01AC01F60160817181828193810E944C
:10C820005798F6016083718382839383C501B401B5
:10C83000F70120813181428153810E94109C9B012C
:10C84000AC01E985FA8560817181828193810E94C2
:10C850005798E985FA8560837183828393830C5F9F
:10C860001F4F20E130E0220E331E4D815E81405F7C
:10C870005F4F5E834D83420E531E8B819C81409699
:10C880009C838B83C20ED31EE981FA817096FA8352
:10C89000E98329853A85205F3F4F3A87298740E120
:10C8A00050E0E40EF51E8F819885081719070CF4E7
:10C8B00075CF2A960FB6F894DEBF0FBECDBFCF91CD
:10C8C000DF911F910F91FF90EF90DF90CF90BF907D
:10C8D000AF909F908F907F906F905F904F903F9020
:10C8E0002F9008952F923F924F925F926F927F9276
:10C8F0008F929F92AF92BF92CF92DF92EF92FF9270
:10C900000F931F93DF93CF93CDB7DEB72E970FB65C
:10C91000F894DEBF0FBECDBF9E878D874B013901D6
:10C92000F801181619065CF00F2EF0E0CF2EF0E09B
:10C93000DF2EF0E0EF2EF0E0FF2EF02D93C141301E
:10C94000510521F40130110519F469C057FD03C0E8
:10C9500060E070E00DC081E090E02D853E85821B97
:10C96000930B489FB001499F700D589F700D112483
:10C97000F7FD03C020E030E00DC081E090E0AD8520
:10C98000BE858A1B9B0BE89F9001E99F300DF89FA5
:10C99000300D11242A01440C551C440C551C8B01EC
:10C9A000000F111F000F111F080D191D4F01880CDA
:10C9B000991C880C991C1901220C331C220C331C65
:10C9C000260C371C0F2EF0E0CF2EF0E0DF2EF0E02B
:10C9D000EF2EF0E0FF2EF02DAA24BB24F801608199
:10C9E000718182819381D1012D913D914D915C9115
:10C9F0000E94109C9B01AC01C701B6010E94579890
:10CA00006B017C010894A11CB11C040D151D280CA0
:10CA1000391CED85FE85AE16BF0604F323C18D8556
:10CA20009E8565E070E00E94159D8C010F2EF0E060
:10CA3000CF2EF0E0DF2EF0E0EF2EF0E0FF2EF02D15
:10CA4000AA24BB24442455241FC0F401E40DF51D81
:10CA5000D301A40DB51D60817181828193812D91D7
:10CA60003D914D915C910E94109C9B01AC01C701CE
:10CA7000B6010E9457986B017C010894A11CB11C5F
:10CA800024E030E0420E531EA016B106F4F2C801B5
:10CA9000880F991F880F991FD401A80FB91FBC8751
:10CAA000AB87F301E80FF91FFA87E9870F5F1F4F84
:10CAB000C801880F991F880F991F9401280F391FEB
:10CAC00038872F83D301A80FB91FBE83AD830F5FB3
:10CAD0001F4FC801880F991F880F991FF401E80F95
:10CAE000F91FFC83EB839301280F391F3A832983B5
:10CAF0000F5F1F4FC801880F991F880F991F1401DE
:10CB0000280E391E2301480E591E0F5F1F4FC80102
:10CB1000880F991F880F991F04501040880E991E86
:10CB20005301A80EB91E380197C0AB85BC856D9125
:10CB30007D918D919C91E985FA8520813181428199
:10CB400053810E94109C9B01AC01C701B6010E9459
:10CB500057987B018C01AF81B8856D917D918D9146
:10CB60009C91ED81FE8120813181428153810E941F
:10CB7000109C9B01AC01C801B7010E9457987B0132
:10CB80008C01AB81BC816D917D918D919C91E981EE
:10CB9000FA8120813181428153810E94109C9B0146
:10CBA000AC01C801B7010E9457987B018C01D101EB
:10CBB0006D917D918D919C91F20120813181428115
:10CBC00053810E94109C9B01AC01C801B7010E94D7
:10CBD00057987B018C01D4016D917D918D919C9131
:10CBE000F50120813181428153810E94109C9B017B
:10CBF000AC01C801B7010E9457986B017C0125E088
:10CC000030E0620E731E8B859C8544969C878B87D3
:10CC1000A985BA855496BA87A987EF81F885749655
:10CC2000F887EF832D813E812C5E3F4F3E832D831D
:10CC30008B819C8144969C838B83A981BA81549675
:10CC4000BA83A983E4E1F0E02E0E3F1E4E0E5F1E74
:10CC50008E0E9F1EAE0EBF1E2D853E85621673067C
:10CC60000CF463CFB601C7012E960FB6F894DEBF61
:10CC70000FBECDBFCF91DF911F910F91FF90EF902D
:10CC8000DF90CF90BF90AF909F908F907F906F90EC
:10CC90005F904F903F902F9008952F923F924F9228
:10CCA0005F926F927F928F929F92AF92BF92CF923C
:10CCB000DF92EF92FF920F931F93DF93CF93CDB745
:10CCC000DEB7EC970FB6F894DEBF0FBECDBF9CA7C2
:10CCD0008BA77EA76DA758AB4FA73AAB29AB1CAB70
:10CCE0000BAB37017601BEAAADAA98AE8FAA6896A3
:10CCF000EEADFFAD689700E010E0CF01815F984D89
:10CD00008F519E4410F001E010E0CF0160E177E226
:10CD10000E94159D9AAF89AF892B21F061E070E0E8
:10CD20007AAF69AF1AA619A6CF0168EE73E00E9428
:10CD3000159D8D599F4F873C910520F081E090E033
:10CD40009AA789A718A61FA2CF0164E670E00E94E7
:10CD5000159D0996439720F0A1E0B0E0B8A7AFA3D6
:10CD6000CF016AE070E00E94159D9CAF8BAF892BCC
:10CD700021F0E1E0F0E0FCAFEBAF8FA598A90197BF
:10CD800029A93AA93A8329838217930714F49A832D
:10CD9000898369817A81672B09F068C0012B51F082
:10CDA000F30180819181A281B381F7018083918316
:10CDB000A283B38329AD3AAD232B59F0F3018081CF
:10CDC0009181A281B381EDA9FEA980839183A28381
:10CDD000B3832BAD3CAD232B69F0F30180819181AE
:10CDE000A281B3816696EEADFFAD66978083918395
:10CDF000A283B38329A53AA5232B21F1ABA5BCA51A
:10CE0000ED90FD900D911C91C801B70120E030E03C
:10CE100040E050E00E943099882329F4E1E0F0E0FE
:10CE2000FEA3EDA311C0D3016D917D918D919C91D5
:10CE3000A80197010E943799EFA9F8AD608371832B
:10CE4000828393831EA21DA22FA138A5232B09F450
:10CE5000F9C380E090E0A0E0B0E06496EEADFFADF5
:10CE6000649780839183A283B383ECC3011511057A
:10CE7000E9F061E070E040E050E013C09701240F5A
:10CE8000351FF301E40FF51F80819181A281B381E9
:10CE9000F90180839183A283B3836F5F7F4F4C5FDF
:10CEA0005F4F2FA538A92617370744F769AD7AAD2C
:10CEB000672BF1F061E070E040E050E014C02DA974
:10CEC0003EA9240F351FF301E40FF51F80819181E6
:10CED000A281B381F90180839183A283B3836F5FC1
:10CEE0007F4F4C5F5F4F2FA538A9261737073CF7B8
:10CEF000012B09F4C7C021E030E069817A81261B4B
:10CF0000370BA901440F551F440F551F50954195EC
:10CF10005F4F8BA99CA9840F951F9C8B8B8BADA514
:10CF2000BEA5A095B095AA0FBB1FAA0FBB1FBA8BB9
:10CF3000A98B615070408DA59EA50196689F200128
:10CF4000699F500C789F500C1124440C551C440CC4
:10CF5000551CEBA5FCA54E0E5F1EAFA5B8A91196FA
:10CF6000B8ABAFA7E981FA81AE1BBF0BB88BAF8717
:10CF7000AFA5B8A91197B8ABAFA7880F991F880FB5
:10CF8000991FEE27FF27E81BF90BFE87ED878DA57C
:10CF90009EA5689F3001699F700C789F700C1124CA
:10CFA000621A730A660C771C660C771CABA5BCA5CD
:10CFB0006A0E7B1E1701240E351EE1E0F0E0FAA395
:10CFC000E9A358C0AB89BC89ED90FD900D911C91EF
:10CFD000C801B70120E030E040E050E00E94309905
:10CFE000882361F1F20180809180A280B380D20118
:10CFF000ED92FD920D931C9313978F859889B30141
:10D0000041E050E0910101E010E06CDC9058F20149
:10D0100020813181428153810E943799AB01BC014B
:10D020008F85988993017101E1E0CE2ED12CBBDA76
:10D03000D2018D929D92AD92BC921397E9A1FAA173
:10D040003196FAA3E9A32B893C89245030403C8BCC
:10D050002B8B69897A89460E571E8F859889019690
:10D06000988B8F87AD85BE856A0E7B1EECEFFFEF38
:10D070002E0E3F1E29A13AA169817A81621773079A
:10D080000CF0A0CF89AD9AAD892B09F489C0ADA56C
:10D09000BEA51196BEA7ADA7AA0FBB1FAA0FBB1FA7
:10D0A000BE8BAD8BEDA5FEA53197FEA7EDA72BA4FA
:10D0B0003CA44FA458A8CF0180959095880F991F44
:10D0C000880F991F22273327281B390B3C832B837A
:10D0D000310161E070E07CA36BA3188E1F8A58C0F9
:10D0E000EBA9FCA98F89988DE80FF91FE080F180EA
:10D0F00002811381C801B70120E030E040E050E038
:10D100000E943099882369F1D1018D909D90AD9056
:10D11000BC90F101E082F18202831383EDA8FEA8A6
:10D120002F89388DE20EF31EC201B30141E050E0B9
:10D13000970101E010E0D6DB9058D1012D913D918F
:10D140004D915C910E943799AB01BC01C2019301E2
:10D15000E1E0CE2ED12C27DAF10180829182A282E9
:10D16000B3822BA13CA12F5F3F4F3CA32BA36F8920
:10D17000788D6C5F7F4F788F6F8B8D899E89280E9D
:10D18000391E089441085108AB81BC816A0E7B1E90
:10D19000EBA1FCA129813A812E173F070CF0A0CF0B
:10D1A00069A57AA5672BF9F061E070E040E050E0F6
:10D1B00015C02FA938AD240F351FEDA9FEA9E40F26
:10D1C000F51F80819181A281B381F90180839183D0
:10D1D000A283B3836F5F7F4F4C5F5F4F29A93AA94A
:10D1E0002617370734F76BAD7CAD672B09F161E08B
:10D1F00070E040E050E017C066962EAD3FAD6697F8
:10D20000240F351FEDA9FEA9E40FF51F8081918140
:10D21000A281B381F90180839183A283B3836F5F7D
:10D220007F4F4C5F5F4F29A93AA92617370724F78C
:10D230006FA178A5672B41F189A99AA9AFA5B8A9D3
:10D240008A179B070CF59C01880F991F880F991F5F
:10D250004DA95EA9480F591F6496EEADFFAD6497C6
:10D26000E80FF91F0AC0DA01ED90FD900D911D91B4
:10D27000AD01E192F192019311932F5F3F4F6FA5A2
:10D2800078A9621773077CF78BAD9CAD892B11F1E0
:10D29000A9A9BAA9EFA5F8A9AE17BF07DCF4CD017B
:10D2A000FD01EE0FFF1FEE0FFF1F66962EAD3FAD87
:10D2B0006697E20FF31F20E030E040E050E004C04A
:10D2C000219331934193519301966FA578A96817E3
:10D2D0007907B4F78FA198A5892BA9F06496EEADD4
:10D2E000FFAD649781E090E020E030E040E050E066
:10D2F00005C021933193419351930196A9A9BAA9ED
:10D30000A817B907B4F7E9A5FAA5EF2B09F49EC051
:10D3100069A87AA8089461087108660C771C660CE5
:10D32000771C2FA938AD620E731E8DA59EA5880FA0
:10D33000991F880F991F66277727681B790B7A8FAB
:10D34000698F89A99AA90197ADA5BEA58A9F4001B9
:10D350008B9F900C9A9F900C1124880C991C880C20
:10D36000991CEBA5FCA58E0E9F1EA095B095AA0F4B
:10D37000BB1FAA0FBB1FBE83AD832DA53EA52F5F8C
:10D380003F4F829F5001839FB00C929FB00C11249D
:10D39000215030403EA72DA7AA0CBB1CAA0CBB1CD9
:10D3A000AE0EBF1E29A83AA8F1E04F2E512C48C05E
:10D3B000C9A8DAA8C418D508D501ED90FD900D9143
:10D3C0001C91C801B70120E030E040E050E00E942D
:10D3D0003099882319F43EA22DA23AC0F30160814E
:10D3E000718182819381A80197010E943799D301AD
:10D3F0006D937D938D939C931397B1E02B1631041D
:10D4000069F0AB01BC017058C601940101E010E065
:10D41000EFA8F8ACE1E0CE2ED12CC5D80894411C81
:10D42000511CECEFFFEF6E0E7F1E089421083108AF
:10D43000298D3A8D820E931E6D817E81A60EB71EB8
:10D4400089A99AA9841595050CF0B2CF1EA21DA238
:10D45000AFA1B8A5AB2B09F466C041E050E0E9816B
:10D46000FA814E1B5F0B9A01220F331F220F331FCD
:10D47000309521953F4F6BA97CA9620F731F78A34C
:10D480006F8F8DA59EA580959095880F991F880F09
:10D49000991F9E8F8D8FBF01615070408DA59EA5F5
:10D4A0000196689F3001699F700C789F700C112461
:10D4B000660C771C660C771CABA5BCA56A0E7B1EA0
:10D4C0008FA498A80894811C911C8E1A9F0A880F1B
:10D4D000991F880F991FEE27FF27E81BF90BFC8F78
:10D4E000EB8F8DA59EA5689F5001699FB00C789F1A
:10D4F000B00C1124A41AB50AAA0CBB1CAA0CBB1CA4
:10D50000AA0EBB1E66962EAC3FAC6697220E331E4B
:10D5100064964EAC5FAC6497420E531EA1E0B0E03F
:10D52000BC87AB8787C0EBADFCADEF2B09F095CF87
:10D5300089C0AF8DB8A1ED90FD900D911C91C801EF
:10D54000B70120E030E040E050E00E9430998823AD
:10D5500009F454C0D3016D917D918D919C916F839D
:10D56000788789879A87F301E082F18202831383A7
:10D570002FA138A5232BD1F0C401B50141E050E023
:10D58000920101E010E0AED99058D3012D913D9168
:10D590004D915C910E943799AB01BC01C40195018A
:10D5A0007201F1E0CF2ED12C0E94D362EBADFCAD25
:10D5B000EF2BD1F0C401B50141E050E0910101E051
:10D5C00010E090D99058D3012D913D914D915C91EF
:10D5D0000E943799AB01BC01C40195017101E1E0E2
:10D5E000CE2ED12C0E94D3626F81788589859A8551
:10D5F000D3016D937D938D939C931397EB85FC855D
:10D600003196FC87EB872F8D38A12450304038A30A
:10D610002F8F6D8D7E8D660E771E0894811C911C58
:10D620008B8D9C8DA80EB91EACEFBFEF2A0E3B1E52
:10D630004A0E5B1EEB85FC8529813A812E173F0738
:10D640000CF077CF8DA19EA1EC960FB6F894DEBFBB
:10D650000FBECDBFCF91DF911F910F91FF90EF9043
:10D66000DF90CF90BF90AF909F908F907F906F9002
:10D670005F904F903F902F9008952F923F924F923E
:10D680005F926F927F928F929F92AF92BF92CF9252
:10D69000DF92EF92FF920F931F93DF93CF9300D00F
:10D6A0000F92CDB7DEB79C838B833A8329833801F1
:10D6B000260114010115110509F100D000D0EDB7C4
:10D6C000FEB73196ADB7BEB71296BC92AE92119727
:10D6D000B382A2828EE690E0958384838B819C81C5
:10D6E00098010A8D1B8D65014201D7DAEDB7FEB7AF
:10D6F00036960FB6F894FEBF0FBEEDBF6101F10183
:10D7000020E030E009C080819181909581959F4F04
:10D71000819391932F5F3F4F89819A812817390711
:10D7200094F3F301EE0FFF1FEE0FFF1FE40DF51D45
:10D73000830180E090E0A0E0B0E006C08193919387
:10D74000A193B1930F5F1F4F29813A8102171307ED
:10D75000ACF3720101E010E0F1E0AF2EB12C46C055
:10D76000D6018D919C91119718161906ACF12227BC
:10D770003327281B390B2D933C932BC0F701408195
:10D78000518162817381C501821B930B9C01880FBB
:10D79000991F880F991FF201E81BF90B60807180B7
:10D7A00082809380D7016D927D928D929C92139787
:10D7B0004083518362837383220F331FF101E21B85
:10D7C000F30B8081918122273327281B390B31836A
:10D7D00020832017310791F60F5F1F4FE2E0F0E042
:10D7E000CE0EDF1E24E030E0E20EF31E89819A8126
:10D7F000801791070CF0B4CF0F900F900F900F90FF
:10D80000CF91DF911F910F91FF90EF90DF90CF901C
:10D81000BF90AF909F908F907F906F905F904F9050
:10D820003F902F9008952F923F924F925F926F9268
:10D830007F928F929F92AF92BF92CF92DF92EF92A0
:10D84000FF920F931F93DF93CF9300D00F92CDB72A
:10D85000DEB79A8389833A014B012901181619060C
:10D860000CF0EAC00130110509F0AFC065E070E0CE
:10D870000E94159D8C017901CC24DD2412C0F70192
:10D880006081718182819381A40193010E94109C27
:10D89000F70161937193819391937F010894C11C67
:10D8A000D11CC016D1065CF31801220C331C220CCB
:10D8B000331C240C351C58010894A11CB11CAA0C63
:10D8C000BB1CAA0CBB1CA40CB51C42E0C42ED12C62
:10D8D000C00ED11ECC0CDD1CCC0CDD1CC40CD51C28
:10D8E00023E0E22EF12CE00EF11EEE0CFF1CEE0CFC
:10D8F000FF1CE40CF51C98012C5F3F4F220F331FD7
:10D90000220F331F240D351D3C832B8357C0F1019B
:10D910006081718182819381A40193010E94109C96
:10D92000F1016083718382839383F501608171814A
:10D9300082819381A40193010E94109CF501608370
:10D94000718382839383F6016081718182819381E7
:10D95000A40193010E94109CF6016083718382836D
:10D960009383F7016081718182819381A401930186
:10D970000E94109CF7016083718382839383EB8103
:10D98000FC816081718182819381A40193010E9455
:10D99000109CEB81FC8160837183828393830B5F96
:10D9A0001F4F24E130E0220E331EA20EB31EC20E22
:10D9B000D31EE20EF31E7496FC83EB8389819A8159
:10D9C000081719070CF4A3CF37C017FD03C060E098
:10D9D00070E00DC081E090E0E981FA818E1B9F0B21
:10D9E000089FB001099F700D189F700D11247801D8
:10D9F000EE0CFF1CEE0CFF1C6B01CC0CDD1CCC0CE8
:10DA0000DD1CC40CD51C00E010E0F60160817181C2
:10DA100082819381A40193010E94109CF60160838E
:10DA20007183828393830F5F1F4FCE0CDF1C29818C
:10DA30003A81021713074CF30F900F900F900F903D
:10DA4000CF91DF911F910F91FF90EF90DF90CF90DA
:10DA5000BF90AF909F908F907F906F905F904F900E
:10DA60003F902F9008954F925F926F927F928F9286
:10DA70009F92AF92BF92CF92DF92EF92FF920F935D
:10DA80001F93CF93DF932C014B0139011816190610
:10DA90000CF0F2C04130510509F09CC00130110575
:10DAA00009F09AC063E070E00E94159DBC018401FA
:10DAB000E901E0E0F0E014C0D8012D913D914D91D5
:10DAC0005C911397C880D980EA80FB80CD92DD926B
:10DAD000ED92FD928D012993399349935993319693
:10DAE000E617F7074CF3CB01880F991F880F991F92
:10DAF0005401A80EB91E6301C80ED91E6F5F7F4F77
:10DB0000CB01880F991F880F991F7401E80EF91E29
:10DB10008301080F191F6F5F7F4FCB01880F991F7B
:10DB2000880F991F62507040E401C80FD91FF3019C
:10DB3000E80FF91F4AC0D5012D913D914D915C919F
:10DB4000D6016D907D908D909C90D5016D927D92C7
:10DB50008D929C921397D6012D933D934D935C9398
:10DB60001397D7012D913D914D915C91D8016D9006
:10DB70007D908D909C90D7016D927D928D929C921C
:10DB80001397D8012D933D934D935C931397288160
:10DB900039814A815B8180819181A281B3818883AF
:10DBA0009983AA83BB8320833183428353836D5F30
:10DBB0007F4F8CE090E0A80EB91EC80ED91EE80E6B
:10DBC000F91E045F1F4F2C963C96641575050CF4E6
:10DBD000B2CF52C057FD03C020E030E00BC081E05F
:10DBE00090E084199509489F9001499F300D589FF6
:10DBF000300D112417FD03C060E070E00BC081E020
:10DC000090E084199509089FB001099F700D189F35
:10DC1000700D11247A01EE0CFF1CEE0CFF1CE901C3
:10DC2000CC0FDD1FCC0FDD1FC80DD91D000F111F3C
:10DC3000000F111FFB01EE0FFF1FEE0FFF1FE60D80
:10DC4000F71D60E070E0288139814A815B81808125
:10DC50009181A281B38188839983AA83BB83208326
:10DC60003183428353836F5F7F4FCE0DDF1DE00F03
:10DC7000F11F641575053CF3DF91CF911F910F9152
:10DC8000FF90EF90DF90CF90BF90AF909F908F90DC
:10DC90007F906F905F904F9008952F923F924F9298
:10DCA0005F926F927F928F929F92AF92BF92CF922C
:10DCB000DF92EF92FF920F931F93CF93DF937C013C
:10DCC0005B014A016E9DC0016F9D900D7E9D900D80
:10DCD0001124880F991F880F991F0E94020B792E1B
:10DCE000482F592F682E6701CC0CDD1CCC0CDD1C95
:10DCF000E0E0F0E060E070E012C0D8012D903D90CF
:10DD00004D905D908D0129923992499259922F5FE1
:10DD10003F4F2E153F058CF331966C0D7D1DEA1596
:10DD2000FB054CF48401060F171FEA01C60FD71F2D
:10DD300020E030E0EECFC301DF91CF911F910F9132
:10DD4000FF90EF90DF90CF90BF90AF909F908F901B
:10DD50007F906F905F904F903F902F9008952F92FB
:10DD60003F924F925F926F927F928F929F92AF926B
:10DD7000BF92CF92DF92EF92FF920F931F93DF93A8
:10DD8000CF9300D00F92CDB7DEB71C01FB01181660
:10DD900019060CF0A8C0141615060CF0A4C081E0FA
:10DDA0002816310499F4E080F18002811381C801C2
:10DDB000B70120E030E040E050E00E943E9B87FF4A
:10DDC0009CC017FB109517F9109597C0DA01AA0FA0
:10DDD000BB1FAA0FBB1FBA83A9832B011C821B8206
:10DDE0000F2EF0E0EF2EF0E0FF2EF0E00F2FF0E02E
:10DDF0001F2FF02D0F2EF0E06F2EF0E07F2EF0E8B9
:10DE00008F2EFFE39F2EF02DF201A080B180C28003
:10DE1000D380C601B50120E030E040E050E00E9430
:10DE20003099882309F445C0C601B50120E030E0EF
:10DE300040E050E00E943E9B87FF04C0D7FAD09498
:10DE4000D7F8D094C801B701A60195010E94309976
:10DE50008823ECF4C801B701A60195010E94379907
:10DE60007B018C01C401B301A80197010E94109CA1
:10DE7000A80197010E94109C20E030E040E85FE399
:10DE80000E9457983B014C018601750112C0C601E2
:10DE9000B501A80197010E9437999B01AC010E942E
:10DEA000109C9B01AC01C401B3010E9457983B0137
:10DEB0004C018B819C8101969C838B83A981BA81C3
:10DEC0004A0E5B1E821593050CF49ECFC401B3016C
:10DED0000E947D9C9B01AC01C801B7010E94109C6F
:10DEE0007B018C010AC00F2EF0E0EF2EF0E0FF2E38
:10DEF000F0E00F2FF0E01F2FF02DB701C8010F90B9
:10DF00000F900F900F90CF91DF911F910F91FF9085
:10DF1000EF90DF90CF90BF90AF909F908F907F90C9
:10DF20006F905F904F903F902F9008952F923F9267
:10DF30004F925F926F927F928F929F92AF92BF9219
:10DF4000CF92DF92EF92FF920F931F93DF93CF93C5
:10DF5000CDB7DEB7C254D0400FB6F894DEBF0FBEC7
:10DF6000CDBF98AB8FA77AAB69AB5CAB4BAB3EAB8D
:10DF70002DAB18AF0FABFAAEE9AEDCAECBAEAB2833
:10DF800031F431E0432E512C22243324E7C0E9AC94
:10DF9000FAACAFA4B8A821E0622E712C91E0492E12
:10DFA000512CCC24CA94DC2C81E0882E912C52C0B8
:10DFB000D7018D919C91119797FF03C0CD92DC9270
:10DFC00003C0F7017182608218161906ACF564145B
:10DFD0007504F9F008944108510829A93AA9429E0C
:10DFE000B001439E700D529E700D11240894411C87
:10DFF000511C660F771F660F771F4FA558A9640F36
:10E00000751F8BA99CA941E050E0950101E010E04B
:10E010002ADDF201E819F909EE0FFF1F89AD9AAD6B
:10E02000E80FF91F80819181D7018D939C937182B4
:10E0300060820894411C511C0894611C711CE2E030
:10E04000F0E0EE0EFF1E24E030E0A20EB31E0894B6
:10E05000C108D1084DA95EA9461557050CF0A8CFF7
:10E060004A01089481089108880C991C89AD9AADE1
:10E07000880E991E89A99AA9880F991F880F991F40
:10E08000AA24BB24A81AB90A41505040A9A9BAA988
:10E090004A9F70014B9FF00C5A9FF00C11244F5F68
:10E0A0005F4F5EAB4DABEE0CFF1CEE0CFF1CEFA503
:10E0B000F8A9EE0EFF1E6A011A014CC0D4012D9181
:10E0C0003C91119737FF3DC088279927821B930BFE
:10E0D0008D939C93C214D30489F1089421083108CC
:10E0E000E9A9FAA92E9EB0012F9E700D3E9E700DDB
:10E0F00011240894211C311C660F771F660F771FAF
:10E100002FA538A9620F731F8BA99CA941E050E08D
:10E11000970101E010E0A7DCF1013197EE0FFF1F3E
:10E1200049AD5AADE40FF51F20813181D4018D91A5
:10E130009C911197918380832D933C93089421089F
:10E1400031080894C108D108EEEFFFEF8E0E9F1E34
:10E15000EA0CFB1C1C141D040CF4B0CF29A93AA92D
:10E16000220F331F220F331F3E872D87089441084B
:10E17000510849A95AA9449E8001459E100D549EFC
:10E18000100D1124000F111F000F111F8FA598A94A
:10E19000080F191FA0E0B0E04A0E5B1E5201AA0C46
:10E1A000BB1CAA0CBB1C0894411C511CEFA8F8AC6A
:10E1B000EA0CFB1C3201670149019094819491089B
:10E1C000939411C0B801680D791D8BA99CA941E0F9
:10E1D00050E0C5DDF60161937193819391936F01D6
:10E1E0000894611C711C2D853E85020F131F261497
:10E1F000370444F7EBADFCADEA0DFB1D92010CC0FA
:10E20000D7014D915D916D917D917D014193519328
:10E21000619371932F5F3F4F221633068CF7EDA960
:10E22000FEA9FAA7E9A72BA93CA92E173F0714F4CA
:10E230003AA729A74FA958AD5C8F4B8F89A99AA9F6
:10E2400080959095880F991F880F991FAA27BB2743
:10E25000A81BB90BB88FAF8BEFA5F8A9FA8BE98B88
:10E2600029A93AA92F5F3F4F3AAB29AB220F331FA1
:10E27000220F331F3E8B2D8B49A95AA94150504084
:10E280005AAB49ABCF01AD85BE858A0F9B1F9CA3BE
:10E290008BA3EBADFCADFC8BEB8B4FA558A9420FCC
:10E2A000531F5A83498389AD9AAD988B8F87ABA949
:10E2B000BCA9BA8FA98FEFA5F8A9F887EF832BA186
:10E2C0003CA13C832B83FE83ED8341E050E05CA7BF
:10E2D0004BA7AFC28BA59CA5841595050CF4A2C0D5
:10E2E000821593050CF09EC07C0123969FAF8EAFE4
:10E2F00023970B8D1C8D8824AA24CC24DD24D801DF
:10E300006C9011967C90119712969C901297139690
:10E31000BC90682D7A2DC6019301492D5B2D0E947A
:10E32000309988232CF42396FFAEEEAE239704C0D9
:10E33000682C7A2C9C2CBD2C0894E11CF11C0C5FE1
:10E340001F4F2E143F042CF0862CA72CC92CDB2C3D
:10E35000D6CF2396EEADFFAD23972BA53CA5E217B4
:10E36000F30709F45FC0319749A95AA9E49F9001C6
:10E37000E59F300DF49F300D112431962396FFAFA9
:10E38000EEAF2397220F331F220F331F8FA598A9BB
:10E39000280F391F8BA99CA96D817E8141E050E037
:10E3A00001E010E060DB21E030E02396AEADBFADD0
:10E3B00023972A1B3B0BF901EE0FFF1FEE0FFF1FE8
:10E3C000F095E195FF4F4FA958AD4E0F5F1FAB8DF4
:10E3D000BC8DED90FD900D911C91DA01ED92FD92B6
:10E3E0000D931C9313974BAD5CADE40FF51FAB89F8
:10E3F000BC894D915D916D917C9140835183628385
:10E400007383220F331FE9ADFAADE21BF30B2081BA
:10E410003181AF85B8898D919C91119791838083CB
:10E420002D933C9320E030E040E050E0AB8DBC8D7C
:10E430002D933D934D935C931397EBA5FCA52BA9CE
:10E440003CA9E217F30709F4ADC12E1B3F0B3EA711
:10E450002DA7398D3FAF4A8D21964FAF21975F8110
:10E460005DAF88858EAF832F942F652F788541E02F
:10E4700050E075DC6DA37EA38FA398A720E030E069
:10E4800040E050E00E943099882309F48BC1A989AB
:10E49000BA89ED90FD900D911C91C801B70120E063
:10E4A00030E040E050E00E9430998823E9F0C80154
:10E4B000B70120E030E040E050E00E94309987FD55
:10E4C00005C020E030E040E85FE304C020E030E039
:10E4D00040E85FEB6DA17EA18FA198A50E94109CE2
:10E4E0006DA37EA38FA398A760E070E080E89FE310
:10E4F0002DA13EA14FA158A50E943799AB01BC01A7
:10E500008FAD21969FAD21972DAD3EAD01E010E07E
:10E510008AD9E989FA89608171818281938120E0B9
:10E5200030E040E85FE30E945798A989BA896D936B
:10E530007D938D939C931397EBA5FCA53196FC8757
:10E54000EB872B8D3C8D2C5F3F4F3AA329A34B8942
:10E550005C894C5F5F4F5E8F4D8F8B819C812396D2
:10E560009FAF8EAF2397A981BA81B8A3AF8FEBA1DC
:10E57000FCA1FA87E987F7C08FAD21969FAD21975F
:10E580006DAD7EAD41E050E022962FAD22972396EF
:10E590003FAD239701E010E00E9472649058A98972
:10E5A000BA892D913D914D915C910E943799AB01B3
:10E5B000BC018FAD21969FAD21972DAD3EAD22962A
:10E5C000EFAC22972396FFAC2397E1E0CE2ED12C1F
:10E5D0000E94D362EB85FC85E415F5050CF49AC026
:10E5E0002E163F060CF496C0A9A1BAA16D907D909D
:10E5F0008D909C90C401B30120E030E040E050E0F9
:10E600000E943099882309F485C0E985FA85E08065
:10E61000F18002811381C801B70120E030E040E0C1
:10E6200050E00E943E9B87FF04C017FB109517F92E
:10E630001095C801B701A40193010E9437999B016D
:10E64000AC010E94109C9B01AC0160E070E080E88E
:10E650009FE30E9456985B016C0120E030E040E0AF
:10E6600050E00E943E9B181654F00F2EF0E0AF2EA3
:10E67000F0E0BF2EF0E0CF2EF0E0DF2EF02DC40151
:10E68000B301AD8DBE8D2D913D914D915C910E9458
:10E6900037999B01AC010E94109C7B018C01C60143
:10E6A000B5012DEC3CEC4CE45DE30E94109CA8010C
:10E6B00097010E94109C20E030E040E85FE30E9458
:10E6C000579820E030E040E85FE30E9430998823CB
:10E6D00069F0C601B5010E947D9C9B01AC01C4019B
:10E6E000B3010E94109CE9A1FAA110C08DA59EA5BE
:10E6F0006F8D78A141E050E032DBA9A1BAA16D9302
:10E700007D938D939C931397ED8DFE8D6083718324
:10E71000828393832B853C852F5F3F4F3C872B87DC
:10E7200023964EAD5FAD23978D859E85480F591F6B
:10E7300023965FAF4EAF2397A9A1BAA11496BAA3AF
:10E74000A9A3EF8DF8A1E80FF91FF8A3EF8F2D8D86
:10E750003E8D2C5F3F4F3E8F2D8F49855A85480F48
:10E76000591F5A8749878B859C85ADA9BEA9A817D3
:10E77000B9070CF001CFE989FA8980819181A281E2
:10E78000B381EB8DFC8D80839183A283B3838DA1B4
:10E790009EA1AFA1B8A5B058E989FA898083918379
:10E7A000A283B3832BA53CA52F5F3F4F3CA72BA78C
:10E7B0004B8D5C8D4C5F5F4F5C8F4B8F898D9A8D3D
:10E7C00001979A8F898FAF81B885EF89F88DAE0F49
:10E7D000BF1FB887AF8329893A894D895E89240F85
:10E7E000351F3A8B298B8BA19CA1840F951F9CA36D
:10E7F0008BA3AB89BC891496BC8BAB8BE981FA8166
:10E80000E40FF51FFA83E9832B813C814F89588DF2
:10E81000240F351F3C832B838D819E81AD85BE8562
:10E820008A0F9B1F9E838D83EF85F8893296F88B24
:10E83000EF872BA53CA549A55AA5421753070CF015
:10E8400049CDCE5BDF4F0FB6F894DEBF0FBECDBF14
:10E85000CF91DF911F910F91FF90EF90DF90CF90BC
:10E86000BF90AF909F908F907F906F905F904F90F0
:10E870003F902F9008952F923F924F925F926F9208
:10E880007F928F929F92AF92BF92CF92DF92EF9240
:10E89000FF920F931F93DF93CF93CDB7DEB72C97E3
:10E8A0000FB6F894DEBF0FBECDBF9A8389837C83F9
:10E8B0006B832A013901ED82FE820F831887DA8685
:10E8C000C986F50180E090E003C011921192019693
:10E8D00086159705D4F3C301880F991F880F991FD8
:10E8E0000E94020B8B879C8789819A816B817C8136
:10E8F000A201930184017501CB84DC84E1E0AE2E9A
:10E90000B12C14DBE985FA851182108213014614BB
:10E9100057040CF412014B805C800894411C511C7C
:10E92000440C551C440C551C69807A808824992419
:10E9300040C0F301A080B180C280D380C601B50180
:10E9400020E030E040E050E00E943E9B87FF04C0A2
:10E95000D7FAD094D7F8D094E981FA81E080F18099
:10E9600002811381C801B70120E030E040E050E0AF
:10E970000E943E9B87FF04C017FB109517F9109566
:10E98000640C751C6D817E818F819885A80197012B
:10E990000E94109C9B01AC01C601B5010E943099F8
:10E9A00018167CF40894811C911CE985FA859182E3
:10E9B0008082821493040CF4BCCF8B859C850E94CA
:10E9C000AC0B2C960FB6F894DEBF0FBECDBFCF9127
:10E9D000DF911F910F91FF90EF90DF90CF90BF904C
:10E9E000AF909F908F907F906F905F904F903F90EF
:10E9F0002F9008952F923F924F925F926F927F9245
:10EA00008F929F92AF92BF92CF92DF92EF92FF923E
:10EA10000F931F93DF93CF93CDB7DEB728970FB631
:10EA2000F894DEBF0FBECDBF9A8389833B012A01D4
:10EA30001901DC82CB82BE82AD8298868F828CA146
:10EA40009DA1641775071CF42FEF3FEF36C0121617
:10EA500013061CF02EEF3FEF30C0181619061CF0FD
:10EA60002DEF3FEF2AC0019749F489819A81CB802D
:10EA7000DC80A8A0B9A08AA09BA0FDDE0F920F9217
:10EA8000EB81FC81008111818AA19BA1EDB7FEB7CA
:10EA90009283818389819A81B301A2019101ED80E2
:10EAA000FE80CF80D884AE8CBF8C88A099A00E94B5
:10EAB0003D6B20E030E00F900F90C90128960FB613
:10EAC000F894DEBF0FBECDBFCF91DF911F910F91A4
:10EAD000FF90EF90DF90CF90BF90AF909F908F907E
:10EAE0007F906F905F904F903F902F9008952F925E
:10EAF0003F924F925F926F927F928F929F92AF92CE
:10EB0000BF92CF92DF92EF92FF920F931F93DF930A
:10EB1000CF93CDB7DEB72C970FB6F894DEBF0FBEFC
:10EB2000CDBF4C016B837C835901B7D81C01C40154
:10EB30006B817C81A1010E9434622B013C010B811D
:10EB40001C817801EE0CFF1CEE0CFF1CC7010E941B
:10EB5000020B8D839E83C801880F991F0E94020BB0
:10EB60008F839887C7010E94020B89879A87C40107
:10EB7000880F991F880F991F0E94020B8B879C8713
:10EB80008DB79EB708970FB6F8949EBF0FBE8DBF86
:10EB9000CDB6DEB60894C11CD11C60E070E080E800
:10EBA00095E2A30192010E9437997B018C018B852C
:10EBB000F60180839C8591838F81828398859383DE
:10EBC000898584839A85958381E090E09783868305
:10EBD000C101B401A4012B813C816E010894C11CC8
:10EBE000D11C8D809E8006DFEDB7FEB738960FB63C
:10EBF000F894FEBF0FBEEDBFC1010E94AC0B8F8128
:10EC000098850E94AC0B89859A850E94AC0B8B85F8
:10EC10009C850E94AC0B8D819E812C960FB6F8943A
:10EC2000DEBF0FBECDBFCF91DF911F910F91FF903F
:10EC3000EF90DF90CF90BF90AF909F908F907F909C
:10EC40006F905F904F903F902F9008951092860D97
:10EC500010928D0D1092940D0895809303040895E1
:10EC6000EFE6F0E080818260808308951F93FC01CD
:10EC70001FB7F89480819181A281B38180935E0D4A
:10EC800090935F0DA093600DB093610DFB018081A7
:10EC90009181A281B3818093620D9093630DA093C3
:10ECA000640DB093650DFA0180819181A281B381D9
:10ECB0008093660D9093670DA093680DB093690DD6
:10ECC000F90180819181A281B38180936A0D909333
:10ECD0006B0DA0936C0DB0936D0D1FBF1F91089528
:10ECE000FC012FB7F89480819181A281B381809338
:10ECF0006A0D90936B0DA0936C0DB0936D0D2FBFAB
:10ED00000895E82F8FB7F894F0E0EE0FFF1FEE0F95
:10ED1000FF1FE25AF24F20813181428153818FBF20
:10ED2000B901CA010895CF93DF932FB7F894C82F84
:10ED3000D0E0CC0FDD1FCC0FDD1FFE01E25AF24FF9
:10ED400060817181828193812FBF0E94D299CB53C0
:10ED5000D84F288139814A815B810E943799DF91A0
:10ED6000CF910895E8ECF8E0949108C08091C0003C
:10ED700085FFFCCF9093C600319694919923B1F70B
:10ED8000E4ECF8E0949108C08091C00085FFFCCFCE
:10ED90009093C600319694919923B1F788E20E942E
:10EDA000F496BC018EE295E04AE050E00E94111C0E
:10EDB00089E20E94F496BC018EE295E04AE050E0C0
:10EDC0000E94111C8091C00085FFFCCF8AE08093D7
:10EDD000C600E0ECF8E0949108C08091C00085FF87
:10EDE000FCCF9093C600319694919923B1F785E4B6
:10EDF0000E94F496BC018EE295E04AE050E00E9449
:10EE0000111C87E20E94F496BC018EE295E04AE074
:10EE100050E00E94111C8091C00085FFFCCF8AE069
:10EE20008093C600ECEBF8E0949108C08091C0009C
:10EE300085FFFCCF9093C600319694919923B1F74A
:10EE400084E40E94F496BC018EE295E04AE050E032
:10EE50000E94111C83E40E94F496BC018EE295E0AE
:10EE60004AE050E00E94111C8091C00085FFFCCF59
:10EE70008AE08093C600E7EBF8E0949108C08091A7
:10EE8000C00085FFFCCF9093C600319694919923E2
:10EE9000B1F781E40E94F496BC018EE295E04AE06D
:10EEA00050E00E94111C82E40E94F496BC018EE2A4
:10EEB00095E04AE050E00E94111C8091C00085FF5F
:10EEC000FCCF8AE08093C600E2EBF8E0949108C0A2
:10EED0008091C00085FFFCCF9093C600319694913D
:10EEE0009923B1F78FE30E94F496BC018EE295E07E
:10EEF0004AE050E00E94111C80E40E94F496BC019C
:10EF00008EE295E04AE050E00E94111C8091C00022
:10EF100085FFFCCF8AE08093C60008950F931F936E
:10EF2000182F042F67FD19C0823081F0833028F438
:10EF3000882341F0813089F407C0833049F0843060
:10EF400061F408C088E207C085E405C084E403C01A
:10EF500081E401C08FE30E94C29607FD1AC01230FF
:10EF600081F0133028F4112341F0113091F407C0DF
:10EF7000133049F0143069F408C089E207C087E211
:10EF800005C083E403C082E401C080E4602F0E94D6
:10EF9000C2961F910F910895643089F0653028F46E
:10EFA000613041F0623099F407C0683051F060314F
:10EFB00071F40AC060E001C061E040E004C060E0BC
:10EFC00001C061E041E0AACF61E041E0A7CF089530
:10EFD000CF93DF938FE361E00E940F9680E461E0BE
:10EFE0000E940F9688E261E00E940F9689E261E03C
:10EFF0000E940F9685E461E00E940F9687E261E02F
:10F000000E940F9684E461E00E940F9683E461E021
:10F010000E940F9681E461E00E940F9682E461E015
:10F020000E940F96C0E0D0E0FE01EE56FB4F8C2F01
:10F030006081B2DF2196C530D105B1F7DF91CF9164
:10F0400008959B01882399F4B901882777FD80955D
:10F05000982F2FEF30E040E050E00E94E29C20ED3E
:10F0600037E040E050E00E944A9D8CE214C08130BD
:10F07000A9F4B901882777FD8095982F2FEF30E00C
:10F0800040E050E00E94E29C20ED37E040E050E09C
:10F090000E944A9D8DE2B9010C9423978230A9F415
:10F0A000B901882777FD8095982F2FEF30E040E059
:10F0B00050E00E94E29C20ED37E040E050E00E94EA
:10F0C0004A9D8EE2B9010C94239708958CE261E089
:10F0D0000E940F968DE261E00E940F968EE261E041
:10F0E0000E940F966091F7037091F80380E0A9DF0A
:10F0F0006091F9037091FA0381E0A3DF6091FB0353
:10F100007091FC0382E09DDFE1E2F1E08081887F85
:10F11000816080830895DADF5BDFEAE0F1E08081DF
:10F12000826080838081816080838081846080832D
:10F130008081806480838081806880830F9A179AA1
:10F140000E9A169A0D9A159A0C9A149A0B9A139A6B
:10F1500026982E9A25982D9A24982C9A3F98479A6B
:10F160000A98129A0998119A389A4098179A109208
:10F170005D05399A4198169A10925E053A9A42981E
:10F18000159A10925F053B9A4398149A3C9A4498BA
:10F19000A1E8B0E08C918F7E8C938C9188608C93E9
:10F1A000E0E8F0E080818D7F808380818E7F8083A6
:10F1B00080818F73808380818F7C80838C91887F16
:10F1C00082608C9380E090E4909389008093880023
:10F1D0001092850010928400EFE6F0E0808182605A
:10F1E000808381E080930304789408959091320D98
:10F1F0008091330D981729F00E94E2860E94122A0E
:10F20000F5CF0895F3DF179A10925D05169A1092C4
:10F210005E05159A10925F05149A08951F920F9239
:10F220000FB60F920BB60F921124AF92BF92CF92EE
:10F23000DF92EF92FF920F931F932F933F934F9381
:10F240005F936F937F938F939F93AF93BF93CF936E
:10F25000DF93EF93FF938091500D9091510D892B87
:10F2600009F099C19091320D8091330D981719F4DE
:10F27000E0E0F0E014C08091330D90E021E530E053
:10F28000829FF001839FF00D929FF00D1124EE5D9F
:10F29000F74FE05BFF4F81E08083E055F040F09353
:10F2A000510DE093500D309709F46FC1E05BFF4FB3
:10F2B00081E0808310929F0D1092A00D1092A10DFD
:10F2C0001092A20DE091500DF091510D60AD71AD15
:10F2D0002CE96134720718F060E47CE904C03EE474
:10F2E0006132730730F0769567957695679584E07F
:10F2F00007C047E26131740730F07695679582E088
:10F300008093980D07C08093980D6032710510F4BA
:10F3100060E270E06052704058E060307507E8F0DD
:10F32000472F50E0440F551F440F551F4A52574F67
:10F330009A012E5F3F4FF901859194919C01AA2774
:10F34000639FC001629F810D9A1F06948A1F9A1FB6
:10F350001124FA01459154911EC0CB0196958795D1
:10F360008C7F8A52934FFC0145915491FC01329657
:10F3700025913491862F90E087709070FC012E9F2C
:10F38000C0012F9F900D3E9F900D112403E0969594
:10F3900087950A95E1F7481B590B44365105A8F4A7
:10F3A000E9E2F3E007C08091C00085FFFCCF319611
:10F3B0009093C60090819923B1F78EE295E04AE0E0
:10F3C00050E00E94381C44E650E05093A40D409356
:10F3D000A30D8091980D992787FD90959093A60D88
:10F3E0008093A50DE091500DF091510D64AD75AD78
:10F3F00070939E0D60939D0DFCE961347F0718F0BA
:10F4000060E47CE904C02EE46132720730F0769546
:10F4100067957695679584E007C037E26131730799
:10F4200030F07695679582E08093980D08C081E072
:10F430008093980D6032710510F460E270E06052C4
:10F44000704048E060307407E8F0472F50E0440F08
:10F45000551F440F551F4A52574F9A012E5F3F4F79
:10F46000F901859194919C01AA27639FC001629F35
:10F47000810D9A1F06948A1F9A1F1124FA01459143
:10F4800054911EC0CB01969587958C7F8A52934FDD
:10F49000FC0145915491FC01329625913491862FBF
:10F4A00090E087709070FC012E9FC0012F9F900DFF
:10F4B0003E9F900D1124E3E096958795EA95E1F73C
:10F4C000481B590B44365105A8F4E9E2F3E007C0A4
:10F4D0008091C00085FFFCCF31969093C60090814B
:10F4E0009923B1F78EE295E04AE050E00E94381C83
:10F4F00044E650E0CA01A0E0B0E08093990D9093FB
:10F500009A0DA0939B0DB0939C0D5093890040934E
:10F510008800E091500DF091510D80899189A28968
:10F52000B389B695A79597958795B095A095909531
:10F5300081959F4FAF4FBF4F80936E0D90936F0D8E
:10F54000A093700DB093710D8093720D9093730D15
:10F55000A093740DB093750D8093760D9093770DF5
:10F56000A093780DB093790D80937A0D90937B0DD5
:10F57000A0937C0DB0937D0D10927E0D10927F0DA7
:10F580001092800D1092810D06C080ED97E090934F
:10F59000890080938800E091500DF091510D3097D3
:10F5A00009F418C680A18093820D80FF0AC08FB72E
:10F5B000F89490910B019D7F90930B018FBF8FEF7B
:10F5C00009C08FB7F89490910B01926090930B0152
:10F5D0008FBF81E08093FF038091820D81FF0AC07D
:10F5E0008FB7F89490910B01916090930B018FBFAE
:10F5F0008FEF09C08FB7F89490910B019E7F909385
:10F600000B018FBF81E0809300048091820D2091D7
:10F61000030480FF56C0222309F4A8C01E994AC0E3
:10F620008091830D882309F441C0E091500DF09141
:10F63000510D80819181A281B381181619061A0695
:10F640001B0654F52091840D3091850D8091FD03AA
:10F650009091FE0382179307F8F480915E0D9091CC
:10F660005F0DA091600DB091610D8093520D90934C
:10F67000530DA093540DB093550D81E08093860DEA
:10F6800080899189A289B38980937E0D90937F0DA3
:10F69000A093800DB093810D8091840D9091850D84
:10F6A00001969093850D8093840D60C081E08093D6
:10F6B000830D5CC01092830D1092850D1092840D05
:10F6C00055C0222309F452C037994AC08091870D52
:10F6D000882309F441C0E091500DF091510D8081D3
:10F6E0009181A281B381181619061A061B0654F5DA
:10F6F0002091880D3091890D8091FD039091FE033A
:10F7000082179307F8F480915E0D90915F0DA091A0
:10F71000600DB091610D8093520D9093530DA093A5
:10F72000540DB093550D81E08093860D80899189A9
:10F73000A289B38980937E0D90937F0DA093800D55
:10F74000B093810D8091880D9091890D01969093D1
:10F75000890D8093880D0AC081E08093870D06C0D3
:10F760001092870D1092890D1092880D8091820D54
:10F770002091030481FF56C0222309F4A8C01D99DB
:10F780004AC080918A0D882309F441C0E091500D50
:10F79000F091510D84819581A681B78118161906C3
:10F7A0001A061B0654F520918B0D30918C0D80911B
:10F7B000FD039091FE0382179307F8F48091620D88
:10F7C0009091630DA091640DB091650D8093560DDD
:10F7D0009093570DA093580DB093590D81E08093ED
:10F7E0008D0D80899189A289B38980937E0D909334
:10F7F0007F0DA093800DB093810D80918B0D909122
:10F800008C0D019690938C0D80938B0D60C081E0E0
:10F8100080938A0D5CC010928A0D10928C0D10920C
:10F820008B0D55C0222309F452C002994AC0809121
:10F830008E0D882309F441C0E091500DF091510DD7
:10F8400084819581A681B781181619061A061B06B0
:10F8500054F520918F0D3091900D8091FD03909182
:10F86000FE0382179307F8F48091620D9091630D67
:10F87000A091640DB091650D8093560D9093570D36
:10F88000A093580DB093590D81E080938D0D808920
:10F890009189A289B38980937E0D90937F0DA09367
:10F8A000800DB093810D80918F0D9091900D0196F8
:10F8B0009093900D80938F0D0AC081E080938E0D00
:10F8C00006C010928E0D1092900D10928F0D8091A7
:10F8D000820D2091030482FF61C08FB7F89490914C
:10F8E0000B019B7F90930B018FBF8FEF80930104DF
:10F8F000222309F4B1C01C994AC08091910D88233C
:10F9000009F441C0E091500DF091510D8085918531
:10F91000A285B385181619061A061B0654F5209100
:10F92000920D3091930D8091FD039091FE0382170B
:10F930009307F8F48091660D9091670DA091680D82
:10F94000B091690D80935A0D90935B0DA0935C0D5F
:10F95000B0935D0D81E08093940D80899189A28997
:10F96000B38980937E0D90937F0DA093800DB0930B
:10F97000810D8091920D9091930D01969093930D2E
:10F980008093920D69C081E08093910D65C01092C3
:10F99000910D1092930D1092920D5EC09FB7F89446
:10F9A00080910B01846080930B019FBF41E04093E5
:10F9B0000104222309F450C0019948C08091950D9B
:10F9C000882309F440C0E091500DF091510D8085DD
:10F9D0009185A285B385181619061A061B064CF5E3
:10F9E0002091960D3091970D8091FD039091FE032B
:10F9F00082179307F0F48091660D9091670DA091A6
:10FA0000680DB091690D80935A0D90935B0DA09392
:10FA10005C0DB0935D0D4093940D80899189A2890E
:10FA2000B38980937E0D90937F0DA093800DB0934A
:10FA3000810D8091960D9091970D01969093970D61
:10FA40008093960D09C04093950D06C01092950DB8
:10FA50001092970D1092960D8091820D83FF0AC02F
:10FA60008FB7F89490910B01906490930B018FBF26
:10FA70008FEF09C08FB7F89490910B019F7B909303
:10FA80000B018FBF81E08093020460E07EC1809112
:10FA9000C00087FF19C04091C600E0912A05F0918F
:10FAA0002B0531969F012F773070319780912C056F
:10FAB00090912D052817390739F0E655FB4F408303
:10FAC00030932B0520932A05E091500DF091510DB4
:10FAD000208131814281538180916E0D90916F0D13
:10FAE000A091700DB091710D280F391F4A1F5B1F37
:10FAF00020936E0D30936F0D4093700D5093710DE8
:10FB000012161306140615066CF5409A8089918921
:10FB1000A289B389281B390B4A0B5B0B20936E0D0E
:10FB200030936F0D4093700D5093710D20915E0DC9
:10FB300030915F0D4091600D5091610D8091FF03F8
:10FB4000992787FD9095A92FB92F820F931FA41F86
:10FB5000B51F80935E0D90935F0DA093600DB093E1
:10FB6000610D4098E091500DF091510D2481358147
:10FB7000468157818091720D9091730DA091740D03
:10FB8000B091750D280F391F4A1F5B1F2093720D0E
:10FB90003093730D4093740D5093750D1216130628
:10FBA000140615066CF5419A80899189A289B3895A
:10FBB000281B390B4A0B5B0B2093720D3093730D8E
:10FBC0004093740D5093750D2091620D3091630D2B
:10FBD0004091640D5091650D80910004992787FD37
:10FBE0009095A92FB92F820F931FA41FB51F809343
:10FBF000620D9093630DA093640DB093650D4198D1
:10FC0000E091500DF091510D20853185428553854D
:10FC10008091760D9091770DA091780DB091790D2E
:10FC2000280F391F4A1F5B1F2093760D3093770DE5
:10FC30004093780D5093790D12161306140615068D
:10FC40006CF5429A80899189A289B389281B390B66
:10FC50004A0B5B0B2093760D3093770D4093780D14
:10FC60005093790D2091660D3091670D4091680D8C
:10FC70005091690D80910104992787FD9095A92FD6
:10FC8000B92F820F931FA41FB51F8093660D909309
:10FC9000670DA093680DB093690D4298E091500DE7
:10FCA000F091510D248535854685578580917A0DD3
:10FCB00090917B0DA0917C0DB0917D0D280F391F87
:10FCC0004A1F5B1F20937A0D30937B0D40937C0D70
:10FCD00050937D0D12161306140615066CF5439A03
:10FCE00080899189A289B389281B390B4A0B5B0B48
:10FCF00020937A0D30937B0D40937C0D50937D0DB6
:10FD000020916A0D30916B0D40916C0D50916D0DED
:10FD100080910204992787FD9095A92FB92F820F12
:10FD2000931FA41FB51F80936A0D90936B0DA09332
:10FD30006C0DB0936D0D439880917E0D90917F0D69
:10FD4000A091800DB091810D0196A11DB11D8093F0
:10FD50007E0D90937F0DA093800DB093810D209127
:10FD60007E0D30917F0D4091800D5091810DE0917D
:10FD7000500DF091510D80899189A289B38928177E
:10FD800039074A075B0730F46F5F8091980D681759
:10FD90000CF47DCE20917E0D30917F0D4091800D31
:10FDA0005091810DE091500DF091510D848995890C
:10FDB000A689B78982179307A407B50708F4E3C09B
:10FDC000E090990DF0909A0D00919B0D10919C0D73
:10FDD000A48CB58CC68CD78CA8019701C601B5013F
:10FDE000AA27279FB12D389FE001489FD00D479F3C
:10FDF000C00DD11D289FB00DC11DDA1F379FB00D5A
:10FE0000C11DDA1F469FB00DC11DDA1F369FB10D0F
:10FE1000CA1FDA1FB695CA1FDA1F112484AD95AD2B
:10FE20008C0F9D1F90939E0D80939D0D20AD31AD45
:10FE300042AD53ADA0E0B0E0281739074A075B0791
:10FE400020F430939E0D20939D0D60919D0D709137
:10FE50009E0D8CE96134780718F060E47CE904C0F9
:10FE60009EE46132790730F07695679576956795CF
:10FE700084E007C0E7E261317E0730F07695679550
:10FE800082E08093980D08C081E08093980D6032E5
:10FE9000710510F460E270E060527040F8E060308C
:10FEA0007F07E8F0472F50E0440F551F440F551FC0
:10FEB0004A52574F9A012E5F3F4FF9018591949115
:10FEC0009C01AA27639FC001629F810D9A1F06941F
:10FED0008A1F9A1F1124FA01459154911EC0CB012B
:10FEE000969587958C7F8A52934FFC01459154914A
:10FEF000FC01329625913491862F90E087709070A6
:10FF0000FC012E9FC0012F9F900D3E9F900D11244C
:10FF100003E0969587950A95E1F7481B590B4436FF
:10FF20005105A8F4E9E2F3E007C08091C00085FF25
:10FF3000FCCF31969093C60090819923B1F78EE261
:10FF400095E04AE050E00E94381C44E650E05093AF
:10FF50008900409388009A0140E050E08091990D1B
:10FF600090919A0DA0919B0DB0919C0D820F931FC3
:10FF7000A41FB51F8093990D90939A0DA0939B0D8C
:10FF8000B0939C0D02C120917E0D30917F0D409168
:10FF9000800D5091810D808D918DA28DB38D821732
:10FFA0009307A407B50708F0E4C060919F0D709116
:10FFB000A00D8091A10D9091A20D248D358D468DBF
:10FFC000578DAA27639FB12D749FE001849FD00DA8
:10FFD000839FC00DD11D649FB00DC11DDA1F739F9B
:10FFE000B00DC11DDA1F829FB00DC11DDA1F729FB7
:10FFF000B10DCA1FDA1FB695CA1FDA1F11248091EE
:020000021000EC
:100000009D0D90919E0D8C179D0738F4E05CFF4F7D
:1000100060817181E054F04003C0BC016C1B7D0B1A
:10002000E05CFF4F2081318142815381CB01A0E010
:10003000B0E082179307A407B50708F4B901FCE9FB
:1000400061347F0718F060E47CE904C02EE461327B
:10005000720730F0769567957695679584E007C0CE
:1000600037E26131730730F07695679582E08093CF
:10007000980D08C081E08093980D6032710510F4EE
:1000800060E270E06052704048E060307407E8F071
:10009000472F50E0440F551F440F551F4A52574FEA
:1000A0009A012E5F3F4FF901859194919C01AA27F7
:1000B000639FC001629F810D9A1F06948A1F9A1F39
:1000C0001124FA01459154911EC0CB019695879554
:1000D0008C7F8A52934FFC0145915491FC013296DA
:1000E00025913491862F90E087709070FC012E9FAF
:1000F000C0012F9F900D3E9F900D1124E3E0969537
:100100008795EA95E1F7481B590B44365105A8F449
:10011000E9E2F3E007C08091C00085FFFCCF319693
:100120009093C60090819923B1F78EE295E04AE062
:1001300050E00E94381C44E650E050938900409300
:1001400088009A0140E050E080919F0D9091A00DB1
:10015000A091A10DB091A20D820F931FA41FB51FF6
:1001600080939F0D9093A00DA093A10DB093A20D2D
:100170000CC08091A30D9091A40D90938900809361
:1001800088008091A50D8093980D20917E0D30916F
:100190007F0D4091800D5091810DE091500DF091B7
:1001A000510D80899189A289B389281739074A0797
:1001B0005B0780F01092510D1092500D9091320D0E
:1001C0008091330D981731F08091330D8F5F8F70D0
:1001D0008093330DFF91EF91DF91CF91BF91AF915C
:1001E0009F918F917F916F915F914F913F912F914F
:1001F0001F910F91FF90EF90DF90CF90BF90AF9045
:100200000F900BBE0F900FBE0F901F90189580910E
:10021000860D882349F480918D0D882329F48091DF
:10022000940D882309F490C0E6EDF0E1949108C0A4
:100230008091C00085FFFCCF9093C60031969491C9
:100240009923B1F7E8EEF0E1949108C08091C000E5
:1002500085FFFCCF9093C600319694919923B1F716
:100260008091860D8823D1F06091520D7091530DCD
:100270008091540D9091550D0E94D2992091C507FF
:100280003091C6074091C7075091C8070E9437991F
:10029000AB01BC0184EE90E10E94092180918D0D9B
:1002A0008823D1F06091560D7091570D8091580DB3
:1002B0009091590D0E94D2992091C9073091CA0797
:1002C0004091CB075091CC070E943799AB01BC01FC
:1002D00080EE90E10E9409218091940D8823D1F055
:1002E00060915A0D70915B0D80915C0D90915D0D48
:1002F0000E94D2992091CD073091CE074091CF072F
:100300005091D0070E943799AB01BC018CED90E170
:100310000E940921EDE3F3E007C08091C00085FF52
:10032000FCCF31969093C60090819923B1F78091CC
:10033000C00085FFFCCF8AE08093C6001092860D36
:1003400010928D0D1092940D089560E070E08CE590
:1003500093E4209108043091090440910A045091DB
:100360000B040E9437996093D50D7093D60D80933E
:10037000D70D9093D80D60E070E08CE593E4209168
:1003800018043091190440911A0450911B040E94E2
:1003900037996093DD0D7093DE0D8093DF0D9093A0
:1003A000E00D0895FC0197FF03C08091B70D03C0D5
:1003B000E854F24F808190E008952F923F924F923F
:1003C0005F926F927F928F929F92AF92BF92CF92E5
:1003D000DF92EF92FF920F931F93CF93DF93EC0185
:1003E00021E030E0A901440F551F440F551FFA01C9
:1003F000E155FE4E85919491C817D9070CF059C06C
:10040000B90161507040660F771F660F771FCB01EF
:100410008F549E4EFC010591149161557E4EFB0157
:10042000C590D490FA01EF54FE4EE590F490FA0195
:10043000E155FE4EA590B490B801882777FD8095D0
:10044000982F0E94D2991B012C01CC19DD09BE0105
:10045000882777FD8095982F0E94D2993B014C0107
:10046000E01AF10A0027F7FC0095102FC801B70128
:100470000E94D2999B01AC01C401B3010E94109C5F
:100480007B018C01AC18BD08CC24B7FCC094DC2CDB
:10049000C601B5010E94D2999B01AC01C801B70108
:1004A0000E9437999B01AC01C201B1010E9457988B
:1004B00019C0822F8F5F2F5F3F4F2A33310509F01C
:1004C00091CF8A3329F0E0E070E080E060E00CC07A
:1004D000E5E9F2E165917491882777FD8095982F81
:1004E0000E94D299E62F692F2E2F372F482F562F93
:1004F000B901CA01DF91CF911F910F91FF90EF9049
:10050000DF90CF90BF90AF909F908F907F906F9033
:100510005F904F903F902F90089508951092A80DEE
:100520001092A70D1092B80D75981092AA0D109206
:10053000A90D1092B90D9FB7F894E2E0F1E0808127
:100540008F7E80839FBF1092AA0D1092A90D1092EA
:10055000B70DA59808952DEB37E346E05EE30C94C4
:10056000109C2DEB37E346E05EE30C9437992DEBBE
:1005700037E346E05EE30C9437992DEB37E346E032
:100580005EE30C94109CA5980E94361D882319F5F3
:10059000E7EFF0E1949108C08091C00085FFFCCFA7
:1005A0009093C600319694919923B1F7EEEFF0E164
:1005B000949108C08091C00085FFFCCF9093C60045
:1005C000319694919923B1F78091C00085FFFCCFBB
:1005D0008AE08093C6000C947D1D1F93182F9EDF28
:1005E0000E94361D882391F5E7EFF0E1949108C051
:1005F0008091C00085FFFCCF9093C6003196949106
:100600009923B1F78EE295E0612F70E04AE050E067
:100610000E94111C8091C00085FFFCCF8AE080936E
:10062000C600E8E3F1E1949108C08091C00085FF25
:10063000FCCF9093C600319694919923B1F78091A5
:10064000C00085FFFCCF8AE08093C6000E947D1D1C
:100650001F9108951F93182F61DF0E94361D882374
:1006600091F5E7EFF0E1949108C08091C00085FF1B
:10067000FCCF9093C600319694919923B1F78EE206
:1006800095E0612F70E04AE050E00E94111C8091DB
:10069000C00085FFFCCF8AE08093C600E5E6F1E16B
:1006A000949108C08091C00085FFFCCF9093C60054
:1006B000319694919923B1F78091C00085FFFCCFCA
:1006C0008AE08093C6000E947D1D1F9108951F92AD
:1006D0000F920FB60F920BB60F9211242F933F93E8
:1006E0004F935F936F937F938F939F93AF93BF933A
:1006F000EF93FF9390912204992391F48091B80D88
:100700008093BF0D882311F0759A01C07598809170
:10071000B70D8093BE0D882311F0A59A01C0A5984E
:100720008091BF0D891708F475988091BE0D8917C7
:1007300008F4A5989F5F9F779093220480912304EB
:10074000843009F46BC0853050F4813009F1813078
:1007500098F08230D9F1833009F094C043C08630DC
:1007600009F484C0863008F465C0873009F480C07D
:10077000883009F087C084C010927B0080E48093A9
:100780007C0080917A00806480937A0081E01BC0B5
:100790008091780090917900A0E0B0E02091CC0D9C
:1007A0003091CD0D4091CE0D5091CF0D280F391FB6
:1007B0004A1F5B1F2093CC0D3093CD0D4093CE0D7F
:1007C0005093CF0D82E0809323045CC010927B0095
:1007D00082E480937C0080917A00806480937A0028
:1007E00083E0F1CF8091780090917900A0E0B0E0B3
:1007F0002091C00D3091C10D4091C20D5091C30D9B
:10080000280F391F4A1F5B1F2093C00D3093C10D65
:100810004093C20D5093C30D84E0D5CF10927B005E
:1008200081E480937C0080917A00806480937A00D8
:1008300085E0C9CF8091780090917900A0E0B0E088
:100840002091C80D3091C90D4091CA0D5091CB0D2A
:10085000280F391F4A1F5B1F2093C80D3093C90D05
:100860004093CA0D5093CB0D86E0ADCF87E0ABCF60
:10087000109223048091D00D8F5F8093D00D02C021
:10088000109223048091D00D803108F463C08091D0
:10089000B90D882381F48091CC0D9091CD0D90936A
:1008A000AC0D8093AB0D8091C00D9091C10D9093D4
:1008B000B20D8093B10D81E08093B90D1092D00DEF
:1008C0001092CC0D1092CD0D1092CE0D1092CF0D36
:1008D0001092C80D1092C90D1092CA0D1092CB0D36
:1008E0001092C40D1092C50D1092C60D1092C70D36
:1008F0001092C00D1092C10D1092C20D1092C30D36
:100900002091AB0D3091AC0D8091BA0D9091BB0D43
:100910008217930714F080E09DDE2091AB0D30919B
:10092000AC0D80912004909121042817390714F010
:1009300080E053DE2091B10D3091B20D8091BC0D5D
:100940009091BD0D821793072CF01092AA0D109272
:10095000A90D19DEFF91EF91BF91AF919F918F91FA
:100960007F916F915F914F913F912F910F900BBEAF
:100970000F900FBE0F901F9018952F926F927F923D
:100980008F929F92AF92BF92CF92DF92EF92FF929F
:100990000F931F93DF93CF93CDB7DEB729970FB691
:1009A000F894DEBF0FBECDBF8C01E62E662369F141
:1009B000E7EFF0E1949108C08091C00085FFFCCF83
:1009C0009093C600319694919923B1F78EE295E009
:1009D0006E2D70E04AE050E00E94111CE2E9F1E166
:1009E000949108C08091C00085FFFCCF9093C60011
:1009F000319694919923B1F78091C00085FFFCCF87
:100A00008AE08093C6000E94BB1DAE2DB0E0FD01C0
:100A1000EE0FFF1FE956FB4F608171817987688770
:100A2000672B09F49FC0A756BB4F7C917B83222480
:100A3000239479C0222D30E0A901440F551F440FA3
:100A4000551FE885F985E40FF51F859194910817E6
:100A500019070CF067C0C9010197880F991F880F0B
:100A6000991FFC013296A885B985EA0FFB1FC59036
:100A7000D4908A0F9B1FFC01659174917A836983DE
:100A8000FA013296EA0FFB1FE590F490FD01E40FA6
:100A9000F51FA590B490B601882777FD8095982F13
:100AA0000E94D2996C837D838E839F8389819A81F2
:100AB000081B190BB801882777FD8095982F0E9495
:100AC000D2993B014C01EC18FD080027F7FC00957A
:100AD000102FC801B7010E94D2999B01AC01C4013B
:100AE000B3010E94109C7B018C01A981BA81AA1AD2
:100AF000BB0ACC24B7FCC094DC2CC601B5010E9413
:100B0000D2999B01AC01C801B7010E9437999B01A2
:100B1000AC016C817D818E819F810E945798E62F68
:100B2000692F09C02394BB812B1608F483CFE0E022
:100B300070E080E060E0FB812F1679F5E22DF0E0B7
:100B4000EE0FFF1FEE0FFF1F329768857985E60FC6
:100B5000F71F65917491882777FD8095982F0E94E3
:100B6000D29919C0B801882777FD8095982F0E94E7
:100B7000D29920E030E04AEF5EE30E94109C20E032
:100B800030E040E85DE30E94109C20E030E040E06F
:100B900050E00E945798E62F692F2E2F372F482FAD
:100BA000562FB901CA0129960FB6F894DEBF0FBEC1
:100BB000CDBFCF91DF911F910F91FF90EF90DF900C
:100BC000CF90BF90AF909F908F907F906F902F901D
:100BD0000895EF92FF920F931F93CF93DF930F2E01
:100BE000F0E0EF2EF0E0FF2EF0E00F2FF0E01F2FEF
:100BF000F02DE092D10DF092D20D0093D30D109311
:100C0000D40D60E070E08CE593E42091080430910D
:100C1000090440910A0450910B040E943799609393
:100C2000D50D7093D60D8093D70D9093D80DE0928B
:100C3000D90DF092DA0D0093DB0D1093DC0D60E01E
:100C400070E08CE593E420911804309119044091F0
:100C50001A0450911B040E9437996093DD0D709324
:100C6000DE0D8093DF0D9093E00D6D9A8091010170
:100C70008061809301019D9A80910101806280933F
:100C8000010188E061E070E00E94391D87ED8093EA
:100C90007A0010927E0010927D0080917E0081602B
:100CA00080937E0080917E00826080937E008091A0
:100CB0007E00846080937E0080E888BD80916E0015
:100CC000846080936E006AEF70E080E090E00E94A4
:100CD000549585E090E09093E20D8093E10D09C07A
:100CE0008091200490912104409790932104809357
:100CF0002004809120049091210460E03EDE20E0F9
:100D000030E040EA50E40E94309987FDE9CF81E36A
:100D100091E0909325048093240409C08091BA0D3A
:100D20009091BB0D40969093BB0D8093BA0D80912E
:100D3000BA0D9091BB0D60E020DE20E030E848E97C
:100D400053E40E943E9B18164CF3C091BC0DD09109
:100D5000BD0DEC2E1D2FCE0130DB609620E030E083
:100D600046E153E40E943E9B18169CF3E092BC0DB2
:100D70001093BD0DDF91CF911F910F91FF90EF90D8
:100D800008958091AB0D9091AC0D60E0F6DD60931D
:100D9000AD0D7093AE0D8093AF0D9093B00D80911B
:100DA000B10D9091B20D09DB6093B30D7093B40D4A
:100DB0008093B50D9093B60D8FB7F8941092B90D3E
:100DC0008FBF08952F923F924F925F926F927F92C2
:100DD0008F929F92AF92BF92CF92DF92EF92FF924B
:100DE0000F931F938091B90D882309F478C2C9DF4E
:100DF0006090AD0D7090AE0D8090AF0D9090B00DE5
:100E0000C090A70DD090A80DB601882777FD8095DA
:100E1000982F0E94D299A40193010E9456987B01B9
:100E20008C016093E30D7093E40D8093E50D909336
:100E3000E60D20E030E040E851E40E943E9B1816A9
:100E400074F481E08093E70D0F2EF0E0EF2EF0E0D8
:100E5000FF2EFCE50F2FF3E41F2FF02DF3C0C80188
:100E6000B70120E030E040E851EC0E94309987FD66
:100E700002C0CD2821F481E08093E70DC4C08091A9
:100E8000E70D882371F080E090E0A0E0B0E080936F
:100E9000E80D9093E90DA093EA0DB093EB0D10923D
:100EA000E70DC801B7012091040430910504409179
:100EB0000604509107040E94109C1B012C016093B2
:100EC000EC0D7093ED0D8093EE0D9093EF0DC80136
:100ED000B7012091E80D3091E90D4091EA0D509154
:100EE000EB0D0E9457985B016C01E090D10DF090E2
:100EF000D20D0091D30D1091D40DA80197010E943D
:100F0000309987FD12C0E090D50DF090D60D00917C
:100F1000D70D1091D80DC601B501A80197010E9407
:100F20003E9B181614F086017501E092E80DF092D0
:100F3000E90D0093EA0D1093EB0DC801B701209164
:100F400008043091090440910A0450910B040E9456
:100F5000109C5B016C016093F00D7093F10D809318
:100F6000F20D9093F30DC401B3012091F40D309173
:100F7000F50D4091F60D5091F70D0E945698209175
:100F80000C0430910D0440910E0450910F040E9406
:100F9000109C20ED3CEC4CE45DE30E94109C7B0136
:100FA0008C016091F80D7091F90D8091FA0D90917E
:100FB000FB0D23E333E343E75FE30E94109C9B01B7
:100FC000AC01C801B7010E9457987B018C01609366
:100FD000F80D7093F90D8093FA0D9093FB0DC201FB
:100FE000B101A60195010E945798A80197010E949E
:100FF00056987B018C0120E030E040E050E00E94F8
:10100000309988235CF40F2EF0E0EF2EF0E0FF2EF5
:10101000F0E00F2FF0E01F2FF02D14C0C801B70132
:1010200020E030E041E653E40E943E9B181654F461
:101030000F2EF0E0EF2EF0E0FF2EF1E60F2FF3E49D
:101040001F2FF02D6092F40D7092F50D8092F60D29
:101050009092F70D6091E10D7091E20D882777FD78
:101060008095982F0E94D2999B01AC01C401B301D5
:101070000E943E9B1816DCF46091240470912504B4
:10108000882777FD8095982F0E94D2999B01AC010B
:10109000C401B3010E94309988234CF4C801B70100
:1010A0000E949F99759567956093B80D02C0109244
:1010B000B80D6090B30D7090B40D8090B50D909008
:1010C000B60D6091A90D7091AA0D882777FD8095C6
:1010D000982F0E94D299A40193010E9456987B01F7
:1010E0008C016093FC0D7093FD0D8093FE0D909329
:1010F000FF0D209114043091150440911604509175
:1011000017040E94109C1B012C016093000E709329
:10111000010E8093020E9093030EC801B701209137
:10112000040E3091050E4091060E5091070E0E945C
:1011300057985B016C01E090D90DF090DA0D0091A9
:10114000DB0D1091DC0DA80197010E94309987FDFD
:1011500012C0E090DD0DF090DE0D0091DF0D1091DA
:10116000E00DC601B501A80197010E943E9B18162B
:1011700014F086017501E092040EF092050E0093C2
:10118000060E1093070EC801B70120911804309184
:10119000190440911A0450911B040E94109C5B0199
:1011A0006C016093080E7093090E80930A0E909361
:1011B0000B0EC401B30120910C0E30910D0E409125
:1011C0000E0E50910F0E0E94569820911C043091E3
:1011D0001D0440911E0450911F040E94109C20ED9C
:1011E0003CEC4CE45DE30E94109C7B018C0160911F
:1011F000100E7091110E8091120E9091130E23E338
:1012000033E343E75FE30E94109C9B01AC01C801FC
:10121000B7010E9457987B018C016093100E709368
:10122000110E8093120E9093130E60920C0E70921A
:101230000D0E80920E0E90920F0EC201B101A6010A
:1012400095010E945798A80197010E9456987B012A
:101250008C0120E030E040E050E00E94309988238B
:101260005CF40F2EF0E0EF2EF0E0FF2EF0E00F2FF9
:10127000F0E01F2FF02D14C0C801B70120E030E0CE
:101280004FE753E40E943E9B181654F40F2EF0E0F3
:10129000EF2EF0E0FF2EFFE70F2FF3E41F2FF02DCE
:1012A000C401B30120E030E040EA50E40E943E9BDC
:1012B00018169CF4C401B30120E030E046E153E489
:1012C0000E94309988234CF4C801B7010E949F996D
:1012D000759567956093B70D02C01092B70D1F9179
:1012E0000F91FF90EF90DF90CF90BF90AF909F90C5
:1012F0008F907F906F905F904F903F902F900895C8
:101300002F923F924F925F926F927F928F929F9215
:10131000AF92BF92CF92DF92EF92FF920F931F9303
:10132000DF93CF93CDB7DEB7E6970FB6F894DEBF65
:101330000FBECDBF6C8F7D8F8E8F9F8F5EAB4DAB01
:1013400039A328A30E944695698B7A8B8B8B9C8B43
:101350002DA93EA9223031051CF4EEE3F3E019C0BB
:10136000E1E5F3E007C08091C00085FFFCCF319636
:101370009093C60090819923B1F78091C00085FFBA
:10138000FCCF43C48091C00085FFFCCF3196909381
:10139000C60090819923B1F78091C00085FFFCCFF2
:1013A0008AE08093C600BAD84DA95EA957FF0EC047
:1013B0008FE78093B70D2FE7A22EB12CC12CD12C33
:1013C0009FE7292E312C412C512C10C0EDA9FEA9EC
:1013D000E854F24F80E7808380E7A82EB12CC12C1F
:1013E000D12C00E7202E312C412C512C89899A894F
:1013F000AB89BC898D879E87AF87B88B89879A8791
:10140000AB87BC8719AA1AAA1BAA1CAA1F8A1E8A04
:1014100091E09D8B1D821E821F82188620E030E0A5
:1014200040E050E029833A834B835C830F2EF0E049
:101430006F2EF0E47F2EFCE18F2EF6E49F2EF02D30
:101440004DA95EA94854524F5BA34AA3E8E7F3E1D4
:1014500054915CA3E3E7F3E184918DA3ECE6F3E11F
:1014600094919EA3E5E6F3E1A491AFA3EFE5F3E148
:10147000B491B8A7E9E5F3E1249129A7ECE4F3E1FD
:1014800034913AA7E6E4F3E144914BA7E0E4F3E1B9
:1014900054915CA7EAE3F3E184918DA7ADA9BEA9BD
:1014A000AA0FBB1FAA0FBB1FA355B24FBFA7AEA762
:1014B000E0E0F3E1B491B8AB8091B90D882309F471
:1014C000CDC25FDCEDA9FEA9F7FF0DC0F091B30D11
:1014D000F9AB2091B40D2AAB3091B50D3BAB4091E7
:1014E000B60D4CAB11C0AEA5BFA5BC91B9ABEEA576
:1014F000FFA5F181FAABAEA5BFA51296BC91BBAB1F
:10150000EEA5FFA5F381FCAB69817A818B819C817B
:1015100029A93AA94BA95CA90E943E9B181644F040
:1015200089A99AA9ABA9BCA989839A83AB83BC83F7
:10153000C401B30129A93AA94BA95CA90E94309919
:1015400087FD06C089A99AA9ABA9BCA93C014D0198
:101550002D89222309F451C069A97AA98BA99CA9D4
:101560002C8D3D8D4E8D5F8D0E943E9B18160CF08C
:1015700075C20E94469529853A854B855C85621B1C
:10158000730B840B950B695873418040904008F4AD
:1015900065C2D601C50182199309A409B5094DA9EF
:1015A0005EA957FF07C0B595A79597958795809336
:1015B000B70D07C0B595A79597958795EAA1FBA1AB
:1015C00080830E9446956D877E878F87988B9B01CD
:1015D000AC0189859A85AB85BC85281B390B4A0BE4
:1015E0005B0B2D833E834F8358872C8D3D8D4E8D15
:1015F0005F8D29833A834B835C8369A97AA98BA980
:101600009CA92C8D3D8D4E8D5F8D0E943099882335
:101610000CF023C20E9446952D853E854F85588942
:10162000621B730B840B950B69587341804090408B
:1016300008F413C20E94469569877A878B879C8736
:101640004E895F89452B09F4E3C1DC01CB012D856F
:101650003E854F855889821B930BA40BB50B2D81BA
:101660003E814F815885280F391F4A1F5B1F288FE5
:10167000398F4A8F5B8F2D813E814F815885281B82
:10168000390B4A0B5B0BCA01B901A20191010E94FF
:10169000E29C288D398D4A8D5B8D0E944A9DA20E59
:1016A000B31EC41ED51E34E1A316B104C104D10477
:1016B00034F14DA95EA957FD05C08DEC90E0A0E086
:1016C000B0E004C08BEE90E0A0E0B0E08A159B058E
:1016D000AC05BD05CCF48DA99EA997FD0AC020EEEE
:1016E00030E040E050E07DECA72EB12CC12CD12C95
:1016F0002DC06BEEA62EB12CC12CD12C0EC054E106
:10170000A52EB12CC12CD12CADA9BEA9B7FD05C009
:1017100080E790E0A0E0B0E004C08FE790E0A0E0B8
:10172000B0E08A159B05AC05BD051CF0150126012E
:1017300013C0EDA9FEA9F7FD05C020EE30E040E0A2
:1017400050E004C02EEF30E040E050E019012A01E3
:101750002A183B084C085D089CA1E8E7F3E108C0A3
:101760008091C00085FFFCCF9093C6003196949184
:101770009923B1F78EE295E0B601A5012AE030E0A9
:101780000E94DE1B9DA1E3E7F3E108C08091C00049
:1017900085FFFCCF9093C600319694919923B1F7C1
:1017A0008EE295E0B201A1012AE030E00E94DE1B4A
:1017B0009EA1ECE6F3E108C08091C00085FFFCCF5C
:1017C0009093C600319694919923B1F78EE295E0FB
:1017D000B401A30122E030E00E94E41C9FA1E5E6F1
:1017E000F3E108C08091C00085FFFCCF9093C60054
:1017F000319694919923B1F78EE295E049815A810F
:101800006B817C8122E030E00E94E41C8091C0006A
:1018100085FFFCCF8AE08093C6002E893F89233064
:1018200031050CF4F5C0C201B1010E94D29920E04B
:1018300030E040E850E40E94109C7B018C016981FB
:101840007A818B819C81A40193010E94569820ED9E
:101850003FE049E450E40E94109C20E030E040E08A
:101860005FE30E94109C9B01AC01C801B7010E947C
:1018700037997B018C01688D798D8A8D9B8D0E94B3
:10188000D29920E030E04AE754E40E9437993B01C6
:101890004C0198A5EFE5F3E108C08091C00085FFF9
:1018A000FCCF9093C600319694919923B1F78EE2C4
:1018B00095E0B801A70122E030E00E94E41C99A560
:1018C000E9E5F3E108C08091C00085FFFCCF90936B
:1018D000C600319694919923B1F78EE295E0B40158
:1018E000A30122E030E00E94E41C8091C00085FF4B
:1018F000FCCF8AE08093C600C801B7012AE939E924
:1019000049E15FE30E94109C7B018C019AA5ECE405
:10191000F3E108C08091C00085FFFCCF9093C60022
:10192000319694919923B1F78091C00085FFFCCF47
:101930008AE08093C6009BA5E6E4F3E108C08091AD
:10194000C00085FFFCCF9093C600319694919923F7
:10195000B1F78EE295E0B801A70122E030E00E94E5
:10196000E41C8091C00085FFFCCF8AE08093C60014
:101970009CA5E0E4F3E108C08091C00085FFFCCFA6
:101980009093C600319694919923B1F7C801B7019D
:10199000A80197010E945798A40193010E943799CA
:1019A000AB01BC018EE295E022E030E00E94E41C35
:1019B0008091C00085FFFCCF8AE08093C6009DA582
:1019C000EAE3F3E108C08091C00085FFFCCF90936B
:1019D000C600319694919923B1F7C801B701A401CB
:1019E00093010E94109C20E030E040E05EE30E9402
:1019F000109CAB01BC018EE295E022E030E00E9439
:101A0000E41C8091C00085FFFCCF8AE08093C60073
:101A1000D201C1018A0D9B1DAC1DBD1D4DA95EA942
:101A200057FF07C0B595A795979587958093B70DF4
:101A300007C0B595A79597958795EAA1FBA18083E7
:101A40002E893F892F5F3F4F3F8B2E8B6C8C7D8C77
:101A50008E8C9F8C31E03D8B01C01D8A6C8D7D8DFD
:101A60008E8D9F8D20E030E040EA51E40E9457982F
:101A70009B01AC0169A97AA98BA99CA90E943E9BF4
:101A800018169CF4E0E1F3E1949108C08091C00045
:101A900085FFFCCF9093C600319694919923B1F7BE
:101AA0008091C00085FFFCCFB0C0F0D729893A896A
:101AB0004B895C89621B730B840B950B615D7740CE
:101AC0008040904008F453C04DA95EA957FF11C053
:101AD0006091B70DEAE0F3E1949108C08091C000F5
:101AE00085FFFCCF9093C600319694919923B1F76E
:101AF00011C0AAA1BBA16C91E4E0F3E1949108C0EC
:101B00008091C00085FFFCCF9093C60031969491E0
:101B10009923B1F7162F8EE295E049A95AA96BA92E
:101B20007CA922E030E00E94E41C98A9E0E0F3E107
:101B300008C08091C00085FFFCCF9093C60031960D
:101B400094919923B1F78EE295E0612F70E04AE01D
:101B500050E00E94111C8091C00085FFFCCF8AE0FC
:101B60008093C60093D7698B7A8B8B8B9C8B8ED797
:101B70007B018C018BD72D853E854F855889E21AD4
:101B8000F30A040B150B29853A854B855C85E21A0F
:101B9000F30A040B150BE60EF71E081F191F31E898
:101BA000E3163FE4F30632E1030730E0130798F051
:101BB000E3EEF2E1949108C08091C00085FFFCCF74
:101BC0009093C600319694919923B1F78091C0000B
:101BD00085FFFCCF1AC04E895F8988A199A184171F
:101BE00095070CF069CCE7E9F2E1949108C0809187
:101BF000C00085FFFCCF9093C60031969491992345
:101C0000B1F78091C00085FFFCCF8AE08093C600C9
